:020000040800F2
:100000000080002055F900084D060108F53600086B
:100010004F060108510601085306010800000000C0
:100020000000000000000000000000009127000810
:100030005506010800000000212800086528000876
:1000400057060108590601085B0601085D0601080C
:100050005F06010861060108E1050108E7050108DE
:10006000ED050108F3050108F9050108630601081B
:100070006506010867060108690601086B060108A4
:100080006D0601086F060108710601087306010874
:10009000750601087706010879060108FF050108C1
:1000A0007B0601087D0601087F060108810601081C
:1000B00083060108850601088706010889060108EC
:1000C0008B0601088D0601088F06010891060108BC
:1000D00093060108510D0108310F0108950601082A
:1000E00023060108CD0601089706010899060108B4
:1000F0009B06010800000000000000000000000056
:1001000000000000000000005FF808F110B5054C89
:10011000237833B9044B13B10448AFF300800123B3
:10012000237010BDC005002000000000B8F50108D4
:1001300008B5034B1BB103490348AFF3008008BD6A
:1001400000000000C4050020B8F5010810B5044601
:10015000C06910B1012109F047FB206910B10121EC
:1001600009F042FB204610BD2DE9F04385B004F0B4
:10017000F9FF424C054694F850301BB11C21404811
:1001800003F026FA4FF000083E4F04AE284606F86A
:10019000058D04F067FB284607F0EAFA3B1F32465C
:1001A00039492846009704F09FFE384804AA42F8CF
:1001B000048D07F12001206209F0BEFF039B1BB1F3
:1001C0005421334803F004FADFF8FC90DFF8FC8098
:1001D000304B324630492846CDF80490CDF80080A7
:1001E00004F052FE2D492846CDF80490CDF8008049
:1001F0002B4B324604F048FE616C206C16F0C8F8B8
:1002000028B128480AF0C4F901238DF80B30DFF833
:10021000C090DFF8C080244B324624492846CDF8F0
:100220000490CDF8008004F02FFE21492846CDF837
:100230000490CDF800801F4B324604F025FEE16C9F
:10024000A06C16F0A5F828B11B480AF0A1F901230B
:100250008DF80B309DF80B302BB118480AF098F947
:10026000102010F058FF164B164A9F621A610123A6
:1002700084F8503005B0BDE8F08300BFDC050020F5
:1002800081960108E0050020C1960108CA96010880
:10029000D69601081C060020169701081F97010832
:1002A0002006002028970108240600205597010801
:1002B0005F970108280600206997010898970108B0
:1002C000080000200006002000007A4400007AC4E4
:1002D00000247449002474C9F8B50025C0E901124E
:1002E0000570C0E90335C0E90555C0E90755456209
:1002F00006990446164600F11C0703F02BFD38B999
:10030000314607480AF044F92021064803F060F915
:10031000069A3946204603F007FD2046F8BD00BF87
:10032000AB970108D697010830B58DB004F01AFFDD
:10033000044600F045FD214608F058FA0322002348
:100340000392354D354A364902A88DF80830049598
:10035000CDE90523CDE90733CDE909330B9303F04C
:10036000DDFD38B929462F480AF012F920212E4820
:1003700003F02EF92A4A09A902A803F097FD02A961
:10038000204604F095FF02A8FFF7E0FE0023274A6D
:1003900000930221264B02A8FFF79EFF02A92046E8
:1003A00004F086FF02A8FFF7D1FE0F23214A009335
:1003B00002211F4B02A8FFF78FFF02A9204604F07D
:1003C00077FF02A8FFF7C2FE40F233331A4A0093C8
:1003D00002211A4B02A8FFF77FFF02A9204604F072
:1003E00067FF02A8FFF7B2FE42F69053144A00934B
:1003F0000221144B02A8FFF76FFF02A9204604F068
:1004000057FF02A8FFF7A2FE00F0DAFC0722214600
:1004100008F000FA0DB030BDC196010894950108AE
:10042000C3950108AB970108D697010816970108F4
:10043000D19501081F970108559701080B960108EF
:100440005F97010846960108014B1878704700BF76
:10045000580C00202DE9F84F07F0AAFE036D50302C
:100460001B6898473D4C06460F463D4821680AF0F8
:100470008FF8D4E902010AF00BF8D4E9022305460B
:10048000B01A67EB03010AF019F82946024635480D
:100490000AF07EF83946304609F0FAFF0146324844
:1004A0000AF076F8D4E9060109F0F2FFDFF8D0A0EF
:1004B0002E4D94F8202094F82130002A14BF524683
:1004C0002A46002B14BF53462B46014628480AF003
:1004D0005FF83B463246206909F0EEFE80468946C9
:1004E00009F0D6FF8346B8EB060069EB070109F077
:1004F000E5FF594602461F480AF04AF8D4E90C01C4
:1005000009F0C6FF94F8382094F83930002A14BF57
:1005100052462A46002B14BF53462B460146164826
:100520000AF036F83B463246A06A09F0C5FE80461E
:10053000894609F0ADFF0446B8EB060069EB0701F8
:1005400009F0BCFF214602460A480AF021F802F0F1
:100550006FFF0A4B1878BDE8F88F00BF0800002035
:100560007198010894980108B59801086E980108DF
:10057000CB980108F598010815990108580C00203E
:100580006A98010810B50020002107F019F8044608
:1005900078B1417980290FD1094B02790168186837
:1005A00004F0EEF8204607F0A7FB0821204609F0EA
:1005B0001BF9044B187810BD034809F0E9FFF1E777
:1005C0006C070020580C0020C599010870B50D4635
:1005D000044609F073FF0E4E01460E4809F0D8FF9D
:1005E0002946204606F0B8FE22462B46304609F042
:1005F0000CFF22462B4606F1100009F006FF2246AA
:100600002B4606F12800BDE8704009F0FEBE00BF91
:1006100010000020029B010808B507F0C9FDBDE8E5
:10062000084007F011BE000008B5044809F0B0FF0B
:10063000BDE80840112010F06EBD00BF769B010898
:1006400008B5044809F0A4FFBDE80840132010F0E5
:1006500062BD00BF1D9B010808B5044809F098FF62
:10066000BDE80840122010F056BD00BF4D9B0108A8
:1006700008B5044809F08CFFBDE80840102010F0D0
:100680004ABD00BF609B010838B507F091FD0546E3
:1006900007F004FF034C2080284607F00BFF608022
:1006A00038BD00BF380600201FB56123CDE90131F8
:1006B00001A9039205F054FB05B05DF804FB07B5F2
:1006C0008DF8041001A98DF805208DF8063005F08D
:1006D0000DFC03B05DF804FBD0B51F4600231646A1
:1006E0004374D0E90223B3F1004F08BF002A044647
:1006F0000AD0006809F0E0FD864277EB0103ACBF49
:10070000012300232374D0BD0123FBE7037C13B135
:10071000437C83F0010318467047000037B5184842
:10072000FFF7F4FF40B3174C204600F07BFB164B5D
:1007300016491870206815F079FC15F03DFE054645
:100740001349606815F072FC15F036FE6424114AF6
:1007500090FBF4F395FBF2F102FB1152B02504FB80
:100760001304002CB8BF6442002A01950094B8BF5E
:100770005242094809F00CFF084B187803B030BD0D
:10078000300000203C06002078000020002474493E
:100790000000C84240420F00679A0108580C002030
:1007A000F0B54E4E85B0336804465B680F4683B1A2
:1007B0004B4D4C4809F0ECFE6B463A4629463068F2
:1007C00003F062FD9DF8003025606371207105B073
:1007D000F0BD4548FFF79AFF054670B3434D4448C6
:1007E00009F0D6FE0F224349684608F050FF2968F9
:1007F000684608F0ACFF4049686815F017FC15F032
:10080000DBFD01B2684608F089FFB5F908106846BB
:1008100008F084FF684608F070FF0546684608F057
:100820006EFF0122354B627120712560D3E9020110
:1008300083F83920C3E90C01C9E73148FFF766FFA7
:100840000028C4D02F4809F0A3FE1E222E49684676
:1008500008F01DFF03222D49684608F025FF2946B0
:10086000684608F03FFF0321684608F03BFF01217E
:10087000684608F037FF264B68461B78254D002B4D
:100880000CBF6521002108F02DFF10F019FC014676
:10089000684608F027FF10F01BFC0146684608F088
:1008A00021FF2988684608F046FFB5F9021068461E
:1008B00008F027FF684608F020FF0546684608F064
:1008C0001EFF4023012263710C4B20712560D3E988
:1008D000020183F82120C3E9060178E76C070020B4
:1008E0004806002005980108300000203C06002042
:1008F0002B980108380700200000C842080000209B
:100900001800002049980108470700206698010850
:1009100078000020380600200A4B10B51B685B6881
:1009200073B90948FFF7F2FE044638B90748FFF7E4
:10093000EDFE044610B9064809F02AFE204610BD17
:100940000124FBE76C070020300000201800002085
:10095000AC99010808B5054B93F850301BB932210A
:10096000034802F035FE014808BD00BFDC05002049
:10097000819601082DE9F04F87B0FFF7D5FCFA20EA
:1009800000F0CCFFFFF7F0FB704809F001FE07F024
:100990000FFC6F4D06462B686E4C13F0010F04D10F
:1009A00005F0C4F9012320602B6006F15001206896
:1009B00005F082F86849206805F080F8FFF7CAFF63
:1009C000266802680546654903A805F05FF803A993
:1009D000304605F0B5F826682A6A8DF804006049AB
:1009E00003A805F053F803A9304605F0A9F85D4ABD
:1009F0008DF807005C492068FFF756FE8DF805006A
:100A0000206806F0D9FA594A8DF80600584920683E
:100A1000FFF74AFE574A814657492068FFF744FED0
:100A2000564A824656492068FFF73EFE554B064619
:100A3000554A5649206807F061F8554A804655499D
:100A40002068FFF731FE544A834654492068FFF777
:100A50002BFE9DF804208DF803005149206806F014
:100A600071FC07464F4D20689DF805302A7880F8C4
:100A700028309DF805109DF80630FFF720FE4A4A01
:100A80004B469DF8061020681278FFF718FE534673
:100A90002A7849462068FFF712FEDFF8189143468E
:100AA0002A7851462068FFF70AFE43462A785946BD
:100AB0002068FFF704FE5B4699F800204146206855
:100AC000FFF7FDFD9DF803302A7841462068FFF7C7
:100AD000F6FD364A33469DF8031020681278FFF77A
:100AE000EEFD3B462A789DF803102068FFF7E7FDEE
:100AF0005B4699F8002039462068FFF7E0FD334651
:100B00009DF8042039462068FFF7D9FD33469DF84B
:100B1000072039462068FFF7D2FD53462A78314630
:100B20002068FFF7CCFD206805F000FC204809F0A4
:100B30002FFD01224FF4AF71206805F065FB002006
:100B400000F052FC07B0BDE8F08F00BFEB99010840
:100B5000340600206807002019060008089A0108DA
:100B60000D9A01089D0C0008F0B401084904000822
:100B7000189A01081D070008249A01086D0C000846
:100B80002F9A0108A107000819090008369A0108E0
:100B90008505000823B4010855040008439A01089C
:100BA000D3B40108580C00205C0C00205B0C002022
:100BB0004D9A0108220D0020F8B507F0F9FA044615
:100BC000FFF7C8FE236D04F150001B689847204CC6
:100BD000064620460F4623683246013340F8103B54
:100BE0000B46C4E90267FFF777FDD4E9022304F15D
:100BF0002800FFF771FD2168164809F0C9FCD4E907
:100C0000020109F045FC0146134809F0C1FCD4E992
:100C1000060109F03DFC114E94F82020104D0146CC
:100C2000002A14BF32462A460E4809F0B1FCD4E926
:100C30000C0109F02DFC94F838200146002A14BF5D
:100C400032462A46BDE8F840074809F0A1BC00BF7B
:100C500008000020959A0108AE9A01086A980108D8
:100C60006E980108C49A0108E39A010808B507487C
:100C700009F08EFCFFF708FD054B1A88054B1A8119
:100C8000FFF79AFF044B187808BD00BF9C99010834
:100C9000380600203C060020580C002000230020CD
:100CA0004FF000412E4A30B5136013745374C2E9FB
:100CB00002012C4C2C4A85B01360137453742368C2
:100CC000C2E90201DB0708D404F066FA802201467B
:100CD000264803F07FFA01232360244A244B254C45
:100CE0001A6007F065FA244B244D8366244B04A850
:100CF0000393244B0293244B0193244B40F8103D63
:100D000006F0D2FF07F054FA214B4365FFF7BCFC15
:100D1000204B1B88238107F04BFA204600F082F815
:100D200004461D4809F034FC1C4A1D4B002C08BF2A
:100D30002A461C491C4809F02BFC1C491C48002C65
:100D400008BF294609F024FC1A4809F021FC1A4B77
:100D50001C70FFF731FF194B187805B030BD00BF8C
:100D600060000020300600204800002028070020F6
:100D70006C0700203C060020A57500084499010876
:100D800029060008410600085906000871060008F7
:100D9000CD050008380600204C9901083F9901084C
:100DA000ADA301085C9901086299010849990108FD
:100DB000799901088E99010878000020580C0020CC
:100DC00007F0F6B913B507F0F3F9044603689B681A
:100DD0009847204607F010FA002401234FF496723A
:100DE0000B49CDE900340B48234600F0FDF90A48D1
:100DF00009F0CEFB094809F0CBFB00F0E5FB4FF40E
:100E0000BC71074802F0E4FB204602B010BD00BFF1
:100E10008B9B010875090008949B0108A79B01089A
:100E2000D89B01082DE9F04F884B87B093F85020EC
:100E3000044699461AB93221854802F0C9FB07F0E9
:100E4000B7F9064600F1480707F0B2F9D9F844307F
:100E500000F1440B0393436C05465B685846002140
:100E6000D9F840A0D9F84880D9F84C909847002389
:100E700002211A4677480FF0EFF901220221754846
:100E80000FF0B8FA6B6C58461B6801219847002395
:100E900008211A466F480FF0DFF9002208216D483B
:100EA0000FF0A8FA142000F039FD002300251A469F
:100EB000022168480FF0D0F90022022165480FF0A6
:100EC00099FA0A2000F02AFDB36C38461B6898474F
:100ED000322000F023FDB36C38465B689847B36C52
:100EE0000095D3F810B00422502304A93846D847FF
:100EF000142000F013FDB36C0095D3F810B0042259
:100F0000502304A93846D8478346B36C38469B68BB
:100F10009847BBF1000F0AD14F4809F039FB5846FA
:100F20004E4B23604E4B636007B0BDE8F08F4946DF
:100F3000404615F02DFA40B14A4809F029FB474BCD
:100F400028462360464B6360EEE79DF810309DF81D
:100F5000110003F03F0300EB032015F013F80546E2
:100F60000146404615F01EFA002852D1256021683E
:100F7000484615F0F9F908B1C4F8009041462068D8
:100F800014F04AFF51460546039814F045FF014608
:100F9000284615F04BF841460546484614F03CFFFC
:100FA0000146284615F0F6F82F4915F03FF8206065
:100FB00005469DF813009DF8123000F0E00000EBAC
:100FC0000320400914F0DAFF284915F0E3F8284916
:100FD00015F02CF8274914F01FFF27496060804660
:100FE00015F0B8F9C0B1254809F0D2FA0122022162
:100FF00018480FF0FFF90122082116480FF0FAF9FE
:101000000A2000F08BFCB36C38461B68984701201F
:101010008AE7C4F80080AAE7404614F06FFB00227C
:10102000174B14F0C3FB14F05BFE0446284614F083
:1010300065FB0022134B14F0B9FB14F051FE22465D
:101040000146114809F0A4FAD0E700BFDC050020F2
:101050008196010800000240139C0108003C1CC658
:10106000E1FAC7C2269C010817D7C83D00E0FF443B
:101070000000484300004842000048C2609C01084C
:101080000000244000408F40759C0108064A136808
:101090001968064B19B94FF0FF321A607047126891
:1010A000D268D2685268F8E774070020240800204C
:1010B00010B5044620B940F2F261084802F088FAFF
:1010C0006269074B9A4207D1A06A064B984203D047
:1010D000B0FA80F0400910BD0020FCE7BC9C01087C
:1010E000440800202C080020F8B51B4B1B4E1C6840
:1010F000054630680F46043001F0F9FA334640B92E
:1011000001203168164EC96A3268884022EA00021E
:1011100032606A1C07D137B1196812480431BDE842
:10112000F84001F0C1BA1A686419546007D30E4A36
:1011300010681968BDE8F840043101F0C1BA0B4AE3
:1011400010681968043101F0BBFA094B1A68A24211
:1011500088BF1C60F8BD00BF6C080020700700202D
:10116000F4070020440800207807002074070020BE
:101170002408002080B5DFF86C80164F164D174EFE
:101180002B6863B9164B1B68012BF8D94FF08053BD
:10119000C8F80030BFF34F8FBFF36F8FEEE701F059
:1011A00009FBFB68DC68201D01F0A1FA3368013BF4
:1011B00033602B68013B2B6001F01CFB04F15400F1
:1011C00016F0E4FB206B01F037FC204601F034FC04
:1011D000D6E700BF58080020E4070020E007002001
:1011E0007C07002004ED00E02DE9F84F4FEA820A69
:1011F000804650460D4699460B9E01F01BFC074663
:10120000002800F0B780BC2001F014FC0446002840
:1012100000F0AD80076325B94FF458715C4802F0C7
:10122000D7F95246A521206B15F007FD236BAAF1D3
:10123000040A9A442AF0070A6B1E04F134020F359F
:1012400013F8011F02F8011B197809B1AB42F7D15D
:101250000A9D4FF0000B042D28BF0425271DE562D1
:10126000C4E9135B384684F843B001F01AFAC5F1BB
:10127000050504F1180001F014FAC4F8B4B06022B6
:1012800059462461A561646284F8B8B004F1540041
:1012900015F0D3FC3F4B4A46A3653F4B4146E365FF
:1012A0003E4B5046236601F061FA206006B134607F
:1012B00001F080FA3A4B3B4E1A68DFF82481013284
:1012C0001A603268002A58D134601B68012B25D17E
:1012D000354801F0DBF9354801F0D8F9344801F020
:1012E000D5F9DFF80091334801F0D0F9324D334899
:1012F00001F0CCF9484601F0C9F9284601F0C6F9D9
:101300002F4801F0C3F92F4801F0C0F92E4801F031
:10131000BDF92E4BC3F800902D4B1D6001252D4AC1
:101320002D491368086801331360E26A636405FAA3
:1013300002F3034314200B601B4B394600FB0230C1
:1013400001F0B2F901F056FAD8F8003063B1336811
:10135000DA6AE36A9A4207D24FF080521F4B1A6052
:10136000BFF34F8FBFF36F8F2846BDE8F88F384625
:1013700001F062FB4FF0FF35F6E7D8F80030002BA4
:10138000CCD13368DA6AE36A9A4298BF3460C5E721
:10139000BC9C0108F8F2010818F30108D8F2010812
:1013A000E0070020700700207C0700209007002045
:1013B000A4070020B80700200C080020CC0700205C
:1013C0002C08002058080020440800207407002042
:1013D00078070020F0070020F407002004ED00E06B
:1013E00040080020F807002070B504462A4D01F09F
:1013F000E1F904B92C68261D304601F078F960B98E
:101400001421E06A254B41435B5833B9012224493A
:1014100082400B6823EA02030B60A36A1BB104F14C
:10142000180001F064F91F4A1368013313602B6838
:10143000A34220D131461C4801F036F91B4A1368FB
:101440000133136001F0D6F9194B1B6893B12B6877
:10145000A3420FD1174B1B6823B140F2B641164887
:1014600002F0B6F84FF08052144B1A60BFF34F8F62
:10147000BFF36F8F70BD124A04F154001368013B33
:10148000136016F083FA206B01F0D6FA204601F0C3
:10149000D3FAFFF7FBFDD5E7700700207C0700209B
:1014A000F4070020F007002058080020E40700207F
:1014B00040080020EC070020BC9C010804ED00E07F
:1014C000E0070020F8B5054620B940F24C51174816
:1014D00002F07EF8164B1B68AB4220D001F06AF98F
:1014E000144B6C691F68144B1E6801F083F9BC42F1
:1014F00017D0B44215D0114B9C4208D1AB6A83B9C6
:1015000095F8B830012B0CBF02200320F8BD0C4B1E
:101510009C4208D0002C0CBF04200120F6E70020DC
:10152000F4E70220F2E70420F0E700BFBC9C0108CA
:10153000700700207407002078070020440800206E
:101540005808002070B5044620B940F21C711948B3
:1015500002F03EF8184D2B68A34229D044B301F0A5
:1015600029F92046FFF7A4FDF0B1261D304601F011
:10157000BEF801231149E26A08689340034314202E
:101580000B600F4B314600FB023001F08DF82B68E9
:10159000E26ADB6A9A4207D34FF08052094B1A6025
:1015A000BFF34F8FBFF36F8FBDE8704001F022B9DA
:1015B00070BD00BFBC9C010870070020F40700202C
:1015C0007C07002004ED00E013B500241A4B0094C2
:1015D00001935022234619491948FFF705FE0128B7
:1015E0001DD100F0CBFE012819D14FF0500383F339
:1015F0001188BFF36F8FBFF34F8F124B124A1B68D6
:10160000543313604FF0FF32104B1A60104B1860C8
:10161000104B1C6002B0BDE8104001F04BB9013026
:1016200007D140F604010C4802B0BDE8104001F0BB
:10163000CFBF02B010BD00BF20080020F69C0108FB
:10164000751100087007002078030020240800208E
:10165000400800206C080020BC9C0108024A136866
:1016600001331360704700BFEC070020014B18687E
:10167000704700BF6C08002008B501F075F9014BF8
:10168000186808BD6C080020014B1868704700BF3F
:10169000E00700202DE9F84F3A4B1B68002B6AD178
:1016A000394B1C6801341C609CB9384D2B681B6891
:1016B00023B140F66221364801F08AFF354B2A6893
:1016C000196829601A60344A136801331360FFF700
:1016D000DDFC324D4FF0000B2B68314FA34211D986
:1016E0003A68304BD16A14224A439A58022A28BFDA
:1016F0004FF0010B2C4A1268002A0CBF58460120FB
:10170000BDE8F88FDFF884A0DFF8A490DAF80020B5
:1017100012681AB94FF0FF322A60E1E7DAF80020C8
:10172000D268D66871688C4201D22960D8E706F188
:101730000408404600F0DBFFB16A19B106F1180059
:1017400000F0D5FF01224FF0140CF06AD9F80030F8
:1017500002FA00F11943134BC9F800100CFB0030DA
:10176000414600F0A1FF3868F16AC26A914228BF81
:101770004FF0010BCAE70D4A4FF0000B136801331D
:101780001360B7E7EC0700206C0800207407002006
:10179000BC9C0108780700202808002024080020AD
:1017A000700700207C07002070080020E807002058
:1017B000F40700202DE9F8432E4C236823B940F6A6
:1017C00068012D4801F004FF00F0F4FF2368013B9D
:1017D000236024682CB1002401F00CF82046BDE8F9
:1017E000F883264B1B68002BF5D0254D254EDFF8DE
:1017F000A8801FE0EB680127DC6804F1040904F10C
:10180000180000F074FF484600F071FF1420E26AEF
:10181000316807FA02F30B4300FB0280494633604C
:1018200000F042FF184BE26A1B68DB6A9A4201D360
:10183000164B1F602B68002BDCD10CB1FFF726FC88
:10184000134D2C6844B10127104EFFF723FF00B160
:101850003760013CF9D12C600C4B1B68002BBAD0CF
:101860004FF080520B4B1A60BFF34F8FBFF36F8F57
:101870000124B1E7EC070020BC9C0108E007002030
:101880002C080020F40700207007002070080020BA
:10189000E807002004ED00E07C07002038B50C4686
:1018A000054620B940F2CA41184801F091FE24B91A
:1018B00040F2CB41154801F08BFE154B1B6823B15C
:1018C00040F2CC41114801F083FEFFF7C7FE114BF7
:1018D0002A68186814192CBF0121002182422C604B
:1018E0000CD961B9FFF766FF38B94FF080520A4B47
:1018F0001A60BFF34F8FBFF36F8F38BD09B9A04295
:10190000F0D20021201AFFF7EFFBEBE7BC9C0108A7
:10191000EC0700206C08002004ED00E010B5044640
:1019200040B94FF080520D4B1A60BFF34F8FBFF399
:101930006F8F10BD0A4B1B6823B14FF4A461094897
:1019400001F046FEFFF78AFE00212046FFF7CCFBA0
:10195000FFF730FF0028E4D0EBE700BF04ED00E024
:10196000EC070020BC9C0108244B70B51A68244B7E
:1019700012B101221A6070BD224E1A6033681B6BCF
:101980001A68B2F1A53F0BD15A68B2F1A53F07D151
:101990009A68B2F1A53F03D1DB68B3F1A53F04D04B
:1019A00030683168343101F0E3FD174B1C68B4FA3C
:1019B00084F41423E4B2C4F11F046343134DEB58C1
:1019C00023B940F68831124801F002FE142202FBCE
:1019D00004F3E9184868083340682B44984202FB36
:1019E000045408BF4368486008BF4B606368094AF5
:1019F000DB683360336854331360BCE7EC070020C6
:101A00007008002070070020F40700207C070020E9
:101A1000BC9C01087803002070B504462A4E00F0F3
:101A2000C9FE04B93468251D284600F060FE60B97F
:101A30001421E06A254B41435B5833B90122244904
:101A400082400B6823EA02030B60A36A1BB104F116
:101A5000180000F04CFE29461E4800F025FE94F8C0
:101A6000B8301D4D012B04BF002384F8B83000F0BE
:101A7000C1FE2A682AB100F09DFEFFF707FB00F0C7
:101A8000B9FE3368A34211D12B6883B1134B1B6895
:101A900023B14FF4D961124801F09AFD4FF0805202
:101AA000104B1A60BFF34F8FBFF36F8F70BD094AA1
:101AB00011680D4A1268914201D13360F6E7BDE822
:101AC0007040FFF751BF00BF700700207C07002067
:101AD000F40700204408002040080020EC07002004
:101AE000BC9C010804ED00E0E007002038B50D467D
:101AF000044620B940F69F31074801F069FD074BC5
:101B000020461968183100F0DBFD2846BDE8384052
:101B10000121FFF7E9BA00BFBC9C01087007002053
:101B200070B50E461446054620B940F6CA310A483B
:101B300001F04EFD094B28461968183100F0B4FD3C
:101B4000002C214608BF3046BDE8704018BF4FF05A
:101B5000FF30FFF7C9BA00BFBC9C01087007002026
:101B600038B5C368DC6824B940F6FA31154801F08D
:101B70002FFD04F11805284600F0B9FD124B1B6833
:101B8000E3B9251D284600F0B2FD01230F49E26AA2
:101B900008689340034314200B6029460C4B00FB5C
:101BA000023000F081FD0B4BE26A1B68DB6A9A424F
:101BB00085BF0120084B0020186038BD2946074822
:101BC000EFE700BFBC9C0108EC070020F4070020F1
:101BD0007C07002070070020700800202C080020DF
:101BE000034B1B680360034B1B684360704700BFD7
:101BF000280800206C08002070B50C46054620B966
:101C000040F66541144801F0E3FC24B940F6664112
:101C1000114801F0DDFC00F0CDFD104B1A6823687F
:101C2000591C0FD00E482E6800686968864201D0A2
:101C300091420ED9521A934209D99B1A2360284621
:101C4000FFF7CEFF002400F0D5FD204670BD002335
:101C500023600124F7E700BFBC9C01086C0800204A
:101C6000280800200122014B1A60704770080020EC
:101C700070B50C461646054608B91B4A156805F1AD
:101C800034026260EA6A052B22612A6B2560E261F8
:101C90006A6CA260EA6C62614FF00002A2611BD024
:101CA00011490968A9420BD12273D6B1296B0A46A2
:101CB000531A12F8010BA528FAD09B08238470BD93
:101CC000032B2373F1D1FFF7C9FCAB6A0BB10223DD
:101CD0002373FFF76FFDE8E72846FFF7F3FB207358
:101CE000E3E72684EBE700BF700700202DE9F84FFB
:101CF0000D6881460C4692461DB300254FF0240B1B
:101D00004B6801F108075B68BB424B6004BFCB68BE
:101D10004B604B68D3F80C8063680BFB05915B68E4
:101D200001229F42636008BFE36805F1010508BF17
:101D300063606368DE6853463046FFF799FFB0453D
:101D4000EAD12846BDE8F88F2DE9F8430546174645
:101D5000FFF784FC1F4B1B688B4238D84FF00008FC
:101D600024264446DFF8809009EB080106FB045066
:101D70000122FFF7BBFFA8F1140818F1640F044417
:101D8000F2D1154B0222196806FB0450FFF7AEFF93
:101D9000124B04441968022206FB0450FFF7A6FF09
:101DA000044404220E4906FB0450FFF79FFF04443D
:101DB00006FB045003220B49FFF798FF04440FB1C0
:101DC00000233B60FFF7F6FC2046BDE8F8830024C3
:101DD000F8E700BFE0070020740700207807002024
:101DE0005808002044080020CC07002008B9064B02
:101DF0001868026B1346981A13F8011BA529FAD02C
:101E0000C0F38F00704700BF70070020014B1868B7
:101E1000704700BF70070020054B1B6833B1054BAE
:101E20001B68002B0CBF0220002070470120704768
:101E300040080020EC0700202DE9F041044600286E
:101E400036D0234AC36A11681746C96A8B4237D213
:101E5000142682691F4D002AA8BF3A6806FB035367
:101E6000A2BFD26AC2F10502826142699A4221D1BF
:101E700000F10408404600F03AFC174B48B9E06A0C
:101E80004643AA592AB901211A68814022EA01026F
:101E90001A603A681968D26AE262012404FA02F010
:101EA000084318601420414600FB025000F0FCFB80
:101EB000204603E03B68DB6AC3620120BDE8F08195
:101EC0001368C06CDC6AA0422CBF00200120F5E73B
:101ED000700700207C070020F4070020F8B50446B6
:101EE00008B90020F8BD1F4B1B68834204D040F6A0
:101EF0007A711D4801F06CFB236D23B940F67B71AC
:101F0000194801F065FB236DE16AE26C013B9142E7
:101F10002365E6D0002BE4D1251D284600F0E7FB21
:101F2000124E134A50B91421E76A794373582BB9FA
:101F300001201368B84023EA00031360E36CC3F187
:101F40000501A161E3620124116804FA03F008436A
:101F500010601420294600FB036000F0A5FB20461A
:101F6000C0E700BF70070020BC9C01087C07002070
:101F7000F4070020F8B50D460446002845D0036D4F
:101F800023B940F6C971214801F022FBE36C9D4260
:101F900038BF1D46E36AAB4237D0236D012B34D1E5
:101FA0001B4B1B68A34204D140F6E471174801F0B3
:101FB0000FFB1426A269E36A002AE562A4BFC5F1FB
:101FC0000505A561134D626906FB03539A421CD1B6
:101FD000271D384600F08BFBE26A0F4C40B9564390
:101FE000AB592BB901212368914023EA01032360F7
:101FF00001231420216893400B432360394600FBE2
:102000000250BDE8F84000F04FBBF8BDBC9C010891
:10201000700700207C070020F4070020044B1A689A
:102020001AB119680A6D01320A651868704700BF55
:10203000700700202DE9F041214C1E4680460F46D6
:10204000154600F0B7FB236893F8B830022B16D082
:1020500001212368D3F8B42022EA0802C3F8B4208F
:10206000236883F8B81056B13046FFF73DF84FF0BB
:102070008052144B1A60BFF34F8FBFF36F8F00F085
:10208000B9FB00F097FB1DB12368D3F8B4302B6087
:102090002368002293F8B830022B09BF01250025E0
:1020A0002368D3F8B41004BFB943C3F8B41023684D
:1020B00083F8B82000F09EFB2846BDE8F08100BF01
:1020C0007007002004ED00E0F8B50E4617461D46E7
:1020D000044620B941F219212E4801F079FA00F0A6
:1020E00069FB15B1D4F8B4302B60022394F8B850D2
:1020F00084F8B830EDB2042F1AD8DFE807F00E03E9
:1021000009061500D4F8B4301E43C4F8B46004E0E6
:10211000D4F8B4300133C4F8B430012D12D0012406
:1021200000F068FB2046F8BD022DEED10024F7E751
:10213000D4F8B4300133F0D041F24A21154801F00F
:1021400047FAEAE7261D304600F0D1FA1420124A79
:10215000E36A11689D400D431560104A314600FB4B
:10216000032000F0A1FAA36A23B141F259210948E2
:1021700001F02EFA0A4BE26A1B68DB6A9A42CED95A
:102180004FF08052074B1A60BFF34F8FBFF36F8F32
:10219000C5E700BFBC9C0108F40700207C070020B5
:1021A0007007002004ED00E02DE9F843DDF8208001
:1021B0000E4691461D46044620B941F28C2138480E
:1021C00001F006FA00F0D0FBEFF311874FF0500357
:1021D00083F31188BFF36F8FBFF34F8F15B1D4F81E
:1021E000B4302B60022394F8B85084F8B830EDB2C4
:1021F000B9F1040F1AD8DFE809F00E03090615003B
:10220000D4F8B4301E43C4F8B46004E0D4F8B43059
:102210000133C4F8B430012D12D0012087F31188A6
:10222000BDE8F883022DEED10020F7E7D4F8B430F2
:102230000133F0D041F2CF21194801F0C9F9EAE7A2
:10224000A36A23B141F2DA21154801F0C1F9154B17
:102250001B6803BB251D284600F049FA01231249DB
:10226000E26A08689340034314200B6029460F4B31
:1022700000FB023000F018FA0D4BE26A1B68DB6AC3
:102280009A42CAD90123B8F1000F01D0C8F8003032
:10229000084A1360C1E704F118010748EAE700BFE4
:1022A000BC9C0108EC070020F40700207C070020FC
:1022B00070070020700800202C08002038B5054663
:1022C00008B9084B1D68002400F074FA95F8B8307E
:1022D000022B04BF85F8B840012400F08BFA204699
:1022E00038BD00BF70070020F8B50F4C00F062FA4F
:1022F0002568ADB90D4F0E4E384600F0C7F930468F
:1023000000F0C4F90B4B2A461F600B4B0C210A202E
:102310001E6000F06DFC206010B1084901F02CF83F
:10232000BDE8F84000F066BAA80800207C0800204C
:10233000900800207408002078080020FB9C010809
:10234000914208B5416000610AD8D21A83699A4265
:102350000DD2084B011D186800F0B2F9002008BD2D
:102360009A4201D2994202D2011D034BF3E70120A8
:10237000F5E700BF780800207408002007B5FFF7D4
:10238000B3FF0C4B1B6843B90B484FF4897101F044
:102390001FF9002003B05DF804FB084BC82201932D
:1023A00001230749009307480023FEF71DFF00287B
:1023B000EAD0EFE7A8080020009D0108AC08002043
:1023C0003B9D0108E12400082DE9F04180462C20C6
:1023D0000D4617461E4600F02DFB044688B125B970
:1023E0004FF4B671084801F0F3F8FFF77DFF069B44
:1023F000C4F80080C4E9065726626362201D00F01D
:1024000050F92046BDE8F081009D01082DE9FF410B
:102410000D4690461F46064620B94FF4C3710F483B
:1024200001F0D6F80E4C206878B1052DCDE90158A1
:1024300003960DDCFFF7F0FC002302280CBF0A9A7C
:102440001A4601A9206800F0F7FB04B0BDE8F0814E
:1024500000233A4601A900F0A5FCF6E7009D01081B
:10246000A80800202DE9F74300271A4DDFF86C80FB
:102470002B681A6832B9184A11681360296003B0D2
:10248000BDE8F083DB68DC681E6804F10409484697
:1024900000F02DF9636A20469847E369012BE7D1E4
:1024A000A36933449E4206D263602461494628688A
:1024B00000F006F9DCE70023009732461946204673
:1024C000FFF7A4FF0028D3D140F27231404601F05B
:1024D0007FF8CDE77408002078080020009D0108EF
:1024E0002DE9F04F4FF00108624D89B0DFF898B147
:1024F000DBF80020136843B30024D368D3F80090BE
:10250000FFF7ACF8FFF7B2F85B4B82461A681F463C
:1025100090425A4E1CD31860002C4CD0584B1B686C
:102520001A68B2FA82F25209A9EB0A01306800F087
:102530005BFFFFF73FF998B94FF08052514B1A609B
:10254000BFF34F8FBFF36F8F0AE001249946D7E79F
:102550000393FFF787FF039BC3F800A0FFF72AF957
:10256000002205A9306800F0C1FC0028BED0059B00
:10257000002BF5DB079C636913B1201D00F0B7F851
:10258000FFF774F83B688146984201D2FFF76AFF73
:10259000059BC7F80090092BE2D808FA03F313F45F
:1025A000047A57D113F0C70F33D19B06D8D52046F4
:1025B00000F042FAD4E7814529D8FFF7FBF8DBF8B1
:1025C0000030DB68D3F80CB00BF1040000F08FF89A
:1025D000DBF81C30012B15D1DBF818104B465246A6
:1025E00049445846FFF7ACFE60B1009423464A4682
:1025F00021465846FFF70AFF20B94FF4F4712846E8
:1026000000F0E6FFDBF8243058469847A8E722465A
:102610008AE7A169069B4A4619442046FFF790FEC7
:1026200000289DD0636A20469847E369012B97D123
:10263000A2690699CDF800A00A44534651462046A7
:10264000FFF7E4FE00288BD140F20131284600F06C
:10265000BFFF85E7069BA36123B94FF44671284667
:1026600000F0B6FFA1694B464A4649442046FFF7B1
:1026700067FE75E7009D0108A4080020A808002057
:102680007808002004ED00E0740800204FF0FF32CD
:1026900000F108034360C0E90223036100230360E3
:1026A000704700230361704743689A684B608A60F3
:1026B0009A6851609960036808610133036070474C
:1026C0000A6830B5531C0AD103695A684A609160A0
:1026D0008B605960036808610133036030BD00F10D
:1026E00008035C6825689542EFD82346F9E703693B
:1026F000D0E901128A60826851605968814208BF3E
:102700005A60002202611A68013A1A60186870471C
:1027100006480068006880F3088862B661B6BFF3B7
:102720004F8FBFF36F8F00DF00BF000008ED00E0A8
:10273000002307B501930B4B1B68013303D0CA215B
:10274000094800F045FF4FF0500383F31188BFF3B1
:102750006F8FBFF34F8F019B002BFCD003B05DF850
:1027600004FB00BF7C000020439D01084FF08073F4
:1027700040F8043C054B21F0010140F8081C40F8EA
:102780000C3C40F8202C4038704700BF312700082F
:10279000074B19680868B0E8F00F80F30988BFF3A9
:1027A0006F8F4FF0000080F311884EF00D0E7047D0
:1027B000700700204FF0500383F31188BFF36F8F31
:1027C000BFF34F8F084A13680133012B136009D1FF
:1027D000064B1B6813F0FF0F04D040F2751104483C
:1027E00000F0F6BE704700BF7C00002004ED00E062
:1027F000439D010810B5074C236823B94FF4BE71FF
:10280000054800F0E5FE2368013B23600BB983F324
:10281000118810BD7C000020439D010800000000CD
:10282000EFF30980BFF36F8F0D4B1A6820E9F00FAB
:1028300010602DE908404FF0500080F31188FFF739
:1028400093F84FF0000080F31188BDE80840196844
:102850000868B0E8F00F80F30988BFF36F8F704706
:102860007007002008B54FF0500383F31188BFF3C1
:102870006F8FBFF34F8FFEF70DFF18B14FF08052EF
:10288000024B1A60002383F3118808BD04ED00E0B9
:102890000022054B05491A600A6041F26701044AAB
:1028A000116007221A60704710E000E018E000E0B5
:1028B00014E000E013B5264B264C1A78D2B20192F0
:1028C000FF221A701B78244ADBB28DF803309DF882
:1028D000033003F0500313700723002223609DF898
:1028E0000310581E090629D402B123602368032B64
:1028F00004D04FF49B71194800F06AFE2368144A13
:102900001B0203F4E06323600024019BDBB213701D
:10291000134B1A6842F470021A601A6842F070424F
:102920001A60FFF7B5FF0F4B1C60FFF7F1FEFFF7D2
:102930001BF8FFF7FDFE204602B010BD9DF80330E6
:1029400001225B00DBB28DF803300346C7E700BF0E
:1029500000E400E0B4080020B0080020439D010816
:1029600020ED00E07C00002008B5EFF305830F2B7D
:102970000AD90D4A9B5C0D4A12789A4204D940F25A
:10298000A5210B4800F024FE0A4B0B4A1B68126875
:1029900003F4E063934206D9BDE8084040F2B52154
:1029A000034800F015BE08BDF0E300E0B0080020C9
:1029B000439D01080CED00E0B408002070B50D4601
:1029C0000646FEF74BFE0D4B0D491C6862198A4204
:1029D00007D90C233360FEF7EDFE4FF0FF3420469D
:1029E00070BD1A60074A13685B1B1360064A1368C0
:1029F0002B441360FEF7DEFEF1E700BF80000020ED
:102A0000E068002084000020B808002008B5EFF33B
:102A100005831BB1C221034800F0DAFDBDE8084080
:102A2000FEF71CBE919D0108FEF7C4BEFEF716BE60
:102A3000FEF7C0BE14F09EB814F0A4B800B58BB079
:102A4000684614F097FB034B08981B6818440BB0BA
:102A50005DF804FB8400002000207047704710B52B
:102A60000446FFF7A7FEA46BFFF7C4FEB4FA84F098
:102A7000400910BD70B51546026C0446866B42B91C
:102A800005689DB98068FFF729FAA5600136A6633D
:102A900070BD6DB9406814F0ACF86368226C1344E3
:102AA000A2686360934201D3236863600020EDE76E
:102AB000C06814F09EF8236CE2685B4221681A44F7
:102AC0008A42E2603EBFA2689B18E360022DEDD10E
:102AD0000EB1013EEAE73046D8E703461A6C10B45F
:102AE000084662B1D9689C681144A142D96028BFE8
:102AF000196810BC28BFD960D96814F07AB810BC26
:102B0000704770B50446FFF755FE94F8455004F140
:102B100024066DB2002D14DCFF2384F84530FFF746
:102B200069FEFFF747FE94F8445004F110066DB2B9
:102B3000002D12DCFF2384F84430BDE87040FFF71D
:102B400059BE636A002BE7D03046FFF709F808B199
:102B5000FFF788F8013D6DB2DCE72369002BE9D06F
:102B60003046FEF7FDFF08B1FFF77CF8013D6DB27E
:102B7000DEE7000038B50D46044620B940F20311E7
:102B8000194800F025FDFFF715FED4E90F314B433E
:102B90002268D0185B1A1344A060E3600020FF2372
:102BA000A063626084F8443084F8453095B92369A5
:102BB00063B104F11000FEF7D3FF38B14FF080523B
:102BC0000A4B1A60BFF34F8FBFF36F8FFFF712FEF0
:102BD000012038BD04F11000FFF758FD04F1240076
:102BE000FFF754FDF2E700BFEB9D010804ED00E0A4
:102BF000F8B50D461746064620B94FF4BB710D488F
:102C000000F0E6FC05FB06F05030FFF713FF04462A
:102C100048B155B92060C4E90F6501212046FFF78E
:102C2000A9FF84F84C702046F8BD00F15003036002
:102C3000F1E700BFEB9D01082DE9FF4788460192AF
:102C40001E46044620B940F2F1214B4800F0C0FC7A
:102C5000B8F1000F06D1236C23B140F2F2214648AF
:102C600000F0B6FC022E07D1E36B012B04D040F23A
:102C7000F321414800F0ACFCFFF7CEF830B9019BDE
:102C800023B140F2F6213C4800F0A2FC0027B946EF
:102C9000DFF8E8A0FFF78EFDA26BE36B9A4201D349
:102CA000022E19D1324641462046FFF7E3FE636A01
:102CB0001BB104F12400FEF753FF38B14FF08052EE
:102CC0002E4B1A60BFF34F8FBFF36F8FFFF792FD4C
:102CD000012004B0BDE8F087019D1DB9FFF78AFD12
:102CE0000020F6E717B902A8FEF77AFFFFF782FD8A
:102CF000FEF7B4FCFFF75EFD94F84430FF2B08BFED
:102D000084F8449094F84530FF2B08BF84F8459030
:102D1000FFF770FD01A902A8FEF76EFF28BBFFF7C1
:102D200049FDA26BE36B9A420ED1FFF763FD019957
:102D300004F11000FEF7DAFE2046FFF7E2FEFEF790
:102D400039FD48B10127A5E7FFF754FD2046FFF7FD
:102D5000D8FEFEF72FFDF5E74FF08053CAF800309C
:102D6000BFF34F8FBFF36F8FECE72046FFF7C9FE2D
:102D7000FEF720FDB4E700BFEB9D010804ED00E085
:102D800010B5024600210120FFF732FF044638B19A
:102D9000002383600360C3601A461946FFF74CFFA7
:102DA000204610BD2DE9F843894690461F4604464B
:102DB00020B940F2C331274800F00AFCB9F1000FF6
:102DC00006D1236C23B14FF47171224800F000FC4E
:102DD000022F07D1E36B012B04D040F2C5311D480F
:102DE00000F0F6FBFFF7C0FDEFF311864FF0500344
:102DF00083F31188BFF36F8FBFF34F8FA26BE36B29
:102E00009A4201D3022F22D194F845503A466DB22E
:102E100049462046FFF72EFE6B1C13D1636A0BB99F
:102E200001200BE004F12400FEF79AFE0028F7D001
:102E3000B8F1000FF4D00120C8F8000086F3118823
:102E4000BDE8F88301356DB284F84550E8E700200D
:102E5000F4E700BFEB9D010870B50D46044620B9AC
:102E60004FF48C61204800F0B3FB236C23B140F297
:102E700064411D4800F0ACFB236833B9A36823B15B
:102E800040F26941184800F0A3FBFFF76DFDEFF336
:102E900011864FF0500383F31188BFF36F8FBFF398
:102EA0004F8FA26BE36B93421CD994F845300132EB
:102EB0005BB2A2635A1C10D1636A0BB9012009E00E
:102EC00004F12400FEF74CFE0028F7D0002DF5D0C9
:102ED0000120286086F3118870BD01335BB284F84D
:102EE0004530EBE70020F5E7EB9D01082DE9F043C5
:102EF00085B00F460192044620B94FF4A0614248C4
:102F000000F066FB37B9236C23B140F204513E4810
:102F100000F05EFBFEF780FF30B9019B23B140F269
:102F20000951394800F054FB0026B046DFF8DC9028
:102F3000FFF740FCA56BD5B139462046013DFFF7B0
:102F4000CCFDA563236963B104F11000FEF708FE10
:102F500038B14FF080522D4B1A60BFF34F8FBFF343
:102F60006F8FFFF747FC012005B0BDE8F083019D9E
:102F70001DB9FFF73FFC0020F6E716B902A8FEF7DF
:102F80002FFEFFF737FCFEF769FBFFF713FC94F801
:102F90004430FF2B08BF84F8448094F84530FF2B61
:102FA00008BF84F84580FFF725FC01A902A8FEF7B9
:102FB00023FEF0B92046FFF752FDA0B1019904F1BC
:102FC0002400FEF793FD2046FFF79BFDFEF7F2FB82
:102FD00038B94FF08053C9F80030BFF34F8FBFF3BB
:102FE0006F8F0126A4E72046FFF78BFDFEF7E2FB7B
:102FF000F7E72046FFF785FDFEF7DCFB2046FFF7ED
:103000002EFD0028EDD0B6E7EB9D010804ED00E0B1
:103010002DE9FF410446019120B940F291515248F7
:1030200000F0D6FA236C23B140F295514E4800F0DF
:10303000CFFAFEF7F1FE30B9019B23B140F29A516D
:10304000494800F0C5FA00252F462E46DFF81C81BE
:10305000FFF7B0FBA36BE3B1013BA363236813B994
:10306000FEF7DCFFA060236963B104F11000FEF7F6
:1030700077FD38B14FF080523C4B1A60BFF34F8F51
:10308000BFF36F8FFFF7B6FB0125284604B0BDE8FC
:10309000F081019B4BB925B140F2E151324800F07B
:1030A00097FAFFF7A7FB0025EFE717B902A8FEF78D
:1030B00097FDFFF79FFBFEF7D1FAFFF77BFB94F834
:1030C0004430FF2B08BF84F8446094F84530FF2B50
:1030D00008BF84F84560FFF78DFB01A902A8FEF741
:1030E0008BFD40BB2046FFF7BAFCF0B123683BB92B
:1030F000FFF760FBA068FEF79FFE0546FFF77AFB2F
:10310000019904F12400FEF7F1FC2046FFF7F9FCD9
:10311000FEF750FB38B94FF08053C8F80030BFF3CA
:103120004F8FBFF36F8F012792E72046FFF7E9FC2F
:10313000FEF740FBF7E72046FFF7E3FCFEF73AFB1C
:103140002046FFF78CFC0028EDD0002D9DD0FFF726
:1031500031FB616A19B1236B1968C1F10501A068DF
:10316000FEF708FF9DE700BFEB9D010804ED00E0BE
:103170002DE9F04385B00F460192044620B94FF483
:10318000CD61424800F024FA37B9236C23B140F2F4
:103190006C613E4800F01CFAFEF73EFE30B9019B20
:1031A00023B140F27161394800F012FA0026B046AE
:1031B000DFF8DC90FFF7FEFAA36BD3B13946204667
:1031C000E568FFF78AFC636AE56063B104F12400F7
:1031D000FEF7C6FC38B14FF080522D4B1A60BFF39A
:1031E0004F8FBFF36F8FFFF705FB012005B0BDE8E0
:1031F000F083019D1DB9FFF7FDFA0020F6E716B92F
:1032000002A8FEF7EDFCFFF7F5FAFEF727FAFFF745
:10321000D1FA94F84430FF2B08BF84F8448094F826
:103220004530FF2B08BF84F84580FFF7E3FA01A97A
:1032300002A8FEF7E1FCF0B92046FFF710FCA0B1B0
:10324000019904F12400FEF751FC2046FFF759FCD8
:10325000FEF7B0FA38B94FF08053C9F80030BFF329
:103260004F8FBFF36F8F0126A4E72046FFF749FC7D
:10327000FEF7A0FAF7E72046FFF743FCFEF79AFABD
:103280002046FFF7ECFB0028EDD0B6E7EB9D0108E8
:1032900004ED00E02DE9F84389469046054620B943
:1032A00040F2FB61204800F093F9B9F1000F06D11C
:1032B0002B6C23B140F2FC611B4800F089F9FFF749
:1032C00053FBEFF311874FF0500383F31188BFF3E3
:1032D0006F8FBFF34F8FAC6B1CB395F844604946BA
:1032E00076B22846FFF7F9FB013C731CAC6313D19F
:1032F0002B690BB901200BE005F11000FEF730FC43
:103300000028F7D0B8F1000FF4D00120C8F8000071
:1033100087F31188BDE8F883013676B285F84460FA
:10332000E8E72046F4E700BFEB9D010810B504462E
:1033300020B940F28A71054800F04AF9FFF73AFADD
:10334000A46BFFF757FA204610BD00BFEB9D0108A4
:1033500038B5054620B940F2A471064800F038F9A6
:10336000FFF728FAA86BEC6B241AFFF743FA204604
:1033700038BD00BFEB9D0108002330B5064A52F866
:10338000335002EBC3041DB942F83310606030BD06
:103390000133052BF3D1FAE710180020002310B5F4
:1033A000074A02EBC3014C68844204D1002042F872
:1033B0003300486010BD0133052BF2D1FAE700BF9E
:1033C0001018002010B5044620B94FF4F8610548E4
:1033D00000F0FEF82046FFF7E1FF2046BDE8104070
:1033E000FFF72ABBEB9D010870B504460D46164653
:1033F000FFF7E0F994F84430FF2B04BF002384F872
:10340000443094F84530FF2B04BF002384F8453046
:10341000FFF7F0F9A36B2BB93246294604F12400DB
:10342000FEF77EFB2046BDE87040FFF76ABB000058
:103430002DE9F04741488AB007F0AAF8FEF724F9D1
:103440002425079007993E4807F0A2F8079868439B
:1034500007F03AF904463B4807F09AF894B1079907
:103460000DEB05022046FEF76FFC0023DFF8F0A00D
:10347000354F07900893089A079B9A421DD3204620
:1034800007F00CF9FFF7DAFA0446FFF7E5FA2146F0
:1034900002462E4807F07CF82D4B2E4819889A8852
:1034A0008B1A07F075F82C4B1B6803B198472B4813
:1034B00007F06EF80AB0BDE8F087089B05FB0343F0
:1034C0001B7B042B98BF1AF80320099B88BF3F225F
:1034D000642B83BF6420B3FBF0F30899002382BF01
:1034E00005FB01418969B1FBF3F308990898DDF800
:1034F00020C0DDF820E0DDF82080DDF8209005FB1D
:10350000004005FB0949D9F81C6005FB0141CDE9E4
:10351000033605FB08439B69029305FB0E439B683A
:10352000019305FB0C431B8C0093036949683846E3
:1035300007F02EF8089B013308939CE72A9E0108A8
:10354000369E0108419E0108769E0108A89E01084A
:1035500038180020C79E010834090020CC9B0108C0
:10356000259E0108014B1860704700BF50090020DC
:1035700073B5124C064623780D46114A1BB91378D1
:103580000BB172B6FEE70123002113700D486422CF
:1035900013F053FB2B4600960B4A6421094814F0A4
:1035A00051FA0A4B1B6803B198470125054E304676
:1035B00007F032F872B62570F9E700BF2C09002039
:1035C000C0080020C2080020FE9E0108500900200B
:1035D000F7B5184C064623780D46174A1BB91378E1
:1035E0000BB172B6FEE70123002113701348642269
:1035F00013F023FB2B460096114A64210F4814F068
:1036000021FA104B1B680BB10C4898470E4B1B68F6
:1036100003B198470125094E0C4F304606F0FCFFD8
:10362000384606F0F9FF72B6094B257000BF013B22
:10363000FCD1F2E72D090020C1080020C2080020BB
:10364000269F0108BC08002050090020359F010872
:10365000FFFF0F00F8B5DFF898C003681A4FCCF8E9
:1036600000304368194E3B608368194D3360C3686E
:10367000184C2B60036918492360436982690B6009
:10368000164BC0691A60164A1060DCF800003868F2
:103690003068286820681C460968124D1968124E67
:1036A000126864220021284613F0C7FA23683246C4
:1036B0006421284614F0C6F9284606F0ADFF0B4BEE
:1036C00000BF013BFCD1ECE7400900204809002085
:1036D0004C0900204409002028090020300900205E
:1036E00038090020C2080020EB9E0108FFFF0F00F0
:1036F0003C090020074B1B6803B198471EF0040FDC
:103700000CBFEFF30880EFF309808169004A10478E
:10371000553600085009002010B1012106F064B8A8
:10372000704708B106F0D0BF7047806870474068A6
:1037300070474368012B08D1D0E90432934204D08A
:103740001878003018BF01207047002070474B6880
:1037500070B5042B04460E464FF0000304D0C0E9B8
:1037600000338360204670BDD1E90425AD1AC0E95D
:10377000003383602846FFF7D4FFC4E90000054406
:10378000A560D6E90453024629468B4205D00AB10A
:103790000E78167001310132F7E75B1B1844606048
:1037A000E0E742680346022A06D1D3E904031B1A64
:1037B000032B01D906F0E9BF002070474368032BB3
:1037C00006D1D0E904329A4208BF00231846704758
:1037D0000023FBE7037870B581680446B3B1284A3B
:1037E000284806F0D5FE6368022B12D12046FFF769
:1037F000D8FF0146244806F0CBFEE1680B78002B89
:103800003CD02248BDE8704006F0C2BE204A2148A4
:10381000E7E7032B05D12046FFF7D0FF01461E48FE
:10382000E9E7042B0ED100251C4ED4E90431C91A56
:103830008D4205D2595D304606F0AAFE0135F4E707
:103840001748D8E7012B08D12046FFF772FF15492A
:10385000154B002818BF1946E1E700250F4ED4E9A3
:1038600004239B1A9D4205D2515D304606F090FE1E
:103870000135F4E70D4806F08BFEBEE70C48C1E7C2
:10388000D4960108D99F0108ED9F01080FA00108F7
:10389000ADA30108E39F010862A101087BE00108D4
:1038A000F79F0108D39F0108CE9F0108FD9F0108E3
:1038B000ACA30108B1F5705F2DE9F84304460F464B
:1038C00002D9174805F050FF066883689B1B994290
:1038D00019D9D0F804900846FFF723FF05460346A0
:1038E000A9EB0608B14505D00BB132781A70013644
:1038F0000133F7E72068FFF70FFF05EB08032560AA
:103900003D446360A56025683DB92846C4E901557A
:10391000FFF702FF2846BDE8F8830120FBE700BF60
:10392000519F01082DE9F0410368561A90468268BC
:103930000446D21A96420D4615D93046FFF7F1FEDD
:1039400007460346A84505D02A7803B11A70013509
:103950000133F7E720683E44FFF7DEFEC4E9016665
:103960002760BDE8F0814768481EFF1ABE420ED8A6
:103970001A469D19A91A002904DD10F8011F02F842
:10398000011BF7E7002EA8BF9B196360E9E73D44E0
:103990001F44FA1A002A04DD10F8012F03F8012B46
:1039A000F7E763682E461846B04505D0327800B177
:1039B000027001360130F7E7A8EB05084344E4E75D
:1039C00008B509C81B1AC3F57050884202D21046C8
:1039D00005F0CAFE994238BF1946581805D2B0F50D
:1039E000705F28BF4FF4705008BD4FF47050FBE774
:1039F0002DE9F8430C46591C204615461F46FFF793
:103A000059FF064680B14FF00003EA1929462046C7
:103A1000FFF788FFD4E901539D4208D00DB1002380
:103A20002B706368013363603046BDE8F8831B4A3E
:103A300001212046FFF7C4FF23680746A5EB0309D1
:103A4000FFF76FFE10EB090F1CBF002300F80930D1
:103A5000236880461A460146954205D009B1107880
:103A6000087001320131F7E7D31A0133434410469D
:103A700019466568954207D019B192F800C081F8DF
:103A800000C001320131F5E72D1A1D44206847447A
:103A9000FFF742FEC4E90085A760C5E78C9F0108D7
:103AA0002DE9F04105460E4661B1D0E90132D21A46
:103AB0008A4209D300221E4403B11A700133B34273
:103AC000FAD16B60BDE8F081114AFFF779FF8046BB
:103AD000FFF727FED5E9001407460A46034694423D
:103AE00005D00BB11078187001320133F7E70023CD
:103AF000641A3C44264404B123700134B442FAD120
:103B00002868FFF709FEC5E900744744AF60D9E7AC
:103B1000C0A00108D0E90032D21A914210B503D9F1
:103B2000891AFFF7BDFF10BD3CBF5B184360FAE781
:103B300070B50C46012120461646FFF7BBFE054630
:103B400028B101212046FFF7E5FF23681E702846B3
:103B500070BD0000426808B5012A06D1BDE80840E2
:103B60000A4600F11001FFF7E3BF8168024806F042
:103B70000FFD002008BD00BF4FA0010810B50C1AB2
:103B8000134605D001462246184613F03DF8034679
:103B9000181910BD2DE9F0410446A2EB01081646A4
:103BA000A368226808469B1A98450F4615D94046D7
:103BB000FFF7B7FD05460346BE4205D00BB13A7884
:103BC0001A7001370133F7E72068FFF7A5FD25607C
:103BD0004544C4E90155BDE8F0816568AD1AA845C2
:103BE00004D83146FFF7CAFF6060F4E70D44294668
:103BF000FFF7C4FF636829461A468E4205D00AB112
:103C00000878107001310132F7E7751B1D446560BB
:103C1000E1E770B50E46D2E900313046C91A1446C4
:103C2000FFF748FE054630B1D4E900124FF000031B
:103C30003046FFF7AFFF284670BD000070B5D0E9F1
:103C4000043100F110060446C91A3046FFF732FE6F
:103C5000054640B1D4E90712914206D1A168064851
:103C600006F096FC0025284670BD4FF00003304654
:103C7000FFF790FFF7E700BFA69F01082DE9F0418D
:103C80008368A2EB01081746026804469B1A984510
:103C90000E4615D94046FFF744FD05460346B74298
:103CA00005D0327803B11A7001360133F7E7206886
:103CB000FFF732FD25604544C4E90155BDE8F081B8
:103CC0004568AD1AA84505D839463046FFF756FF76
:103CD0006060F3E70D4429463046FFF74FFF636805
:103CE00029461A468F4205D0087802B1107001317A
:103CF0000132F7E77D1B1D446560DFE737B50D46F0
:103D000001A8114606F051FD04212846FFF7D2FD17
:103D1000044630B14FF0000302AA01A92846FFF77C
:103D2000ADFF204603B030BDFFF7E8BF426808B5DD
:103D3000022A06D1BDE808400A4600F11001FFF74B
:103D4000DDBF8168024806F023FC002008BD00BFEB
:103D500087A00108FFF7EABF2DE9F0410E460021D8
:103D60001C4617468AB00DF108082022C0E9001150
:103D700081600546404612F060FF1E2C94BF22462B
:103D80001F223946404612F034FF7368013B032B73
:103D900014D8DFE803F00230404722462F49384666
:103DA00013F003FF28B122462D49384613F0FDFEDB
:103DB00040B9012229463046FFF7BAFE28460AB02C
:103DC000BDE8F08122462749384613F0EEFE28B1BF
:103DD00022462549384613F0E8FE08B90022E9E7F3
:103DE00000220AA941F8242D404614F001F8021CD3
:103DF00018BF0122DEE700220AA941F8242D40461F
:103E000013F0F6FF019B02464345D7D029463046C2
:103E1000FFF774FFD2E723463A4629463046FFF7BC
:103E2000E7FDCBE714F00106C8D164082146284617
:103E3000FFF740FD0028C1D021462846FFF76AFE63
:103E4000B442BBD0022107EB460006F0DBFC0028A1
:103E5000B4DB2B6898550136F2E700BFCE9F01080E
:103E6000619F0108D39F0108669F010830B5134682
:103E7000426885B0032A044600F110050A460FD0B7
:103E8000014601A8FFF768FF204601AA2946FFF76F
:103E9000C0FE04460198FFF73FFC204605B030BD48
:103EA0002946FFF7A5FD0446F7E70000F0B50446F4
:103EB00085B0104616460F4613F06FFE6268034643
:103EC000032A16D03246214601A8FFF745FFDDE957
:103ED000011291420BD04FF000033846FFF75AFE13
:103EE00001250198FFF718FC284605B0F0BD002514
:103EF000F7E7441C21463846FFF7DCFC054618B9B5
:103F0000054806F045FBEFE74FF000033219314654
:103F10003846FFF707FDE7E76C9F01080A4600F106
:103F20001001FFF7C3BFF8B50D46194628461646DF
:103F30001F46FFF7BFFC044630B14FF00003F219F3
:103F400031462846FFF79AFE2046F8BD13464268E0
:103F500010B5042A06D1BDE810400A4600F1100150
:103F6000FFF7E1BF8168024806F012FB002010BD98
:103F700016A001082DE9F0410C4690461D46064664
:103F800040B139B10849184605F02AFC074618B96E
:103F900030602060BDE8F0812A46414612F029FEDB
:103FA00037602560F6E700BF9BF2010870B5054653
:103FB00010460E46144613F0F0FD224603463146E5
:103FC0002846BDE87040FFF7D5BF000010B50C468D
:103FD00031B1044900F016FD231A5842584110BD72
:103FE0000846FCE785A2010810B500B121B90648D2
:103FF00006F0CEFA002010BD1AB9044AFFF7D6FF2A
:10400000F8E70120F7E700BFDAA00108E7A0010800
:104010002DE9F74305460E4617469846FFF7E4FF9D
:10402000C0B10F49222005F0DBFB0446A8B1384699
:10403000FFF77BFB81463846FFF7C0FB13F0ADFD71
:104040004346CDE90090074A2221204613F0FAFCAE
:1040500030602C6003B0BDE8F0833060F9E700BF4A
:104060009BF2010819A101082DE9F8430E46984674
:1040700016F8013B02F1FF3903704660C0F8089062
:10408000044615463D214A46304612F095FD074646
:1040900068BB4B46182B28BF1823C4F83001A36215
:1040A00004F10C05A26A3146284612F0A2FD002256
:1040B000A66AA3191A7337B1D4F83021791C04F118
:1040C0002C0012F096FD0022D4F83031234483F8FE
:1040D0002C202EB12946404600F094FCC4F834014F
:1040E000D4E901120A48BDE8F84306F0C7BA831BB9
:1040F000023DED1A182B1A46A8BF1822B5F5807F8D
:1041000028BF4FF48075A262C4F83051C8E700BFE1
:1041100021A1010830B504460D46084B9DB000931F
:10412000074A084B642103A813F08CFC03AA294614
:104130002046FFF73BFF1DB030BD00BF13A10108B3
:104140000BA10108F6A001082DE9F04316466422F0
:1041500003F10C048FB00746884620461849ADF895
:10416000042013F008FD70B9336B23B1154A3221D6
:1041700001A813F067FC01AA41463846FFF716FF75
:104180000FB0BDE8F08320460F4913F0F4FC04465D
:10419000A0B9736B002BEED00125DFF83490736B60
:1041A00001A81B5DC5F1320128444A46013413F0D1
:1041B00049FC102C05F10205F1D1DCE7034ADBE7ED
:1041C0002DA1010832A1010836A101083EA1010874
:1041D0007BE00108016000210273C0E90111704712
:1041E000F8B5054617460E4639B332B320491820B4
:1041F00005F0EAFA044608B3C0E9006700261D4B43
:1042000000F108074361C0E9026606618021384673
:1042100005F0FAF9D4E90012384605F033FA1449EA
:10422000082005F0D1FA90B16B68C0E9004603B9E7
:104230006860AB6803B15860A860F8BD0E4806F02E
:10424000A7F901213046BDE8F84005F0CDBA0B488A
:1042500006F09EF90A4A40F255110A4806F098F90C
:104260000121206805F0C0FA18212046EBE700BFC5
:104270009BF20108808182830CE10108CBA1010837
:10428000E7A101081EA2010870B54468054604B301
:10429000266806F1080005F0BFF9D6E903239A4223
:1042A000C4B216D16B681BB96A210B48FFF790F9AD
:1042B0006868082143686B6005F096FA6B6803B97B
:1042C000AB600121306805F08FFA1821304605F007
:1042D0008BFA204670BD00BF7AA1010810B50446D4
:1042E000006810B1012105F07FFA204610BD7FB5AE
:1042F0000546FFF71AFA13F050FC0446861C2846C0
:10430000FFF715FA013803281DD8DFE800F0020690
:10431000080F0734601C04B070BD0D34FAE728465E
:10432000FFF74CFA13F039FC3418F3E701A82946DB
:10433000FFF70DFADDE9014301A81B1B06EB43045F
:10434000FFF7CCFFE6E70B34E4E700002DE9F04788
:1043500086B08146884614461D46FFF745FE68B183
:104360002046FFF7C4FF4049074605F039FA0646E4
:10437000C9F8000028B93D4806F00AF906B0BDE8C2
:10438000F0872046FFF7D3F90138032864D8DFE827
:1043900000F00214253D2046FFF7C7F9814620466C
:1043A000FFF7C7F9324B334A002814BF18461046AE
:1043B000CDE900902B46304A0AE02046FFF7B5F9D8
:1043C00081462046FFF7EDF92B46CDE900902B4AB8
:1043D0003946304613F036FB05463AE0612D20465B
:1043E0000DD1FFF7A2F905462046FFF7E7F92B4666
:1043F000234A00903946304613F024FBECE7FFF7E0
:1044000094F981462046FFF7D9F9D1E72046FFF716
:104410008CF92B4600901B4A3946304613F012FBAC
:10442000DFF868902146054603A8FFF790F9DDE91B
:10443000034AA2450AD0AF4214F8013B06D9791BC2
:1044400070194A4613F0FEFA0235F2E703A8FFF7A7
:1044500045FFC8F8005091E72046FFF766F92B4664
:104460000090094AC6E700BF9BF201080CE1010871
:10447000CE9F0108D39F01084DA1010855A1010855
:104480005EA1010865A101086BA101087BE001089C
:104490002DE9F0430E4607469046D1B04FF49C728A
:1044A000002102A81D46589C12F0C7FB31463B462E
:1044B000424602A8FFF7D8FD3678622E00F0F98058
:1044C00029D83F2E54D008D82E2E5BD09DF8081046
:1044D0007D4806F05DF87D4A58E0532E00F0A1803B
:1044E000612EF3D10DF1340979484A4605A906F049
:1044F0004FF84F98002800F0D580FFF718F90328EF
:1045000000F0AF802846734A2146FFF74FFD7248FE
:1045100006F03EF833E0722E48D00ED8642E3AD022
:10452000672ED3D105A96D4806F032F833464F9A6D
:1045300021462846FFF70AFF21E0732E51D0772E3F
:10454000C4D1674806F024F80399002900F0BA8026
:10455000644813F010FB0646002840F0B380624820
:1045600006F016F83146384600F068FF5F4AA4E0CE
:104570005F4806F00DF821462846FFF7CBFD51B005
:10458000BDE8F0835B4806F003F85B4A2146284605
:10459000FFF70CFDF3E70399584805F0F9FF02AB6C
:1045A0003A4621462846FFF7CFFDE8E705A95448DB
:1045B00005F0EEFF0399534813F0DDFA20B93846B1
:1045C00000F03AF9504AE1E74F993846FFF7FEFC10
:1045D00008B14E4ADAE74F9808B1FFF72FFB722374
:1045E000A5E705A94A480DAA05F0D2FF4F9938461C
:1045F000FFF7ECFC0028ECD14F9810B10DA9FFF7A4
:104600008DFC73234F9A21462846FFF79FFE2168B1
:10461000404805F0BDFF2868216806F01FF83E48B5
:1046200076E705A93D480DAA05F0B2FF4F99384637
:10463000FFF7CCFC0028CCD14F9810B10DA9FFF7A3
:104640006DFC2146284673234F9AFFF77FFE012118
:10465000384600F0F3FE324805F09AFF01F056F9B3
:104660008DE74F98FFF7AAF813F097FA08F10106C3
:1046700006442C49304605F0B3F8074690B14F98F0
:10468000FFF79CF8284A03463146CDF8009038469B
:1046900013F0D8F939464F98FFF740FC012138460E
:1046A00005F0A2F861234F9A21462846FFF7B0FC97
:1046B000ADE71E4805F06CFF1D4A21462846FFF76E
:1046C00075FCC8E701214EE78CA30108AEA30108E1
:1046D000DEA20108F7A2010803A301084FA2010806
:1046E0003FA3010867A301086DA301088AA301087D
:1046F0002CA2010836A2010816A1010840A2010857
:1047000060A20108D496010873A2010876A20108EC
:1047100090A20108A9A20108ACA30108BAA201084D
:10472000BFA301089BF2010815A301081AA3010801
:104730003DA301082DE9F0410C4680460D48154681
:104740001E46069F05F024FF04B14DB90A4805F046
:104750001FFF39463046BDE8F041084AFFF726BC46
:10476000069733462A4621464046BDE8F041FFF70A
:104770008FBE00BFEBA3010800A4010813A4010829
:104780007FB504460D4600680C49164600F000FB54
:1047900078B100F001FD03AB00933246294602AB2D
:1047A000FFF7C8FFDDE902122046FFF719FD04B04C
:1047B00070BD034805F0ECFEF9E700BF85A20108D3
:1047C000ACA1010810B10C2105F00EB8704710B172
:1047D000012105F009B8704730B513460D4604466F
:1047E000AC4207D01BB194E8070083E807000C3304
:1047F0000C34F5E7184630BD10B5044638B1FBF768
:10480000A5FC2046BDE81040282104F0EDBF10BDF6
:1048100070B50446406AFFF7D5FFD4E90656AE42AC
:1048200004D02846FBF792FC2835F8E7A06908B1C8
:10483000FFF7E2FF204670BDF8B5054600242826A4
:10484000074FD5E906031B1ADB107B439C4205D2B8
:1048500006FB0400FFF7F2F90134F2E7F8BD00BFF0
:10486000CDCCCCCCF8B50446224805F091FE2248C8
:1048700005F08EFED4E90631994218D0C91A1F4EB0
:10488000C91071431E4805F083FE00252827D4E98E
:1048900006031B1ADB1073439D4205D207FB05007C
:1048A000FEF798FF0135F2E7164805F071FED4E9EE
:1048B0000931154EC91A89107143144805F068FE74
:1048C00000250C27D4E909031B1A9B1073439D4252
:1048D00005D207FB050001F02BF80135F2E70C4883
:1048E00005F056FE0B4805F053FEBDE8F8400A48B7
:1048F00005F04EBE18A5010820B80108CDCCCCCCDF
:1049000022A5010834A50108ABAAAAAA6DA5010831
:10491000ACA301087DA50108B29B01082DE9F04375
:10492000002487B006466846CDE90044029404F0AE
:10493000C9FC684604F05EFD4FF028082F4F304D4B
:10494000D6E906239B1ADB107B439C424ED208FB20
:1049500004F302EB0309D35C002B43D14846FEF776
:10496000E4FE0146684604F037FD4846FEF7DFFEE8
:10497000042837D8DFE800F03803101A240048462E
:10498000FEF7D7FE0146684604F0DCFC50BBC221AE
:104990002846FEF71DFE25E04846FEF702FF0146C9
:1049A000684604F0B5FCE8B9C621F1E74846FEF7D1
:1049B00005FF0146684604F00FFD98B9CA21E7E7F4
:1049C000494603A8FEF7C3FEDDE903126846521A02
:1049D00004F0DAFC18B9CF212846FEF7F9FD039858
:1049E000FFF7F5FE0134ABE7D321D1E7684604F0C9
:1049F00029FD029807B0BDE8F08300BFCDCCCCCC38
:104A000062A401082DE9F04305460E4600244FF04C
:104A100028081A4F8DB0D5E906239B1ADB107B437B
:104A20009C4224D208FB042931461822684613F020
:104A3000CEF84846FEF779FE182201460DEB02003B
:104A400013F0C5F8684605F015FF684605F024FF29
:104A500006A805F00FFF06A805F01EFF18226846FD
:104A60000DEB020113F0A1F818B10134D3E74FF0B8
:104A7000000948460DB0BDE8F08300BFCDCCCCCCDA
:104A80002DE9F04F06460F4600244FF00C09DFF8E1
:104A90006C808DB0D6E909535B1B9B1008FB03F3B8
:104AA0009C4224D218223946684613F090F8182206
:104AB00009FB04FB0DEB020055F80B1013F087F80F
:104AC000684605F0D7FE684605F0E6FE06A805F044
:104AD000D1FE06A805F0E0FE182268460DEB0201A3
:104AE00005EB0B0A13F061F818B10134D2E74FF06F
:104AF000000A50460DB0BDE8F08F00BFABAAAAAACD
:104B000010B51446FFF77EFF20B12146BDE81040E6
:104B1000FFF704BA10BD0000F8B50C46064640F297
:104B200001120021224812F088F84FF480722146C9
:104B30001F4812F05EF81E491E4805F029FD1E4967
:104B40001B4813F073F81C490546002013F06EF85B
:104B5000294607463046FFF755FFA0B9294630469B
:104B6000FFF78EFF044600B30168144805F010FDFE
:104B7000A3683846984701242046F8BD39461048B6
:104B800005F006FDF8E73A4629463046FFF7B8FF3C
:104B900004460028F2D00B4805F0FAFC0A4805F05C
:104BA000F7FC3046FFF75EFEE6E729460748E7E7F1
:104BB000D80A0020FFA9010869A1010896A50108EB
:104BC000BFA50108ABA50108ACA30108D8A5010841
:104BD00010B54FF4807204460649043004F0B6FC68
:104BE000002805DD2046BDE810400249FFF794BFCC
:104BF00010BD00BFD809002038B514461D46FFF788
:104C000001FF28B12A462146BDE83840FFF72EB9FA
:104C100038BD10B51446FFF7F5FE20B12146BDE8BA
:104C20001040FFF783B810BD10B51446FFF7EAFE39
:104C300010B12146FEF78EFF002010BD38B5144696
:104C40001D46FFF7DFFE28B12A462146BDE8384061
:104C5000FFF77CB938BD00002DE9F04700248CB087
:104C6000074603A8CDE90344059404F02BFB214635
:104C700003A8009404F042FC0146002834D02146E9
:104C800003A804F0C4FB40F2E73304460093002677
:104C90003546DFF8F890009BB34273D9214603A84C
:104CA00004F0E7FB824600286CD1182321460DEB67
:104CB000030203A804F06EFB0444214603A804F099
:104CC000E6FB8046B0B10CAA214642F828AD03A805
:104CD00004F0FEFA029A044406A93846FFF799FF49
:104CE00000B101350136D6E76A4603A804F096FB09
:104CF0000446CCE7214603A804F013FC70B10CAACB
:104D000002F8288D214603A804F00CFB9DF808202A
:104D1000044406A93846FFF787FFE1E7214603A8C8
:104D200004F0D0FB804668B102AB01AA214603A87B
:104D300004F041FBDDE90123044406A93846FFF7EE
:104D40005BFFCDE7214603A804F0AEFB90B10CABAE
:104D500043F8288D01AA214603A8CDF8048004F069
:104D600002FB9DF808300444019A06A93846FFF773
:104D700065FFB5E7039B4846195D01F0E00105F0CA
:104D800007FCAFE728460CB0BDE8F087A7A40108F0
:104D900008B5FFF737FE18B1BDE80840FEF7C9BCFB
:104DA00008BD10B5044608461146FFF72BFE014624
:104DB00020B9C4E90000A060204610BD2046FEF7DF
:104DC000C6FCF9E708B5FFF71DFE18B1BDE80840BD
:104DD000FEF7E7BC08BD08B5FFF714FE18B1BDE843
:104DE0000840FEF7EBBC08BD037810B5044643B19C
:104DF000044805F0CDFB0021204600F01FFB0023F6
:104E0000237010BD92A401082DE9F0410E469DF8D3
:104E10001840174698469DF81C50FFF7D3FF844270
:104E200005DCA84203DC88F80000BDE8F08101231E
:104E300022463B70314606902B46BDE8F0410148C2
:104E400005F0A6BB3AA401082DE9F0410E46BDF8D5
:104E5000184017469846BDF81C50FFF7B3FF844230
:104E600005DCA84203DCA8F80000BDE8F0810123BE
:104E700022463B70314606902B46BDE8F041014882
:104E800005F086BB3AA40108F0B585B00D4616467C
:104E90001F46FFF797FF11F075F80A99044611F0C5
:104EA00077FA38B10B99204611F068FA10B13C60DE
:104EB00005B0F0BD01230A98337010F01FFC0646C0
:104EC00020460F4610F01AFCCDE902010B9810F0B5
:104ED00015FC3246CDE900013B462946014805F064
:104EE00057FBE5E73AA4010873B51C460E46154684
:104EF000FFF771FF002302AA42F8043D20600699E3
:104F000005F01AF9019B33B122683146034805F0D8
:104F10003FFB01232B7002B070BD00BFFBA5010851
:104F2000002370B5D1E90025AD1A0446C0E900336D
:104F300083600E46284601D005F0C6FBC4E9000098
:104F40000544A560D6E90053024629468B4205D0A8
:104F50000AB10E78167001310132F7E75B1B184475
:104F60006060204670BD38B504460D460B781030A1
:104F700000F8103C4B68103140F80C3C51F8083CEC
:104F800040F8083C51F8043C40F8043CFFF7C8FFE7
:104F900005F11C0104F11C00FFF7C2FF204638BDDB
:104FA0002DE9F843D0E90054641B9146A2101F4C30
:104FB00006465443B4F5705F0F4602D11C4804F016
:104FC000D3FB002C14BF22460122A418A1EB050537
:104FD00026D2B4F5705F23D82CB30C20604305F0C3
:104FE00073FB804618EB05031CBF99E8070083E8B4
:104FF0000700424639463068FFF7EEFB716800F162
:105000000C023846FFF7E8FB05463068FFF7DAFB8D
:105010000C2303FB0484C6E90085B460BDE8F88373
:105020004FF47054D9E7A046DCE700BFABAAAAAAA8
:105030008C9F01082DE9F043054685B008460C46D3
:1050400017461E4612F0A9FD172803D982212D48C4
:10505000FEF7BEFACDE90147D5E9097803962A4A59
:10506000A8EB0706B41054430134B4F5705F02D9BD
:10507000264804F079FBEB6ADB1B9B1053439C42F0
:1050800015D94FF00C0909FB04F91CB1484605F08D
:105090001BFB0446224641463846FFF79DFB686AE3
:1050A000FFF790FB26446C624C44AE62EC62EA6A05
:1050B000D5E9090314491B1A9B10121A4B4392108D
:1050C0004A430133934206D9114805F061FA8C2115
:1050D0000C48FEF77DFAD5E90A3293420AD023B193
:1050E00004AA12E9070083E807000C33AB6205B09D
:1050F000BDE8F08301AA194605F12400FFF750FF2F
:10510000F5E700BF62A40108ABAAAAAA519F010853
:105110001FA4010838B500250346044603F8045BC4
:1051200029461846142211F088FD0A4AC4E906559A
:105130006261C4E90855C4E90A55C4E90C558021E7
:1051400004F0FDF92046044B044A0549FFF772FFBD
:10515000204638BD580900209D5100081EA60108B0
:105160002AA6010810B5084C2368DB0709D40748B4
:10517000FFF7D0FF0123064A0649044823600FF0D9
:10518000FAFF024810BD00BF54090020DC0B0020CC
:105190000000002011480008FFF7E4BF08B5FFF742
:1051A000E1FFBDE80840FFF75DBB0022C0E9002237
:1051B000826010B50C6804600A6042684C68446004
:1051C0004A6082688C6884608A6010BD70B50E4643
:1051D00005461446B54217D09CB12B7805F1100155
:1051E00023706B6804F110006360AB68A360EB6828
:1051F000E360FFF7DAFF05F11C0104F11C00FFF783
:10520000D4FF28342835E5E7204670BD2DE9F84362
:10521000D0E90064A41BE310234C05465C43B4F5BD
:10522000705F0F46914602D1204804F09DFA002C91
:1052300014BF23460123E418A1EB060623D2B4F5DC
:10524000705F20D814B32820604305F03DFA8046F3
:1052500018EB060002D04946FFF785FE3946424664
:105260002868FFF7B3FF696800F128023846FFF7A6
:10527000ADFFD5E900690746B14509D03046FAF7D8
:1052800065FF2836F8E74FF47054DCE7A046DFE707
:10529000286808B1FFF7B0FA282303FB0484C5E9A6
:1052A0000087AC60BDE8F883CDCCCCCC8C9F0108E6
:1052B0002DE9F047D0E9065704460E46DFF80C8189
:1052C0008AB0AF421BD029466846FFF74CFE6846BD
:1052D000FEF72BFA81463046FEF727FA014648468C
:1052E00005F009FB30B13046FEF71FFA0146404693
:1052F00005F04EF96846FAF729FF2835E1E7D4E9C9
:1053000006892E4AA9EB0807FD1055430135B5F56E
:10531000705F02D92A4804F027FA236AA3EB080336
:10532000DB1053439D4220D94FF0280A0AFB05FAAF
:105330001DB1504605F0C8F90546494640462A4683
:10534000FFF744FFD4E90689C14505D04046FAF786
:10535000FDFE08F12808F7E7A06908B1FFF74CFA4D
:105360002F44A5615544E7612562226AD4E906030A
:1053700012491B1ADB10121A4B43D2104A43013355
:10538000934206D90F4805F003F977210E48FEF73E
:105390001FF9D4E90703984209D010B13146FFF74D
:1053A000E2FDE3692833E3610AB0BDE8F087014616
:1053B000324604F11800FFF729FFF5E7CDCCCCCC3D
:1053C000519F0108F9A4010862A40108C7A40108BB
:1053D000002313B502A941F8043D094B0422D3E987
:1053E0000140084B20445B689847044628B10648B2
:1053F00005F0CEF8204602B010BD0448F8E700BF23
:105400002C0C0020180C002073A8010887A80108A4
:1054100008B5084805F0BCF8FFF7A4FEFFF70CFA42
:10542000054805F0B5F8FFF79DFEBDE80840FFF719
:1054300019BA00BFA4A80108BCA8010873B50546A5
:105440004FF416700C4605F03FF9064630B9214876
:1054500005F09EF822212048FEF7BAF84FF41672A4
:105460000021304611F0E9FB314628464FF4167210
:10547000FFF754FA194D014601902CB3184805F076
:1054800087F8D5E901431C44164DEB681BB101991F
:105490002046083198476B680422104920469847F7
:1054A00004226B680DEB0201A01898476B68019A03
:1054B000314604F1080098470B4805F069F830467A
:1054C00005F0ECF802B070BD084805F061F86C68B2
:1054D000DAE700BFF5C8010827A701082C0C002057
:1054E00065A70108180C00209FA7010884A70108E0
:1054F0002DE9F74FFFF736FE2F4F06462F4805F0F0
:1055000047F8B846DFF8D090DFF8D0A0FCF7AEF847
:105510002B4D38602B68AB462A4C002B37D003F557
:105520006A436033984232D223782BB9264805F07B
:105530002FF8264805F02CF8012330462370FFF79A
:1055400047FB41F2883352464FF0FF310020FCF711
:1055500071FD0190FCF78AF8019BC8F8000023B99F
:10556000237813B13046FFF733FBDAF80030DA075F
:1055700044BFD8F800202A609B07C7D50023CBF88A
:105580000030D9F80830002BBED09847BCE723780C
:105590006BB100213046FFF751FF0D4804F0F8FFD2
:1055A0000C4804F0F5FFD9F8083003B19847002300
:1055B00023702B60C5E700BF440C0020E3A701085F
:1055C000400C0020380C0020F8A701081BA8010897
:1055D0003EA8010850A80108180C00203C0C00202F
:1055E00010B5FFF7BFFD04460021FFF727FF204657
:1055F000FFF738F9BDE810400348002301220221DB
:105600000068FCF761BD00BF140C002010B5FFF767
:10561000A9FD04460021FFF711FF2046BDE8104018
:10562000FFF720B92DE9F743194E074688467568FC
:105630000AB1B3681D440024DFF8609002A941F864
:10564000084D0422D9F8003028469847326800995E
:105650008A4204D00F4804F09BFF204614E0042245
:10566000D9F800300DEB0201A818984701990A48B3
:1056700004F08EFF019A4245EFD8D9F80030394640
:1056800005F108009847019803B0BDE8F08300BF1A
:105690002C0C0020AEA70108C9A70108180C002097
:1056A00084B0F0B585B00AAC84E80F000B9B23B939
:1056B00040F229117F48FDF78BFF0A9B23B94FF475
:1056C00095717C48FDF784FF7B4C0AAD0FCD0FC46C
:1056D0002B682546794C0FAA07CA45F8103984E88B
:1056E000070012B94FF48063A360236823B940F226
:1056F00035117048FDF76CFF2368013304D140F287
:1057000037116C48FDF764FFFFF72CFD06466C4B24
:105710006C4A6D49FFF78EFC6C4B6D4A6D49304603
:10572000FFF788FC6C4B6D4A6D493046FFF782FCF1
:105730004FF4167004F0C8FF074680B9694804F0BA
:1057400027FF694804F024FF3046FFF775F800236F
:105750003370FFF73DFE654804F01AFF2CE04FF46C
:105760001672002111F069FAD4E901032D680422B0
:1057700003A91844A847002861D02268039B9A42D5
:105780005DD15B4804F004FF01224FF416713846E6
:10579000FFF748FF0446574804F0FAFEFFF718FEEB
:1057A000002C48D001233370224639463046FFF79B
:1057B00053FA384604F072FF33783BBB4FF416704F
:1057C00004F082FF044630B9464804F0E1FE7F2130
:1057D0003848FDF7FDFE4FF416720021204611F007
:1057E0002CFA00224FF416712046FFF71BFF0746E4
:1057F00090BB04F053FF204604F050FF3E4804F0F5
:10580000C7FEFFF7AFFC0021FFF718FE3B4BFA2263
:10581000019301233A4900933A480023FBF7E4FC43
:1058200020B94FF4A8712348FDF7D2FE05B0BDE8BA
:10583000F04004B07047344804F0AAFE34700022EF
:105840004FF416713846FFF7EDFE04460028ABD141
:10585000384604F023FF74E74FF4167004F034FF69
:10586000054630B91F4804F093FE8E211148FDF71C
:10587000AFFE4FF416720021284611F0DEF94FF406
:10588000167229463046FFF749F808B92846B0E7AE
:105890008742FBD10023E95CE25C9142F6D10133FF
:1058A0009F42F8D1284604F0F9FE204604F0F6FEA7
:1058B000ACE700BF27A70108180C00202C0C002023
:1058C0000D5600082EA601083AA60108115400083A
:1058D0003FA601085AA60108E155000862A6010882
:1058E0007AA60108F5C80108E1A60108BCA80108CC
:1058F0007FA60108A3A6010805A70108140C002033
:105900001CA70108F1540008B8A6010810B5064C00
:10591000226922B94FF4AA710448FDF759FE2369A0
:10592000BDE81040184700BF180C002027A7010849
:1059300010B504460168074804F02AFE616831B1D9
:105940000B7823B10448BDE8104004F021BE0348A1
:10595000F9E700BFD4A801080FA00108ACA3010813
:105960001FB50B46546801780294127801925A6868
:10597000009242681B68024804F00AFE04B010BDA1
:10598000D9A8010810B50446C06908B104F086FE24
:10599000206908B104F082FE606808B104F07EFE60
:1059A000204610BD10B504460068FDF70BFD2046EB
:1059B00010BD0000CB210148FDF70ABEF7A8010881
:1059C000FE2307B502A901F8043D054B1868002322
:1059D00000681A46FDF7E6F903B05DF804FB00BF66
:1059E000540C0020D0B51F467423C0E900310023B9
:1059F000044683600820164603F0D4FEC0E9006721
:105A0000A0602046D0BD00002DE9D043DDE9066747
:105A100099467223C0E9003100239642836077EBF8
:105A200009030446904603DA2B210748FDF7D0FD11
:105A3000102003F0B7FEC0E90089C0E90267A0604A
:105A40002046BDE8D08300BF5CA90108036837B5D4
:105A5000632B05460C4601D0FFF7ACFF002302AADA
:105A600042F8043DA968204604F066FB019A3AB169
:105A70002146044804F08CFD38210348FDF7A8FDB9
:105A800003B030BD2FA901085CA9010870B56323DC
:105A90000025C0E90031044685601A20164603F04F
:105AA00081FE1A22294611F0C8F83146A06020462E
:105AB000FFF7CCFF204670BD81647047C16470471A
:105AC0002DE9F843D0E90173884600254FF00C0911
:105AD000DB1B0A4E9B105E43ECB2B4420BD209FBB7
:105AE00004724146506812F046F801350028F3D19F
:105AF0002046BDE8F8834FF0FF30FAE7ABAAAAAA28
:105B00002DE9F843D0E90473884600254FF00C09CD
:105B1000DB1B0A4E9B105E43ECB2B4420BD209FB76
:105B200004724146506812F026F801350028F3D17E
:105B30002046BDE8F8834FF0FF30FAE7ABAAAAAAE7
:105B40002DE9F0410E4649680446FFF7B9FFC0B29F
:105B5000FF2807D071682B4804F01AFD7C212A48E1
:105B6000FDF736FDD4E90123284F9B1A9B107B4398
:105B70007E2B03D97F212448FDF72AFDD4E90112A9
:105B80000C25E068531A9B10121A7B4392107A433B
:105B90000133934205FB03F80ED84144A160D4E9D8
:105BA000013496E80700E31A04E9070017489B1040
:105BB00058430138BDE8F081404604F085FD0546B4
:105BC00018B969211248FDF703FDD4E901C3002784
:105BD000A3EB0C039A100D4B5343002B09DD05EB8F
:105BE000070E0CEB070207CA013B8EE807000C37D3
:105BF000F3E7604604F052FD65604544C4E9025590
:105C0000CDE700BF9AAE01085CA90108ABAAAAAA19
:105C1000BAAE01081FB56E23CDE90131002301A9F9
:105C20000393FFF78DFF05B05DF804FBFF2270B50D
:105C3000002380F828204FF000424FF0FF31C0E9E8
:105C40000D23C2636FF07F42C0E910120522C0E944
:105C50000033C0E91423C0E902330022C0E9043351
:105C6000C0E90633C0E908330363C0E91233836532
:105C70004FF000431E4DC0E918232A68044612F075
:105C8000010213D101211B4E084632607160FCF7FE
:105C9000AFFF306018B951211748FDF799FC012377
:105CA000164A174913482B600FF065FA154B1A680E
:105CB0000AB9104A1A6014492046FFF7ABFF134B8C
:105CC000134918702046FFF7A5FF124B12491870B0
:105CD0002046FFF79FFF114B114918702046FFF730
:105CE00099FFFE220F4B18700F4B20461A7070BDA3
:105CF000500C0020D80C0020EDAF0108000000205F
:105D0000A5590008540C00201DB001085C0C0020AF
:105D100025B001085A0C00202DB00108580C0020B5
:105D200032B001085B0C0020590C002010B5084C63
:105D30002368DB0709D40748FFF778FF0123064AE9
:105D40000649044823600FF016FA024810BD00BF50
:105D50004C0C0020700C0020000000208559000829
:105D60002DE9F0410E4649680446FFF7C9FEC0B26E
:105D7000FF2807D071682B4804F00AFC87212A48C5
:105D8000FDF726FCD4E90423284F9B1A9B107B4384
:105D90007E2B03D98A212448FDF71AFCD4E904128A
:105DA0000C25A069531A9B10121A7B4392107A4358
:105DB0000133934205FB03F80ED841446161D4E9F5
:105DC000043496E80700E31A04E9070017489B101B
:105DD00058430138BDE8F081404604F075FC0546A3
:105DE00018B969211248FDF7F3FBD4E904C3002771
:105DF000A3EB0C039A100D4B5343002B09DD05EB6D
:105E0000070E0CEB070207CA013B8EE807000C37B0
:105E1000F3E7604604F042FC25614544C4E90555BA
:105E2000CDE700BFE8AE01085CA90108ABAAAAAAA9
:105E3000BAAE010838B5D0E901239B1A074A9B1076
:105E40005343CDB29D42044603D3A6210448FDF737
:105E5000BFFB0C20636800FB053038BDABAAAAAAC3
:105E60005CA9010838B5CCB2114905460B6813F09E
:105E7000010307D10F4A70201372012310600E48EE
:105E80000B605060FF2C10D0D5E904239B1A0B4AFD
:105E90009B1053439C4203D3B2210948FDF798FB62
:105EA0000C23286903FB040038BD0248FCE700BF4F
:105EB000480C0020600C0020D2A90108ABAAAAAAB5
:105EC0005CA9010810B5D0E90730C9B2D2B283424B
:105ED00009D01C788C4204D15C78944201D1987826
:105EE00010BD0333F3E74FF0FF30F9E72DE9F04140
:105EF000D0E904239B1A514A9B1053430D4609785D
:105F00000446994203D393214D48FDF761FBD4E940
:105F100001239B1A494A9B1053436978994203D342
:105F200094214748FDF754FBD4E904239B1A434AC4
:105F30009B105343A978994205D3FE2903D095219C
:105F40003F48FDF745FB6A7829782046FFF7BAFFFE
:105F5000C3B2FF2B06462CD03A4804F019FB29782F
:105F60002046FFF77FFF697807462046FFF762FF6C
:105F7000314680462046FFF775FF414602463846C7
:105F8000FFF7EEFC29782046FFF76CFF697806469C
:105F90002046FFF74FFFA97807462046FFF762FF2C
:105FA000394602463046FFF7DBFC9C212448FDF7CA
:105FB0000FFBD4E90723214F9B1A7B437E2B03D988
:105FC0009F211F48FDF704FBD4E90762616A931B18
:105FD0007B43521A57430133BB4203EB43080AD8B1
:105FE000464426622A88236A23F8032CAA7803F8F9
:105FF000012CBDE8F081404604F066FB064618B966
:1060000069211148FDF7E4FAD4E90702131A0B4A93
:106010005A430023002A0ADDC118B1F800C0F7185E
:1060200026F803C08978013AB9700333F2E704F027
:1060300035FBE66146446662D3E700BFABAAAAAA75
:106040005CA90108B7A90108BAAE0108FF2337B55A
:106050008DF804300A4B0D461C6823681BB92921B2
:106060000848FDF7B5FA2A4601A92068FCF73EFF6B
:10607000012814BF4FF0FF309DF8040003B030BD7D
:10608000540C0020EDAF010838B5816800681D464A
:10609000144604F0CFFB0346201845EBE37138BDEE
:1060A00008682DE9F04172281F4622D0742812D0CA
:1060B000632823D1886804F0FFF8002871F10003F9
:1060C00004460D4611DA0F4804F062FADD210E484D
:1060D000FDF77EFA09E08B68D3E90045B5F1004F82
:1060E00008BF002C01D0A4187D4120462946BDE8F8
:1060F000F0818868BDE8F041FFF7C6BF00244FF08B
:106100000045F2E719AB01085CA901082DE9F04749
:106110000F460646FFF7A6FE0024DFF85C904268B3
:106120000178FFB2124804F033FAD6E90758454522
:1061300016D02B78BB4211D169783046FFF77AFE32
:10614000016869290AD1D0E9012A484604F020FAF9
:10615000DAF8003003B198470134E4B20335E6E7DA
:106160002146044804F014FA2046BDE8F08700BF39
:106170003FAB010888AB010866AB01082DE9F34786
:1061800007468846FFF76EFE0025426801781B48E7
:1061900004F0FEF9FC693E6ADFF8689003340336C8
:1061A0005FFA88F8A64220D0234633F8032D9B7867
:1061B000ADF804208DF8063014F8033C984512D150
:1061C0009DF805103846FFF735FE016869290AD1A8
:1061D000D0E9012A484604F0DBF9DAF8043003B1CB
:1061E00098470135EDB20334DCE72946044804F052
:1061F000CFF9284602B0BDE8F08700BFA6AB010882
:10620000F3AB0108CFAB0108836C73B504460D46B0
:10621000164623B94FF48E710D48FDF7D9F90D4993
:10622000CDE9006423462A460B48FAF7DDFF012832
:1062300001460AD0094804F0ABF94FF491710448C3
:1062400002B0BDE87040FDF7C3B902B070BD00BF39
:106250005CA9010868AE0108196B000873AE01085B
:1062600038B590F847300446032B0D4604D940F268
:1062700035110648FDF7ACF994F847305A1C84F8FC
:1062800047201C4484F8425038BD00BF5CA9010877
:1062900010B590F84730044623B94FF49D71064875
:1062A000FDF796F994F84730013BDBB284F84730AC
:1062B0001C4494F8420010BD5CA90108CBB2FE2B2F
:1062C00037B5054605D1104803B0BDE8304004F0AD
:1062D0005FB9FFF7C7FD016804466D290DD1017A4A
:1062E0002846FFF7BFFD436800930368D4E9001216
:1062F000064804F04DF903B030BD4268044803B0CD
:10630000BDE8304004F044B986AF01088EAF010803
:10631000F9AC010808B5FFF78DFDBDE80840D0E9EC
:106320000012014804F034B908AF01082DE9F74F15
:1063300004462A4804F02CF94FF00008284FDFF8F3
:10634000B0A0DFF8B090D4E90431C91A89107943BC
:106350005FFA88F6B14232D9504604F019F9204666
:106360003146FFF7ABFF94F82830DFF88CB0B3422A
:106370000CBF1C48484604F00BF9D4E907531A4AED
:10638000AB4219D02978B14214D110460193009242
:1063900004F0FEF869782046FFF7BCFF584604F089
:1063A000F7F8A9782046FFF789FF484604F0F0F88F
:1063B000DDE900230335E3E708F10108C3E7D4E989
:1063C00007239B1AD4E90102121A92107B437A43E5
:1063D000064803B0BDE8F04F04F0DAB810AF01088A
:1063E000ABAAAAAA28AF010834AF010845AF01083B
:1063F0001FAF0108ACA3010841AF01082DE9F0412E
:10640000042290F847100546104804F0C1F8002413
:10641000DFF844800E4E95F84730A34210DD2B196B
:1064200093F842102846FFF71DFD476814B1404617
:1064300004F0AEF83946304604F0AAF80134EAE731
:106440000448BDE8F04104F0A3B800BF79AF0108EB
:1064500062A1010883AF010881AF010800232DE983
:10646000F74FC0E9083388461946D8E907594FF075
:1064700000430446C0E90613C0E90013C0E9021353
:10648000C0E90413FF208A469B46D2B284F820005C
:1064900001924D45D4E9006720D02B78019A9342B0
:1064A0001AD169784046FFF7C5FCDDE90C230146A7
:1064B0004046FFF7F5FD594508BF50450CD05F45F4
:1064C00008BF564503D0B04271EB070304DA6B787E
:1064D000C4E9000184F820300335DAE7B7F1004F52
:1064E00008BF002E08D0DDE90C23B21A67EB0303C6
:1064F00016461F46C4E90467204603B0BDE8F08F86
:10650000F8B50D460E4B896906464B434FF47A7138
:10651000B3FBF1F1FFF79AFD0446C7B2B06C036814
:106520001B689847C6E90E0103F0B2FF0146054813
:1065300004F02EF8FF2F0CBF95F820002046F8BD80
:1065400040420F0094A9010838B5C36C04460D46BB
:1065500043B9204804F01CF829462046BDE83840DD
:10656000FFF7CEBF806C1C4903685B699847A06C3D
:106570000368DB689847D5E9020103F089FF01460B
:10658000164804F005F8A06C03689968D5E9022361
:106590008847A06C03681B699847E36C9847A06C18
:1065A0000368DB689847A06C03681B689847C4E9D8
:1065B0000E0103F06DFF0146094803F0E9FF0021D9
:1065C0002046FFF743FDC0B2FE2808BF95F8200023
:1065D00038BD00BF9CAF0108C1590008BAAF01081F
:1065E000CDAF01082DE97043D1E90689B9F1004F1B
:1065F00008BFB8F1000F06460D4608D11AB1BDE834
:106600007043FFF77DBFBDE87043FFF79DBFB8F152
:10661000010F79F100030CDA58EA090302D0284887
:1066200003F0B6FF274803F0B3FF95F82000BDE85C
:10663000708312B3244803F0ABFF29463046FFF7BE
:106640005FFF95F82030C4B2A34235D1D6E90E8958
:10665000D5E90023904579EB03011EDAB2EB08027D
:1066600063EB09031946104603F028FF014617485B
:1066700003F08EFFFF242046D9E7D0E9142390458C
:1066800079EB030301DA1248D5E7124803F080FFE3
:1066900029463046FFF758FFD3E7B8EB020069EB15
:1066A0000301022871F10003E5DB03F007FF014657
:1066B000094803F06DFFDEE7084803F069FFDAE7F9
:1066C0007EAD0108A3AD0108BBAD010813AE010802
:1066D000DBAD0108F9AD010832AE010851AE010889
:1066E0002DE9F04F8DB004468846FFF7BBFB0368E9
:1066F0000546702B04D04FF4A0716F48FCF768FF7B
:10670000A06C03681B6898474246C4E90C01CDE9B8
:106710000001214602A8FFF7A1FE41462046FFF7EF
:10672000F5FC9DF828300646FF2B0AD148B9297898
:1067300062486A6803F02CFF40F24B115E48FCF798
:1067400047FFD4E90C0103F0A3FE01465C4803F0C7
:106750001FFF31465B4803F01BFF9DF82810FF29FF
:1067600040F08180584803F013FF00224FF00043AF
:10677000CDE90623DDE90223CDE90423DDE9062383
:10678000CDE90823A36D13B39847DDE90223D4E9CB
:106790001801B3F1004F08BF002A09D0DDE9062334
:1067A00010F10B0641F10007964277EB03030EDA76
:1067B000D4E90C23161843EB0107CDE90801CDE914
:1067C000046703F07BFE0146404803F0E1FE4FF012
:1067D000000A4FF0004BDFF800912A7A02A9204608
:1067E000FFF700FFA36D064603B19847F3B2FF2BF6
:1067F0005AD1DDE90223D4E90E01161A63EB010731
:1068000039463046CDE90423CDE90667CDE908676E
:1068100003F054FE0146484603F0BAFEA36D002B78
:10682000DBD0DDE90223D4E918015B4508BF5245FE
:1068300009D0DDE9062310F10B0641F1000796426D
:1068400077EB0303C9DAD4E90E23161843EB0107EB
:10685000CDE90801CDE9046703F030FE01461B488D
:1068600003F096FEB9E72046FFF7E4FAD0E90067A7
:10687000DDE9020103F00CFE3A46034631461448B6
:1068800003F086FED4E90C23DDE90201801A61EBF6
:1068900003010F460646CDE9066703F00FFE0146E9
:1068A0000C4803F075FE65E741462046FFF766FC9D
:1068B00030460DB0BDE8F08F5CA9010811AA0108AF
:1068C00044AA010863AA01087EAA0108D9AA0108FE
:1068D00097AA0108BBAA0108F1AA010870B50446ED
:1068E0000D46FFF7BFFA03686D2B11D0702B09D04E
:1068F000612B14D1836894F8411094F84000BDE8EE
:106900007040184729462046BDE87040FFF7E8BEB2
:10691000034840F22F11FCF75BFE4FF0FF3070BDD3
:106920005CA901082DE9F74F04466B4803F030FEDF
:106930006A4803F02DFE6A4803F02AFE674803F018
:1069400027FE94F82830FF2B04D14FF4E5716548F9
:10695000FCF73EFE94F828102046FFF783FA4268C1
:106960000178614803F014FE94F82830DFF8A4B1F0
:10697000DFF8649184F8463094F846102046FFF71B
:1069800071FA036880466D2B1BD14168574803F0AC
:10699000FFFD94F846102046FFF762FC98F80810B7
:1069A000204684F84610FFF75DFA426801785048A7
:1069B00003F0EEFD2046FFF721FD484603F0E8FD19
:1069C000DAE794F846102046FFF788FFC3B2FF2BA2
:1069D00006460ED1474803F0DBFD40F2DF11414887
:1069E000FCF7F6FD40F2DF11434B444A3D480FF0FF
:1069F000E3FE024694F846102046FFF763FAC5B25C
:106A0000FF2D0CD13E4803F0C3FD40F2E51135489F
:106A1000FCF7DEFD384B394A40F2E511E6E794F821
:106A20004610FE2D204636D1FFF732FC01460746C0
:106A30002046FFF717FAD8F8042098F8001082468D
:106A4000304803F0A5FD324639462046FFF73AFAB2
:106A5000C5B2FF2D12D131462046FFF7EBF9D0E940
:106A60000012294803F094FD40F2F1111D48FCF793
:106A7000AFFD214B214A40F2F111B7E7DAF80410DB
:106A8000584603F085FD2046FFF7B8FC484603F062
:106A90007FFD3946C5E7FFF7E5F931460746204651
:106AA000FFF7C8F9294680462046FFF7DBF9019039
:106AB000164803F06DFD164803F06AFD019A414641
:106AC0003846FEF74DFF94F8463084F8416084F86C
:106AD000403084F846504FE7ACA3010813AC0108DE
:106AE00032AC01085CA9010851AC01086FAC010887
:106AF0008EAC0108A5AC0108D39F01083AB001088B
:106B0000C8AC0108E2AC010801AD010858AD0108AC
:106B10006EAD010842AD010808B503F0A3FEFFF712
:106B200005F9FFF7FFFE00002DE9F8431F46164662
:106B3000FFF780F9B7F1004F08BF002ED0E90058E9
:106B400084681AD0742D01D0FEF734FFD4E9000117
:106B500003F0B4FC39468146304603F0AFFC4A46A8
:106B6000034641460A4803F013FD742D01D0FEF799
:106B700021FFC4E90067BDE8F883742D01D0FEF75A
:106B800019FFD4E9000103F099FC024B0246E8E743
:106B9000E0A9010805AA0108836C10B5044623B9D1
:106BA0004FF427710248FCF713FDA06C10BD00BF25
:106BB0005CA90108FF23054A1370054A1370054AB2
:106BC0001370054A1370054A137070475C0C00205F
:106BD0005A0C0020580C00205B0C0020590C00209F
:106BE000014B1878704700BF580C002010B50446C0
:106BF0000068FCF7E7FB204610BD00002DE9F341DB
:106C000004F052FF4FF6FF71394A3A4E13888B4217
:106C10001CBF01331380FFF789F8FFF7BDFF03683E
:106C20001B689847737807468846F3B9324B1B892F
:106C3000DBB1324AD2E90045B5F1004F08BF002C64
:106C40000ED0844275EB01020FDA2D4A001B02FBC5
:106C500003F261EB0501D317904271EB030304DBF0
:106C6000284803F095FC012373700023ADF804302D
:106C70008DF8063073782BB101238DF804301F4B4B
:106C8000C3E900783378204EABB101241F488DF85A
:106C9000054003F07DFC34701D4A1E491E48019BCF
:106CA00012780978006804F081FFF0B11B4B187866
:106CB00002B0BDE8F08133700F4B9B89002BEBD005
:106CC0004AF6C0025A431649D317D1E900013C1ACB
:106CD00068EB0105944275EB0303DDDB114803F01B
:106CE00057FC01238DF80530D6E70F4BDFE700BFD7
:106CF000240D0020000D00200C0D00209800002025
:106D00008051010099B10108090D0020C2B10108AC
:106D1000030D0020020D0020FC0C0020580C002068
:106D200088000020D7B101085A0C002008B5164B86
:106D30001B892BB9154803F02BFC154B187808BD9F
:106D4000144BD3E90023B3F1004F08BF002A01D050
:106D50001148F0E7114B19780131C9B201291970B6
:106D600001D90F48E7E70F4803F012FC00230E4A51
:106D700013700E4A13700E4A13600E4A13700123EB
:106D800053700D4BDAE700BF0C0D0020EEB1010887
:106D9000580C0020900000200AB20108380D002095
:106DA00024B201083BB20108030D0020020D0020AF
:106DB000FC0C0020000D00205B0C00201FB5702390
:106DC000CDE90131002301A98DF80C30FEF7C8FF91
:106DD00005B05DF804FB00002DE9F04F4A4B85B08B
:106DE0001A780446002A40F08B80012747491F701B
:106DF000FEF710FF464B474918702046FEF70AFF82
:106E0000DFF868A144498AF800002046FEF702FF37
:106E1000DFF85C910A22002389F800003F4901A8AD
:106E2000FEF7E0FD01A92046FEF78AFE3C4E3D49F3
:106E300030702046FEF7EEFE3B4B3C491870204672
:106E4000FEF7E8FE3A4B3B4918702046FEF7E2FE9B
:106E5000394B3A4918702046FEF7DCFE384B394A68
:106E6000187039492046F9F71FFCDFF808B1374A96
:106E70008BF8000036492046F9F716FC35490546DF
:106E80002046FFF79BFF70230193334B804601A9F7
:106E9000204602938DF80C70FEF762FF07462F4ADA
:106EA0002B4612789BF800102046F9F708FC434661
:106EB0009AF8002029462046F9F701FC3B4699F84C
:106EC000002029462046F9F7FAFB2B463278414646
:106ED0002046F9F7F4FB2B46327839462046F9F77D
:106EE000EEFB1F4A2B46127829462046F9F7E7FBAE
:106EF0001C4B1D4A1B78127829462046F9F7DFFB08
:106F000005B0BDE8F08F00BF390D0020F0B30108D7
:106F1000040D0020FAB3010805B4010811B40108FA
:106F2000E90C00201EB40108220D00202CB4010839
:106F3000210D002038B40108260D002045B40108B9
:106F4000270D0020FD6B000853B401086D7E00087A
:106F50005DB4010871B4010884B40108580C002024
:106F60005B0C0020590C00205C0C0020080D002058
:106F7000E80C0020060D002008B504F073FD18B1E0
:106F8000BDE8084004F090BD08BD000030B50446DF
:106F900085B00D46FFF720FF6D22064B01A91B7837
:106FA0002046CDE901258DF80C30FEF7D9FE05B05D
:106FB00030BD00BF060D00202DE9F84F424B434D78
:106FC0001A68044612F0010F01BFFF222A70012245
:106FD0001A602B78FF2B73D1FFF7FEFE3C4A3D4928
:106FE0002046F9F761FB3C4A28703C492046F9F7F6
:106FF0005BFB3B4F3B4A38703B492046F9F754FB5B
:107000003A4E3B4930702046FFF7C0FF394982466F
:107010002046FFF7D3FE384983462046FFF7CEFED1
:107020008146364A3B78127829782046F9F747FBA3
:10703000334ADFF8E0803378127829782046F9F770
:107040003EFB337898F8002039782046F9F737FB73
:107050002B7898F8002031782046F9F730FB294A40
:107060005B46127839782046F9F729FB26493B78A8
:107070000A7820465946F9F722FB244A4B461278F3
:1070800039782046F9F71BFB1F493B780A782046E0
:107090004946F9F714FB1A4A5346127831782046CC
:1070A000F9F70DFB337898F8002051462046F9F7A0
:1070B00006FB174A2B78127831782046F9F7FFFA49
:1070C0002878BDE8F88F00BFE40C00203B0D0020BD
:1070D00061780008EBB40108E9730008F5B4010811
:1070E000050D00202D6D0008FFB40108070D0020DC
:1070F00009B5010815B5010823B50108040D0020E4
:107100005B0C0020080D0020E90C00205A0C002028
:10711000580C00205C0C002038B504460D46FFF7E3
:107120005BFE034A29462046F9F7BEFA38BD00BF88
:1071300031760008344B2DE9F04F5A89002304467C
:1071400089B0CDE900230391002300222F4905A82F
:10715000FEF75AFC05A92046FEF7F2FC2C498246B0
:107160002046FFF72BFE2B4983462046FFF7D4FF2E
:10717000294A804629492046F9F796FA284A0546C1
:1071800028492046F9F790FA0646274FDFF8A890DD
:107190003B7899F8002029462046F9F790FA234ACF
:1071A0005B46294620461278F9F789FA204A434679
:1071B000294620461278F9F782FA33465246594654
:1071C0002046F9F77CFA3346524641462046F9F705
:1071D00076FA184A3B78414620461278F9F76FFA5A
:1071E0003B7899F8002031462046F9F768FA6D237C
:1071F0000593039B05A9204606938DF81C50FEF7C6
:10720000AFFD09B0BDE8F08F0C0D002032B50108CC
:107210003FB501084FB501086D79000860B5010858
:10722000E16B00086FB50108590C0020260D002005
:10723000270D0020220D0020580C00202DE9F04FD2
:10724000044687B008460E4615469A4610F0A5FC3F
:1072500000F106090746484602F0C0FA494633469F
:1072600007F107092F4A804610F0ECFB484602F070
:10727000B5FA0837494633462B4A834610F0E2FBFD
:10728000384602F0ABFA33463946284A814610F0B8
:10729000D9FB274A41462046F9F706FA5946804667
:1072A0002046FFF78BFD494683462046FFF734FF13
:1072B0008146204A5B46127841462046F9F7FFF99D
:1072C0001D4A4B46127841462046F9F7F8F91B4F04
:1072D0001B4A3B78127849462046013DF9F7EFF901
:1072E00005EB0A030193019B9D420ED015F801AFF7
:1072F0003B78524659462046F9F7E1F93B78524629
:1073000049462046F9F7DBF9EDE76D2303A920464E
:10731000CDE903368DF81480FEF722FD07B0BDE8F5
:10732000F08F00BFD0B40108D8B40108E1B401085F
:1073300091790008260D0020270D0020590C00200F
:10734000220D002013B502AC04F8042D01232246BF
:10735000FFF774FF02B010BD2DE970484FF00045F3
:107360000024164E83468C46D6E90001A94208BF88
:10737000A04205D010EB0B0241EB0C03C6E9002341
:107380000F4ED6E90001A94208BFA04205D010EB7C
:107390000B0241EB0C03C6E900230A4BD3E900457D
:1073A000B5F1004F08BF002C05D01BEB04004CEBDF
:1073B0000501C3E90001BDE8708800BF900000200E
:1073C000980000208800002070B50D460446FEF7A6
:1073D000ADFC044922462B46BDE870400978FFF712
:1073E000A3BB00BFE90C0020F8B5524D52482968F4
:1073F0002F460131296003F0CBF804F055FB04F06F
:107400008BFB44F6206004F06FFB417806460429AC
:1074100008D04A4803F0BCF8304603F03FF9012099
:10742000002156E00478466803F038F9012C5BD15E
:10743000434803F0ADF82B68042B0FD9FDF7ACFEE1
:1074400003785BB13F4803F0A3F83F4B9B6803B15F
:10745000984740F29B113D48FCF7BAF83B681E2262
:10746000013BDBB21E2B28BF1E23A3F12005C3F175
:10747000200402FA05F122FA04F4002521434FF416
:10748000E14402FA03F08D4208BF844225D300296B
:1074900008BFB0F5616F06460F4620D2B0F5167FE3
:1074A00071F100031EDA3C2871F10003ACBF1146F4
:1074B0000A21002003F0BEF9341847EBE075294695
:1074C000204602F0FBFF0146214803F061F8204608
:1074D0002946FFF779FF1F4B11E026462F464FF450
:1074E0001671E6E73C21E4E7032C0AD131461A483D
:1074F00003F04EF830460021FFF766FF174B18786F
:10750000F8BD8CB916482C6003F042F804F07CFA00
:10751000FEF70CFCFFF740FB03681B689847114B14
:10752000C3E90001104BEAE71048214603F030F8A8
:107530000A2075E7340D00205FB0010872B0010821
:1075400093B00108AAB001083C0D0020F7B0010873
:1075500039B101085A0C00204FB10108080D002074
:1075600064B10108880000205C0C002074B101089F
:10757000054B1870054B1A700022054B1960054B1E
:107580001A705A70704700BF030D0020020D0020D2
:10759000FC0C0020000D0020027901684079FFF703
:1075A000E7BF00000122014B1A707047200D002038
:1075B00008B504F0DBFBC0B2DE2828BFDE2008BD22
:1075C000002337B54FF47A7401930B4B60431D6869
:1075D000B0FBF4F42B681BB929210848FBF7F8FF2E
:1075E000224601A92868FBF781FC012814BF00206E
:1075F000019803B030BD00BFEC0C0020EDAF0108D6
:107600004FF47A7337B5002403FB00F2074802A950
:10761000056841F8044DB2FBF3F22868FBF7A8FDBA
:10762000012814BF2046019803B030BDEC0C0020A7
:107630002DE9F04F97B0FEF779FB4FF000090646B1
:1076400090F846B0FFF798FCDFF8C8A0DFF8C880D4
:10765000B06C02AD03680CAC1B6898475A46CDE984
:10766000000131460CA8FEF7F9FE0FCC0FC50FCC78
:107670000FC5DDE90C012368B1F1004F08BF0028F8
:107680002B70DDE9104516D11C4802F081FF002562
:1076900001271B4C4FF47A73A4FB030103FB051174
:1076A000FFF7AEFF10B30122164B5A72164B187833
:1076B00017B0BDE8F08F02F0EBFE294607462046E2
:1076C00002F0FCFE39460246504602F061FFA0453A
:1076D00079EB050308DA0021094802F0EFFE0146C4
:1076E0000A4802F055FFD2E70027D3E71FB1084848
:1076F00002F04EFFACE79DF82800D9E787B30108F8
:1077000080510100F00C0020220D0020C1B30108BF
:10771000DAB301089FB301088551010010B50020BC
:107720000021FFF76DFF10B1084B187810BD084C11
:107730002368984720B9074B1B780BB9064BF4E731
:10774000637A0BB1054BF0E7054BEEE7220D002005
:10775000F00C0020280D0020580C00205C0C0020AC
:107760005B0C0020022818BF002004F007BC0000BA
:107770002DE9FF412E4B05461F78002F54D10122E1
:1077800004AE06F8017D1A7003F000FE07230C22F8
:10779000284CCDE9003228493246231D2846FDF702
:1077A00033FB0E23254928466371A3714FF47A7881
:1077B0002761FDF7EDFA04F10803607032462049B5
:1077C0002846CDE90078FDF73FFB42F210733246C0
:1077D000CDE900731B4904F10A032846FDF734FB89
:1077E00019492846FDF7D4FA04F10C03A07032467B
:1077F00016492846CDE90078FDF726FB14492846AE
:10780000FDF7C6FA9DF80F30E07053B1114802F051
:10781000BFFE114B1B6803B1984760210F48FBF76F
:10782000D7FE2069FFF79EFF04B0BDE8F08100BFDE
:107830003A0D00200C0D002098B40108A9D40108CD
:107840009BB40108A4B4010885A20108ADB40108E5
:10785000B8B40108BDB401083C0D0020F7B0010820
:1078600070B5294BC0B21B78984206D1FDF794FC45
:10787000FDF7BAFA254B187870BD254CFDF78CFC46
:10788000FFF776FF94F9050006F06AFC04F082FA2F
:10789000207906F033FC04F073FA1E4DA07904F051
:1078A00081FA607804F054FB2A6812F0010213D1C7
:1078B0000421194E084632607160FBF799F9306077
:1078C00018B951211548FBF783FE0123144A1549C5
:1078D00011482B600DF04FFC134B1A680AB90E4A81
:1078E0001A60FEF723FAFFF757F903681B689847F9
:1078F00001220E4BC3E900010D4B5A72E3780BB124
:107900000C4BB8E70C4BB6E7070D00205C0C0020D1
:107910000C0D0020E00C00202C0D0020EDAF010824
:1079200000000020ED6B0008EC0C00208800002017
:10793000F00C0020040D00205B0C0020034B93F89A
:107940002F30022B0CBF022000207047F8000020CF
:1079500008B5FFF7F3FF02280CBF024B024B187863
:1079600008BD00BF270D0020260D0020054B5B89B8
:1079700013B9054B18787047044B5B7A002BF8D18C
:10798000FFF7E6BF0C0D0020580C0020F00C002083
:10799000FFF7DEBF01232DE9F348474C6372474BE5
:1079A0001B7873B103F022FF58B9454802F0F0FD8F
:1079B000444BDB6803B1984740F23F314248FBF744
:1079C00007FE00200021FFF71BFE10B13F4B187887
:1079D00016E023689847B0B104F018FC012871F153
:1079E000000306460F463DDB394802F0D1FDFEF7A5
:1079F0009DF932463B46217AFFF796F8FFF7A8FF3C
:107A000002B0BDE8F088334B1B78002BE4D103F0C3
:107A1000EDFE0028E0D1304DAB89FBB1FEF786F9D1
:107A2000FFF7BAF803681B689847AB892B4A2C4DBF
:107A30005A43D5E90067861B61EB0707D317B242AB
:107A4000BB410BDA274802F0A3FD1E4B5B6803B174
:107A500098474FF45B711C48FBF7BAFD0023637233
:107A6000214BB4E72368984788B1204802F090FD85
:107A7000002364680093ADF80430FFF799FD0146D8
:107A80006846A0476846FFF787FD194B9FE7114BF3
:107A90001B7863B1174802F07BFD174B1B88022B44
:107AA000DED8002211461046FFF762FDEDE703F035
:107AB0009DFE0028EED1AEE7F00C0020200D002046
:107AC00006B301083C0D0020F7B00108220D00208C
:107AD00026B30108280D00200C0D00208051010064
:107AE0008800002067B30108580C002037B3010854
:107AF000210D002049B30108240D00202DE9F04F8D
:107B00000446574D87B0C5E90023019100230A229E
:107B1000544903A8FDF766FF03A92046FEF710F8B5
:107B2000514A8146287251492046F8F7BDFD504A16
:107B3000054650492046F8F7B7FD4F49074620460D
:107B4000FFF724FA4D498DF802002046FFF736F979
:107B50004B498DF803002046FFF7DEFA494982467B
:107B60002046FFF7E7FA8346474EDFF8388133783F
:107B700098F8002039462046F8F7A1FD434A3378AB
:107B8000394620461278F8F79AFD414A5B46394655
:107B900020461278F8F793FD3E492B460A78204696
:107BA0003946F8F78CFD394A2B465946204612785B
:107BB000F8F785FD337898F8002059462046F8F705
:107BC0007EFD337898F8002029462046F8F777FDA7
:107BD0002E4A3378294620461278F8F770FD2E4A4F
:107BE0009DF80230294620461278F8F768FD2949A9
:107BF0002B460A7820469DF80210F8F760FD274AC8
:107C00009DF80330294620461278F8F758FD2B4698
:107C10004A469DF803102046F8F751FD204A534686
:107C2000294620461278F8F74AFD2B464A46514627
:107C30002046F8F744FD337898F800205146204656
:107C4000F8F73DFD6D230393019B03A920460493A0
:107C50008DF81470FEF784F807B0BDE8F08F00BF10
:107C6000F00C00207EB50108957900088EB501085A
:107C70001D7700089CB50108A9B50108FAB30108F1
:107C800005B40108B5B50108590C0020580C0020B6
:107C90005B0C00205C0C0020210D0020260D002034
:107CA000270D0020220D002010B50FC8014C84E8DC
:107CB0000F0010BD3C0D0020F8B51D46002341719A
:107CC000BDF8181004460360C180174602B115B90B
:107CD00023712046F8BD0749284601F081FD06467C
:107CE00010B920712660F4E72A4639460EF081FF6C
:107CF0002571F7E79BF2010810B50446006808B14A
:107D000001F070FD204610BD2DE9FF4142F21070D8
:107D100003F0EAFE0546464802F03AFC002D00F06A
:107D200085802F78032F03D168680021FFF74CFB73
:107D3000404ED5F8A040336823B940F2C9113E48FF
:107D4000FBF746FC002C62D000223C4B1A80D4E9A1
:107D50001C23134321D03A4BD3F80080F9F786FC5B
:107D600001463848C047D4E91C0102F091FB226F5C
:107D70000146354802F00CFCFDF7D8FFFEF70CFF7A
:107D800003685968D4E91C238847D4E91C232F4988
:107D9000C1E900232E49C1E90023FDF7C7FFFEF723
:107DA000FBFE03681B6898472A4B2B4AC3E9000176
:107DB000237AC3F3C0031370637F43B3237F33B3CA
:107DC0002649082001F000FD804630B16289237FFA
:107DD000617F0092A26EFFF76FFFCDF80C80B8F1C3
:107DE000000F14D0002330681A4603A90068FAF780
:107DF00023FF01280BD01A4802F0CAFB039C34B1C0
:107E00002046FFF779FF0821204601F0EDFC2B7A90
:107E10002BB1144802F0BCFB0022134B1A70284609
:107E200005F018FF384604B0BDE8F0810127F9E7F6
:107E300056B20108EC0C0020F7B00108240D002018
:107E4000F800002074B2010881B2010890000020FF
:107E50009800002088000020280D00209BF20108D7
:107E6000AEB20108D9B20108090D0020002310B5F7
:107E7000134C84F8343003F0F5FD08B103F014FE20
:107E8000FFF742FF01280AD00CD303280DD00D487C
:107E90004FF43171FBF79CFB4FF0FF3004E00A48D0
:107EA00002F076FB094B187810BDFFF747FD02285A
:107EB00009BF0123064B84F83430064BF3E700BFBB
:107EC000F8000020F7B00108ECB201085C0C0020BB
:107ED000080D0020E80C0020FF2300210D4A13703C
:107EE0000D4A13700D4A13700D4A13700D4A13702A
:107EF0000D4A13700D4A13700D4A13700D4A13701A
:107F00000D4A13700D4A13700D4AC2E90011137225
:107F1000704700BF060D0020050D0020070D002052
:107F2000220D0020210D0020270D0020260D00200D
:107F3000040D0020080D0020E80C0020E90C0020B2
:107F4000F00C00207047000038B50A4C05460121AE
:107F5000204608F043FA002320461A46012108F083
:107F60007BF985F001022046BDE83840012108F088
:107F700041BA00BF0000024008B50120FFF7E4FF4E
:107F8000BDE80840032009F013B80846FFF7DCBF3E
:107F900010B504466C2101F027FC204610BD09F005
:107FA000BFB80000024B0121186803681B6818471E
:107FB000580D0020021C18BF01220321014808F0BF
:107FC00019BA00BF0004024010B50C46F9F724FFAF
:107FD000022808D14FF47A704443B4FBF0F0BDE8B6
:107FE0001040F9F79BBC2046BDE8104007F050BF99
:107FF0000321014808F007BA0004024008B503480D
:1080000002F0C6FABDE8084009F08AB808BA0108CB
:1080100010B5094C094802F0BBFA20460B2108F0C4
:10802000DDF9002320461A460B2108F015F9BDE8BA
:10803000104007F013BF00BF0000024090B90108D4
:1080400008B5022007F06EFE07F0D0FE00F0BAFC83
:1080500007F0F6FE00F0A4FE08F05AFC0C48FBF70F
:1080600081FA4FF4E13008F057FF0A4B1A680AB959
:10807000094A1A60094B1A680AB9074A1A6008487F
:1080800002F086FABDE80840064802F081BA00BF57
:10809000797F00082C0E0020B90D0108300E002059
:1080A00052B601086AB601082DE9F3470446254691
:1080B0004FF01B0A11F004FA254B04F1210945F891
:1080C000113B1022002128460EF0B7FD5246002138
:1080D00048460EF0B2FD00231E4A1F4F62641F4A3D
:1080E000C4E90F33A2641E4A84F84C30C4E9142357
:1080F0001C4AC4E91733A26584F86430A3661A48A1
:1081000002F046FA3B68DFF86C800193D8F8003043
:10811000164E00933368164A514648460FF092FCBB
:108120003168284602F033FBD8F8001004F115003E
:1081300002F02DFB396804F1190002F028FB3168C8
:1081400004F11D0002F023FB204602B0BDE8F087D9
:10815000F4B90108F4BA01086400F81F38BB01083B
:1081600090BB010854BB0108C4B901085000F81FB6
:10817000D9B901085400F81F10B5094CFFF760FF8A
:108180002368DB0709D40748FFF78EFF0123064A5F
:108190000649044823600CF0EEFF024810BD00BF02
:1081A000500D00205C0D002000000020457F0008DD
:1081B00038B5064D064C2B6813F0010F04D1FFF7BC
:1081C000DBFF012320602B60206838BD540D0020A8
:1081D000C80D002010B5FFF7EBFF836E11203BB1F7
:1081E00008F08CFFFFF7E4FFBDE81040836E1847EE
:1081F000BDE8104008F08FBF4FF4FA7111F08AB952
:1082000008B50B21054808F003F928B1BDE808407E
:108210000B21024808F010B908BD00BF0000024061
:1082200008B519B1BDE80840FFF7F2BE044802F0F6
:10823000AFF9BDE8084002220B21024808F04AB815
:10824000ACB901080000024070B504462C4804F1A6
:10825000440502F09DF92846002100F0C9FD0021E7
:10826000284600F0DBFD204611F034F903F0CCFB8A
:1082700020460021FFF7D4FF0CF092F901220C21D7
:10828000204808F027F808F073FC23682046DB68D4
:1082900004F15805002198471B4E0021284600F0A4
:1082A00041FE08F027F9194802F072F908F022FDA2
:1082B00007F0C6FD304601220D2108F00BF801221F
:1082C00030460E2108F006F80021084608F0FCFBB5
:1082D00004F1480000F0B8FD0121284600F022FE1C
:1082E0004FF4E13008F018FE094802F051F90CF0A3
:1082F0007DF808F03BFC2046BDE8704011F0FAB86C
:108300005EB90108000402400000024082B9010881
:108310002E9E010838B50546FFF772FF044628B1C6
:1083200000212846FFF77CFF07F098FD07F064FC6A
:1083300005460CB1FFF76CFE284638BD70B50C46FB
:108340000646154920460EF02DF820B9002120469A
:108350000EF00AF870B1114920460DF067FE0EF0DC
:108360002BF801460E4802F013F94FF4C0710D4886
:10837000FBF72EF93046FFF743FF054648B9304674
:10838000FFF7C8FF014620460EF00CF808B1FFF7D2
:108390003FFE284670BD00BF3333534000007A448F
:1083A00080B60108AFB6010870B52D4AD6B0136883
:1083B0000546DB0705D42B4900F158030B60012368
:1083C000136029492846FFF7B9FF0646274802F0FF
:1083D000DFF8002105F1440000F020FD244C254B7E
:1083E000E360254B2361254BA360254B6360254B40
:1083F0002360254B6361254BA361254BE36104F1A9
:1084000010030FCB8DE80F0094E80F000CF0F0FB89
:10841000002305A8EB632B640CF076FB9DF8143069
:1084200005F13C04012B14D1DDF8153005A8EB63F0
:10843000DDF819302B640CF037FB164802F0A8F871
:108440000821204602F00AF9BDF91611124802F07F
:108450009FF831462846FFF7E3FE56B070BD00BFD7
:108460004C0D0020580D002000004040EBB50108E5
:10847000BC18002091FE000819FE0008A57F000826
:10848000F17F0008B57F000891A50008B527000816
:10849000F52700080CB6010832B6010808B5FFF749
:1084A00039FF03490DF0C2FD0DF0ACFF80B208BDED
:1084B00000007A4470B507490546FFF73FFF0646BE
:1084C0000CF0B6FA044631462846FFF7A9FE2046CE
:1084D00070BD00BF000040407FB5F82300F14805A3
:1084E00004AC0646284604F8013D00F0B1FC022326
:1084F000214600930122A123284600F0ADFC4FF451
:1085000000430822009306F15C01A123044628469B
:1085100000F0CCFC0440E4B2284600F09BFC20466E
:1085200004B070BD30B58BB0044608F06FFD014655
:108530005C4802F02DF808F0CBFD01465A4802F0E5
:1085400027F85A4802F024F8204600F0DFFB00F03C
:1085500015FB00F0BFFA564802F01AF804F148057E
:10856000544842F2107102F013F8284600F06CFCF7
:1085700038B9514802F00CF840F23B114F48FBF774
:1085800027F807F06BFC2046FFF7A6FF20B94FF451
:10859000A0714A48FBF71CF894F8630094F85E3029
:1085A000049094F8620094F85D20039094F86100C0
:1085B00094F85C10029094F86000019094F85F00C9
:1085C00000903F4801F0E4FF284600F085FA284675
:1085D00000F0E6FA04F14405002184F8640028461E
:1085E00000F006FC012000F035FD0021284600F0D7
:1085F00015FC012000F04CFD2046FFF7D5FE00F0F1
:108600001BFB304801F0C4FF4FF4FA700EF0B2FAD1
:10861000054600283ED12C4801F0BAFF2B4801F056
:10862000B7FF2B4801F0B4FF2A4801F0B1FF2A48F8
:1086300001F0AEFF294801F0ABFF294801F0A8FF87
:10864000284801F0A5FF284801F0A2FF274A284941
:10865000284801F09DFF2849284801F099FF284843
:1086600001F096FF04F12101264801F091FF26490F
:10867000264801F08DFF07A808F0E2F807A801F0EE
:10868000DDFE0146224801F083FF114801F080FF22
:108690000BB030BD1F4801F07BFF28460EF072FA88
:1086A000BCE700BFE5B60108FBB6010811B7010839
:1086B00028B701083DB7010858B70108AFB601084F
:1086C0006EB70108A3B70108D6B70108ABA301082C
:1086D00014B8010845B8010854B8010876B8010873
:1086E00099B80108BDB80108ACA3010813A101089D
:1086F000F6A00108E0B80108EFB80108F6B80108D3
:1087000001B9010821B901082CB9010832B90108E1
:108710004CB901080AB801082DE9FF4100F14805EC
:10872000284600F095FB04240226284F013C14F053
:10873000FF0432D0A123012239460096284600F0DA
:108740008BFB4FF40043804600930422A12302A92F
:10875000284600F0ABFBB8F1000FE7D00028E5D0C9
:108760009DF80830442B1FD19DF809306E2B1BD18A
:108770000DF10A0001F0FBFF013084B221460DF13A
:1087800009008DF8086002F00BF800230322009323
:10879000A02302A9284600F05FFB284600F05AFB00
:1087A000204604B0BDE8F0814FF488430024ADF8C2
:1087B00008306E2300210DF10B008DF80A3001F016
:1087C000EFFF0094A0230522E3E700BFC0B5010836
:1087D00038B50C461131054602F0C6FF214651F866
:1087E0005C3F28462B604B686B6038BD30B50D464A
:1087F0009DB0044601466846FFF7EAFF69462846F1
:1088000002F0E8FC04F1110321346B632C631DB00A
:1088100030BD000030B508468DB014460F4B104AED
:108820001049FCF707FC00210F4A0A9107920F4AF2
:10883000069108920E490F4A0F4D09920494059132
:1088400004AA01AC07CA0B9584E8070007AB0095A2
:108850000FCBFCF725FF0DB030BD00BF9F7F000898
:10886000C1B50108E5B501084DFF0008D5FE0008B7
:1088700000000808FD7F0008D5810008024B186839
:1088800003685B68184700BFD80D0020024B1868CA
:1088900003689B68184700BFD80D00202DE9FF41F1
:1088A000002315461370022206460D4F04AC3868AB
:1088B00004F8011D03680092D3F80C8001223346AE
:1088C0002146C04748B14FF4004238682946036842
:1088D00000921C6901223346A04704B0BDE8F08134
:1088E000D80D002030B585B08DF80D200022074B43
:1088F0008DF80C101C6803A923680092DD68022221
:1089000003462046A84705B030BD00BFD80D002063
:1089100037B54FF40045064B1C68236800951D6968
:1089200013460A4601462046A84703B030BD00BFA3
:10893000D40D002037B50025054B1C682368009531
:10894000DD6813460A4601462046A84703B030BDFD
:10895000D40D002037B50225054B1C68236800950F
:10896000DD6813460A4601462046A84703B030BDDD
:10897000D40D0020024B186803681B68184700BF1D
:10898000D40D0020024B186803685B68184700BFCD
:10899000D40D0020024B186803689B68184700BF7D
:1089A000D40D00204FF47A735843B0FBF3F0F8F77E
:1089B000B5BF10B50446FFF7FBFB2146BDE81040EC
:1089C000FFF7AABE10B5424C0BF03CFE2046022237
:1089D000002107F07FFC01222046114607F07AFCB7
:1089E00020460122022107F075FC204602220321C5
:1089F00007F070FC20460022042107F06BFC2046A3
:108A00000222082107F066FC20460122092107F016
:108A100061FC204601220A2107F05CFC204602226C
:108A20000B2107F057FC07F00BFA002320461A46EB
:108A30000C2107F011FC204600220C2107F0DAFC83
:108A40002046002204F580640F2107F043FC2046F5
:108A50000122002107F03EFC20460022022107F0FF
:108A600039FC20460022032107F034FC2046022274
:108A7000062107F02FFC20460022082107F02AFCDF
:108A800020460022092107F025FC204601220C2166
:108A900007F020FC204602220D2107F01BFC204697
:108AA00002220E2107F016FC204602220F2107F0B9
:108AB00011FC002304F5806420461A460D2107F0BE
:108AC000CBFB2046BDE8104000220D2107F092BCF0
:108AD0000000024007F01CBF1D4B00B51A6889B0AA
:108AE000D2075FBF1B4A106001221A601A4B1B4A53
:108AF00004931B4B05931B4B03931B4B02931B4B84
:108B0000079308AB43F8082D93E803008DE80300B2
:108B100002AB0FCB0BF01CFF90B1154801F038FDF4
:108B200000221448114607F0D5FB0F230222002132
:108B3000104807F06FFA09B05DF804EB0BF0A2BE25
:108B40006A210D4809B05DF804EBFAF741BD00BF9A
:108B5000D00D0020D80D00207D880008A5890008D0
:108B60008D8800089D880008E588000891A5000808
:108B7000A4BA010800000240B5BA0108002307B5F5
:108B8000ADF8043001238DF8063001980BF0B6FCE7
:108B900007F056F903B05DF804EB0BF001BD0000DF
:108BA000194B10B51A688CB0D2075FBF174A106016
:108BB00001221A60164B0793164B0593164B06932A
:108BC000164B0893164B0993164B0A93164B0B93AF
:108BD0000CAB13E907008DE8070005AB0FCB0BF0DA
:108BE000DBFD044601220F21104807F073FB3CB166
:108BF0000F4801F0CDFC0BF0ADFD20460CB010BDD0
:108C00000C4801F0C5FCF8E7CC0D0020D40D002085
:108C10001189000835890008558900087589000800
:108C2000858900089589000891A500080000024088
:108C300026BA010859BA01082DE9F0479AB002F0A6
:108C4000DDF9DFF8C0A0274C274FDFF8BC8012AD5C
:108C500050B9CDE91544CDE91387CDF848A000946B
:108C600095E80F0002F0E4F9204B00261393204B07
:108C70004FF0010912931F4B06A914931E4B28466F
:108C800015931E4BCDE91887CDE916340423CDE9A1
:108C900006368DF81D9009F0EBFE09F0DDFE01F0BF
:108CA000D7FD174ACDE9096611920322CDE90C449C
:108CB0000B9608928DF8269008AB02AC0FCBCDE94D
:108CC0000F87CDF838A084E80F0010AB93E80300BD
:108CD0008DE803000CAB0FCB02F08EFD1AB0BDE89F
:108CE000F08700BF91A500089DA600082545010852
:108CF000ED430108FD42010895420108A94201081F
:108D0000B3890008FD080108C9A600082DE9F0474D
:108D1000044606F071FF1E4905460DF087F90DF077
:108D20004BFB01461B4801F033FC4FF080412846C5
:108D30000DF01AFB48B30025DFF86090DFF8508093
:108D4000154E06F059FF494607460DF021FBA8B91C
:108D5000414638460DF06AF90DF02EFB01463046CB
:108D600001F016FC236885F001052046DB682946E2
:108D700098474FF47A7007F08BF8E2E723682046B3
:108D8000BDE8F047DB6800211847BDE8F08700BF69
:108D900000007A4477BA010889BA0108000020402F
:108DA00008B50D49012007F009FC0C490B2007F01C
:108DB00005FC0B490A2007F001FC0A49042007F0D2
:108DC000FDFB0949072007F0F9FBBDE8084007490A
:108DD000052007F0F3BB00BFC13D01083541010884
:108DE000853F01087D420108B5410108494201085B
:108DF000002310B50C461A460D21074807F02CFA3F
:108E000014B1012C00D010BD2246BDE810400D2148
:108E1000014807F0EFBA00BF00080240002310B578
:108E20000C461A460C21074807F016FA14B1012C1B
:108E300000D010BD2246BDE810400C21014807F0CB
:108E4000D9BA00BF0000024042F2107007F040BBE8
:108E500007F00EBB07F028BB2DE9F041069F1E4628
:108E600007F00303032B80460C46154603D12F2140
:108E70000D48FAF7ADFB2046BC07324629460AD515
:108E800007F060FB10B10120BDE8F0810123002054
:108E900088F80430F8E7FB0702D507F061FBF1E73B
:108EA00007F042FBEEE700BFFCBA01082DE9F041F4
:108EB000069C0D46E107804616461F4603D54C2109
:108EC0000D48FAF785FBA20703D54F210A48FAF7A8
:108ED0007FFB23043A46314628460AD507F04EFB6D
:108EE00010B10120BDE8F0810123002088F8043092
:108EF000F8E707F00BFBF3E7FCBA010808B503211C
:108F0000034807F080FA003018BF012008BD00BFF9
:108F1000000402400A460248032107F06BBA00BF72
:108F20000004024008B581B1012303211A460A4812
:108F300007F092F90321084807F050FABDE808400D
:108F400003220548114607F067B90122BDE8084031
:108F50000321014807F0BEB90004024007F0CEBC6F
:108F60001FB501A801F01AFA01A807F0A7FD05B086
:108F70005DF804FB07F010BD07F028BD084607F0B8
:108F80009FBBDFB50023CDE90133ADF80C300123E1
:108F90008DF807308DF808306FF01D038DF809301B
:108FA0000723044601A88DF80A3001F01CFA236853
:108FB00006461B6820460F469847864277EB01031A
:108FC000B4BF0120002004B0D0BD70B506461946DC
:108FD00010461D46144602F075F8736823B120460A
:108FE0002946BDE87040184770BD00002DE9FF47D5
:108FF00014461D46824607F081FC80468946261AA3
:1090000022462B4601A865EB010701F0C7F940464F
:10901000494601F03DFA29468046204601F038FADB
:1090200039460446304601F049FA22460346414695
:10903000074801F0ADFA01A807F0F2FB20B1324673
:109040003B465046FFF7C1FF04B0BDE8F08700BFC4
:1090500060BB0108042817D8DFE800F00309100EF0
:109060001200002303211A46084807F0F5B8002231
:109070000321064807F02EB90222F9E70122F7E79B
:109080000321024807F04CB9704700BF00000240BE
:10909000042817D8DFE800F00309100E120000239F
:1090A00002211A46084807F0D7B8002202210648D4
:1090B00007F010B90222F9E70122F7E7022102487E
:1090C00007F02EB9704700BF00000240F0B508B9A4
:1090D0000020F0BD002746684D1CB5421760F7D848
:1090E00003685C185B5C03F01F03A3F118010329FC
:1090F0008FBF38460D49C91811F8180C0544AE4207
:10910000E6D304280DD8DFE800F00403070C0C00B8
:10911000637813600130DCE7B4F801305BBA9BB2CE
:10912000F7E7D4F801301BBAF3E700BFACBB010886
:10913000F7B51F46436816464A1C9A4205460C4638
:1091400017D803685B5C03F0C003402B11D196B1C4
:1091500001AAFFF7BBFF50B1019A04446B68A11844
:10916000994206D8296810440C4434603A6003B030
:10917000F0BD0020FBE73046F9E72DE9F7439946BB
:10918000436817464A1C9A4280460D4624D8036815
:109190005B5C03F0C003402B1ED1FFB101AAFFF7B7
:1091A00095FF0446A0B1019E09F10109B14513D311
:1091B0000544D8F8043072199A420DD8D8F8001036
:1091C0003246294438460DF014FD00233444BB5583
:1091D000204603B0BDE8F0830024F9E73C46F7E7FA
:1091E000F0B5002931D0172A1CD8D3B2A3F1180446
:1091F000032C8CBF0024164C8D689CBFE41814F817
:10920000184C6F1C4E6804EB070CB4451DD20E6859
:1092100018438F60705500200130231A5D1C0BD15C
:10922000601CF0BDFF2A05D9B2F5803F2CBF1A2380
:109230001923DBE71823D9E78E680D68DB00771C5C
:1092400022FA03F38F60AB55E6E70020E9E700BFA1
:10925000ACBB0108172BF8B50D4616461C4612D8B4
:10926000DBB2A3F11802032A8FBF0022144A9B1815
:1092700013F8182CAB680132234413446A689342F4
:109280000BD30020F8BDFF2B05D9B3F5803F34BFC9
:1092900019231A23E5E71823E3E722462946FFF7B7
:1092A0009FFF07460028ECD02868AB683146184479
:1092B0000DF09FFCAA68E0192244AA60E2E700BF13
:1092C000ACBB010818B10023C0E9001283607047ED
:1092D000436873B514464A1C9A4206460D4602D9A5
:1092E000002002B070BD03685B5C13F0C00FF7D1C3
:1092F000002CF5D001AAFFF7E9FE0028F0D0326873
:10930000019B525D12F0E00F18BFDB432360E8E7DA
:109310000A1EABBF014601460020D243B8BF202041
:10932000FFF75EBF03685B5C03F0E001E02907D153
:1093300032B1A3F1F5014B424B411370012070474C
:1093400000207047836810B544685A1CA24208D2B6
:10935000002914BFF524F424016882600120CC5454
:1093600010BD0020FCE7F0B446684F1CB74208D897
:1093700005686C5C04F0E004402C02D1F0BCFFF7FF
:10938000D7BE0020F0BC704713460A460146402075
:10939000FFF760BFF0B446684F1CB74208D80568B5
:1093A0006C5C04F0E004602C02D1F0BCFFF7E5BE79
:1093B0000020F0BC7047F0B446684F1CB74208D894
:1093C00005686C5C04F0E004602C02D1F0BCFFF78F
:1093D000AFBE0020F0BC704770B5054608460C468D
:1093E0000EF0DBFB224603462946BDE870406020B4
:1093F000FFF730BF836841685A1C8A423FBF8260D2
:10940000BF220168012034BFCA540020704703689E
:10941000585CA0F1BF0358425841704713B5036828
:1094200014465B5C03F0E003A02B07D142B101AA14
:10943000FFF74CFE019B236002B010BD0020FBE74C
:109440001046F9E7836841685A1C8A423FBF826030
:10945000FF220168012034BFCA540020704730B198
:109460008068013888428CBF0020012070470120AD
:10947000704708B50246FFF7F2FF30B91268505C3A
:10948000A0F1FF035842584108BD0120FCE74368A2
:109490008B4207D903685B5C13F0C00F0CBF01203F
:1094A000002070470020704743688B4208D903684A
:1094B000585C00F0E000A0F140035842584170476A
:1094C0000020704743688B4208D90368585C00F05D
:1094D000E000A0F1600358425841704700207047F7
:1094E00043688B4208D90368585C00F0E000A0F1A3
:1094F000A0035842584170470020704710B50446F9
:10950000FFF7EEFF50B163688B4208D92368585CBF
:1095100000F01F00A0F11F035842584110BD002069
:10952000FCE743688B4208D90368585C0C30C0B232
:1095300001288CBF002001207047002070470023C5
:10954000C0E9013303690160C3607047F8B503687F
:109550000446002B0D46164603DC3E212948FAF747
:1095600037F83246002128460DF067FBD4E9017038
:10957000B8420CD00021236801EB070C9CFBF3F2EE
:1095800003FB12C2904205D10020884204D14FF063
:10959000FF3031E00131EFE7C21992FBF3FE03FB2C
:1095A0001E2ED4F80CC01CF80EE0BEF10A0F26D116
:1095B00028B3013A92FBF3F103FB1122002106F1DB
:1095C000FF3E71450ED2E7686368FB5C6B546768C9
:1095D0002668013797FBF6F306FB137701318842C3
:1095E0006760EEDA1CF802300D2B4FF0000304D157
:1095F000054405F8013C0138F8BD2B54FCE7013067
:10960000C3E700BFB0BB01084B1C017343738B1C45
:1096100003318373C17370472DE9F04107468846D3
:109620001E4615461AB952211548F9F7D1FFD7E958
:109630000143A34221D2E41ADEB1A3B9A5420ED35D
:109640003B7B3370BB6839682246194440460DF0B5
:10965000D0FABB682344BB602046BDE8F0817B7B29
:1096600033702C46EEE7A54201D3FB7BE9E7BB7BD9
:10967000F6E7AC4228BF2C46E4E70024ECE700BF45
:10968000EEBB01080023C0E900128360704710B5EB
:1096900004460846C4E900120021A16021730DF0C0
:1096A000CCFA204610BD000038B51546D0E901239C
:1096B00004465819904202D9257B55B1D51A206825
:1096C0002A4618440DF095FAA3681D44A5600125AB
:1096D00003E017210248F9F77BFF284638BD00BF99
:1096E00020BC010807B502AB03F8011D0122194691
:1096F000FFF7DAFF03B05DF804FB0068704780688D
:10970000704713B5044689B201A801F049F8022256
:1097100001A92046FFF7C8FF02B010BD13B50446EB
:1097200089B201A801F04AF8022201A92046FFF7F8
:10973000BBFF02B010BD13B5044601A801F030F81C
:10974000022201A92046FFF7AFFF02B010BD13B5FA
:10975000044601A801F037F8042220460DEB02016F
:10976000FFF7A2FF02B010BD08B50146044800F0A3
:109770000FFFBDE808400C210248F9F729BF00BFE0
:109780004EBC01086CBC010808B5044800F000FF9D
:10979000BDE808401E210248F9F71ABFC5BC010800
:1097A000F2BC010810B500F08FFF044630B9044840
:1097B00000F0EEFE27210348F9F70AFF204610BD0E
:1097C000B3BC0108F2BC010800F07EBF10B902482A
:1097D00000F0DEBE00F062BF9EBC0108FFF7E2BFF2
:1097E00000F072BFFFF7F2BFFFF7F0BFF8B50E460B
:1097F000054680B14F1C384600F066FF044640B174
:109800003A4600210DF019FA3246294620460DF05D
:10981000F0F92046F8BD0446FBE738B50D4604468E
:1098200028B10EF0BAF923462044834201D100202A
:1098300038BD13F8012BAA42F7D10120F8E737B55C
:1098400004460D460CF0E4FF002201A90260204608
:109850000EF0CEFA04460CF0DBFF0368222B08D092
:10986000019B1B782BB9002C03DB20462B6003B037
:1098700030BD012300202B60F9E700002DE9F04FF7
:1098800005464FF0010B002687B0CDE9031206F123
:109890000903122B8CBF0320022000F015FF00905B
:1098A000E8B1324636490EF001F9039B53F8269091
:1098B000EDB90024009800F0F1FEBBF1000F02D1D9
:1098C000284600F0EBFE84B1049B0136B3422546E6
:1098D0004FF0000BDBD1204607B0BDE8F08FBBF1A5
:1098E000000F02D1284600F0D9FE0024F3E7254BF3
:1098F0004FF00008B9F1000F08BF994648460EF036
:109900004CF9019000980EF048F90290284649461B
:109910000EF072F9B8B928460EF03FF9DDE90123DF
:1099200001309B1A08FB030000F0CEFE044600281D
:10993000BFD003462F4618F1FF3809D239461846E2
:109940000EF023F9B6E7019B08F101081844DEE7A1
:109950004946384605930EF04FF9059BA0EB070AE0
:109960005246394618460EF032F9009950440EF02E
:109970000CF9019A029B9244C3185744DBE700BFDD
:109980001EA10108ADA3010830B580B10346021F36
:1099900000F1180452F8045F8D4208D0A242F9D1B8
:1099A0001C301A4614680433013401D1116030BDF3
:1099B0008342F6D1FBE770B5044680B1064600EB62
:1099C0008105AE4204D12046BDE8704000F066BE7D
:1099D00056F8040B0028F4D000F060FEF1E770BDEB
:1099E0002DE9F74F89460092002838D00027C45D42
:1099F0008CBB05468346264600EB070AD34538D183
:109A000004B10136002E6FD00137384600F05CFEFD
:109A10008346002866D03A4600210DF00EF9B000CA
:109A200000F052FE0446002860D04FF00008414686
:109A3000AA4532D131B15846FFF7D8FE002855D09B
:109A400044F82800584600F029FE009B1E6020467E
:109A500003B0BDE8F08F0137B7F5807FC7D1002490
:109A60002646204600243146FFF7A5FF009B1C60D8
:109A7000EDE79BF800304B4505D10CB100240136D1
:109A80000BF1010BBAE70DF067F89BF800301844B2
:109A900043781B0758BF0134F2E72B784B4513D1AD
:109AA00081B15846FFF7A2FE00B308F1010344F864
:109AB000280000213A46584601930DF0BEF8019B5C
:109AC000002198460135B3E701910DF045F82B7858
:109AD00001991844407810F0080F04BF0BF80130CA
:109AE0000131EFE70446BCE73446B0E7584600F0E2
:109AF000D5FDB6E72DE9F743002506460820884640
:109B000091461F46009500F0DFFD0446002868D00E
:109B1000C0E9005530460EF040F801280FD13378E7
:109B20002A2B0CD109F1FF33C4F80080636022684E
:109B30004A4502D263684B4543D32B4B0EE02D219F
:109B40003046FFF76AFE0546C0B902A941F8040D88
:109B50003046FFF774FE019B63B1244B3B600099D4
:109B60002846FFF728FF002C37D0204600F096FD4E
:109B7000002432E0C4E900001D46D8E76A462D21E2
:109B80003046FFF72DFF009B0546013B012B01D915
:109B9000174BE3E7002302AE46F8043D3146006868
:109BA000FFF74DFE2060019B0BB1124BD6E731460B
:109BB0006868FFF744FE6060019B002BB7D00E4B36
:109BC000CCE7424501D3434501D20C4BC6E700998F
:109BD0002846FFF7F0FE00233B60204603B0BDE8B7
:109BE000F0830546BBE700BF00BE01087ABD01084F
:109BF00099BD0108C2BD0108E1BD010820BE0108F0
:109C000038B590B1451E15F8014F0CB9204638BD46
:109C10000CF0A2FF23462044427802F00302022AFD
:109C200008BFA4F120032B70EDE70120EFE708B592
:109C300020B34A1C22D0062920D8DFE801F0040D09
:109C4000101316191C00002303600DF0D9F808400A
:109C5000431C5842584108BD00234360F5E70023E8
:109C60008360F2E700238361EFE70123C360ECE741
:109C700000230361E9E700234361E6E70120EAE707
:109C800070B506460D1F01F1180455F8041F4B1C52
:109C900003D1A542F9D1002070BD3046FFF7C7FFC0
:109CA0000028F6D0F8E708234A4291FBF3F302F0CC
:109CB000070201F0070158BF51420122DBB2C9B2CD
:109CC00002FA01F1C25C1143C154704708234A42B1
:109CD00091FBF3F302F0070201F0070158BF514274
:109CE0000122DBB2C9B28A40C15C21EA0201C1543F
:109CF0007047082391FBF3F3DBB2C05C4B4203F0E7
:109D0000070301F0070158BF5942C9B2084100F0EA
:109D1000010070472DE9F047089E8A4690461D468F
:109D2000DDF82890074610B11446A24507D875B94A
:109D3000012200240B9B1A602046BDE8F0872146D3
:109D40003846FFF7D6FF002861D10134EDE7099BC3
:109D5000023B042B04D8DFE803F0282C2C3034001D
:109D60006B6801336B6028460DF04AF8013108BF7B
:109D7000B0F1FF3FDCD031462846FFF758FF0028FE
:109D8000D6D12FB3044621463846FFF7B2FF00284C
:109D900041D10134A245F6D10446013E042E19D822
:109DA000DFE806F02B2D2F313300AB680133AB60B9
:109DB000D9E7EB680133EB60D5E72B6901332B6101
:109DC000D1E76B6901336B61CDE7002DE5D1AFE7DA
:109DD0003C46E2E72C6028460DF012F8013108BF3E
:109DE000B0F1FF3FA4D0B9F1000FA1D049462846F9
:109DF000FFF746FF00289FD09AE76C60EBE7AC6066
:109E0000E9E7AC61E7E7EC60E5E72C61E3E7A04553
:109E1000DBD1444690E7A045BFD1FAE700232DE906
:109E2000F04F06468BB01C200C469046099300F07C
:109E30004BFC0546002800F0E4801C2000F044FCA8
:109E40000746002800F0DD804FF0FF31021F2B1F76
:109E500005F1180043F8041F984242F8041FF9D195
:109E600000230121D4F800A00DF12409CDE900312F
:109E7000CDE902793C21234652463046FFF74AFF9E
:109E8000099900296ED1824502D12846FFF77CFD51
:109E900002234FF0010AD4F804B0CDE900A3CDE9C4
:109EA000025923465A463C2106F10800FFF732FFCB
:109EB000099B002B56D183454CD151462846FFF7CC
:109EC00063FD03234FF0020AD4F808B0CDE900A3E4
:109ED000CDE9025923465A46182106F11000FFF732
:109EE00019FF099B002B3DD1834546D15146284699
:109EF000FFF74AFD40F26F1BA3690593E3680493E3
:109F000006F114030693DDF810A006F1130307937E
:109F100051460698FFF7EDFE28B105990798FFF71F
:109F2000E8FE002836D1BBF1010B33D0E3682046B0
:109F30000133E3600CF064FF013108BFB0F1FF3F73
:109F400024D0A36929462046D4F80CA00593FFF736
:109F500097FEDDE7424621463046FFF75FFF099056
:109F60000028AED0284600F099FB17B1384600F023
:109F700095FB09980BB0BDE8F08F4246214630466C
:109F8000FFF74CFF09900028ECD1B3E701234FF015
:109F9000000A0993099B002BE4D1049B534520D16F
:109FA00004212846FFF7F0FC05230622D4F810A070
:109FB000CDE90032CDE90259234652460C2106F183
:109FC0001800FFF7A7FE099B002BCBD18245C9D013
:109FD0006369A3EB0803042B0CD94FF0FF330993FB
:109FE000C0E7424621463046FFF718FF0990002897
:109FF000B8D1D9E7424621463046FFF70FFF099016
:10A00000B0E74FF0FF330993002DB2D00027A9E746
:10A010002DE9F04F002487B0924606AA894642F8FF
:10A020000C4D2C219846109DFFF7DAFC074688B9A5
:10A030003E4B2B6003993846FFF7BDFC07B0BDE8E7
:10A04000F08FD0F800B072685A451CD2304600F04C
:10A0500025FB0134039BA342ECD957F824602F2140
:10A060003046FFF7DAFBA8B92B4630464246514648
:10A07000FFF740FD2B680646002BE2D00028D9D020
:10A0800000F00CFBD6E759464846FFF70CFE0BF1F3
:10A09000010BD8E700232F21304604AA0493FFF7D1
:10A0A0009FFC049906464B1E012B04D9204B2B60C4
:10A0B000FFF781FCBEE742462B4651460068FFF79A
:10A0C00019FD2A6883462AB108B100F0E7FA04991D
:10A0D0003046EDE72D213068FFF79FFB18B908F1F6
:10A0E000FF32CBF80420002306A941F8043D706834
:10A0F000FFF7A5FB059A00901AB10E4A58462A6050
:10A10000E3E7DBF80020DBF80410914205D230468B
:10A110000499FFF750FC584699E7114648460192CA
:10A12000FFF7C1FDDDE900321A44ECE745BE010846
:10A1300057BE01087CBE01082DE9FF4100230E46F1
:10A140000393144602B902AC236048B90546564B46
:10A15000236003992846FFF72EFC04B0BDE8F08188
:10A1600003AA2021FFF73CFC039B0546062B02D0E7
:10A170004E4B2360EDE71A22002130460CF05DFDC6
:10A18000009400223C2331462868FFF741FF2268F3
:10A19000002ADED100943C2306F108016868FFF72D
:10A1A00037FF2268002AD4D10094182306F1100149
:10A1B000A868FFF72DFF2368002BCAD16869FFF755
:10A1C0001FFD07223A496869FFF758FB80460DF0EA
:10A1D000E4FC012806F1130706D198F800303F2B64
:10A1E00004BF2A2388F8003000220823394640465D
:10A1F0000094FFF70DFF404600F050FA2268002A55
:10A20000A7D107213846FFF774FD30B11146384613
:10A21000FFF749FD0721FFF759FDEF6806F1140824
:10A2200038460DF0BAFC012804D13B783F2B04BF1F
:10A230002A233B7020230022414638460094FFF732
:10A24000E7FE00214046FFF741FD2368002B80D147
:10A250002F693846FFF7D4FC00287FF47AAF3846E0
:10A260000D221449FFF70AFB074600283FF471AF9F
:10A27000183600940D2301223146FFF7C9FE3846F7
:10A2800000F00CFA012421463046FFF732FD30B1D0
:10A29000611E3046FFF707FD2146FFF717FD013429
:10A2A0000D2CF0D155E700BF24BD01083CBD0108CD
:10A2B000A0000020BC000020F0B58DB0CDE9002347
:10A2C000054628B94FF0FF304FF0FF310DB0F0BD1B
:10A2D0002422002103A80CF0B0FC03A968460CF06E
:10A2E0008BFB04460028EDD00CF08AFD4A1C08BF09
:10A2F000B0F1FF3F06460F46E4D06269214628468A
:10A30000FFF78CFD0028DDD120460CF079FD4B1CB9
:10A3100008BFB0F1FF3FD5D08F4208BF864203D0BF
:10A3200020460CF06DFDD1E7236820460133236001
:10A330000CF066FD013108BFB0F1FF3FC2D0626989
:10A3400021462846FFF76AFD0028E9D0BAE770B534
:10A350003C258AB0DDE90E64019496FBF5F405FB1B
:10A3600014640294182493FBF4F505FB1433CDE92F
:10A370000330481E0C2190FBF1F301FB1301002375
:10A38000CDE907339DF84030A2F26C7201A8059127
:10A39000069209930CF034FD0AB070BDF7B504467F
:10A3A00002A860E902230CF015FB0269037A551C30
:10A3B000426990F804C0077B02F26C71067EC269A4
:10A3C0000068A3700033207018BF012320460132BB
:10A3D00084F801C0E7702571A4F80510E6712272B7
:10A3E000637203B0F0BD30B5457A85B0C478837828
:10A3F000B0F8052001790295057801954078009024
:10A400002046FFF7A4FF05B030BD2DE93048D0E964
:10A4100000BCBCF1004F08BFBBF1000F05D01BEB27
:10A4200002044CEB0305C0E90045BDE830889042CA
:10A4300071EB0303B4BF012000207047032210B565
:10A44000104986B00B78013393FBF2F202EB420223
:10A450009B1A0D4A0B7052F823400278B0F8053071
:10A46000049242781A21039282780292C278019271
:10A47000027920460092054A0DF0E4FA204606B023
:10A4800010BD00BF2A0E002028BF0108EBBE010846
:10A49000B1F1004F08BF00281FB502460B4608D097
:10A4A00001A8FFF77BFF01A8FFF7C8FF05B05DF823
:10A4B00004FB0148FAE700BF1DBF01082DE9FF4773
:10A4C00003220D462B4900280B78044603F10103B3
:10A4D00093FBF2F202EB4202A3EB0203264A0B705B
:10A4E00052F8236075F100033EDA4FF0010A44424E
:10A4F00065EB4505214A0023204629460BF0A2FFC3
:10A500001E4A07460023204629460BF09BFF1046B3
:10A5100019464FF4616200230BF094FF4FF461621F
:10A5200080460023204629460BF08CFF1046194632
:10A530003C2200230BF086FF3C228146002320466C
:10A5400029460BF07FFFCDF80080CDE901923B4614
:10A55000BAF1000F0BD00A4A1A2130460DF072FAF8
:10A56000304604B0BDE8F0874FF0000AC2E7054A64
:10A57000F2E700BF2A0E002028BF01088051010029
:10A5800009BF01080ABF01080FB404B070470000FA
:10A590000FB437B51B4C256855B903222946012055
:10A5A000F8F726FB2B462A4629462060F8F744FB9D
:10A5B000154D2A68013A03321ED864212068F8F745
:10A5C00027FD8022002111480CF037FB07AB069ACB
:10A5D00080210E4801930DF07BFE7F2803DD0C499E
:10A5E0000C480DF0D2FA2B680848984700232068E1
:10A5F0001A461946F8F720FB03B0BDE8304004B016
:10A60000704700BFB40E00202C0E0020340E002036
:10A61000AEBC0108AF0E00200FB410B50D4CA2B0B7
:10A620002268013A033210D825AB249A802102A86F
:10A6300001930DF04DFE7F2804DD07490DF18300E5
:10A640000DF0A3FA236802A8984722B0BDE8104095
:10A6500004B07047300E0020AEBC010870B504464F
:10A66000054E4518AC4200D170BD14F8011B3046B0
:10A67000FFF78EFFF6E700BF34BF010838B50C4680
:10A680001546FFF785FF20462946FFF7E7FFBDE89F
:10A6900038400148FFF77CBFACA3010810B5044661
:10A6A00070B1F8F7DBF92046F8F7C6F9F8F782F849
:10A6B000BDE81040034A938801339380F8F79AB8B5
:10A6C00010BD00BF3818002070B5234C8AB0226836
:10A6D00005460132226000283BD0632A1F4E0BDD65
:10A6E000F7F794FB0523002201A9F7F7C1FAF6F763
:10A6F000BDFF002330602360F6F7B8FF336803F531
:10A700007A73984204D9F6F7B1FF002330602360D2
:10A71000134A144C13781BB9236063600123137030
:10A72000F8F79CF92846F8F785F9064668B12A46F5
:10A7300000210CF082FAF8F73DF8238801332380DA
:10A74000F8F758F830460AB070BD6388013363806B
:10A75000F8E70646F6E700BFBC0E0020C00E00205A
:10A76000B80E002038180020006800BA7047008832
:10A7700040BA80B2704700687047837842781B0403
:10A78000007843EA022318437047FFF7F4BF0B0E2B
:10A7900003700B0C43700B0A8370C1700420704768
:10A7A0000B0A03704170022070470B0A017043705E
:10A7B0000B0C090E8370C170042070470170090AE8
:10A7C000417002207047C1F3072301704370C1F349
:10A7D0000743C1F307618370C17004207047A0F183
:10A7E0004103052B02D83738C0B27047A0F161038E
:10A7F000052B01D85738F7E73038C0B20A2828BFF0
:10A80000FF2070470022013910B50144441E8C42DC
:10A8100004D014F8010F08B1002A01DA104610BD67
:10A82000FFF7DDFF0F2802D840EA0212EFE74FF0F2
:10A83000FF32F3E738B505460C460DF065F8611BAD
:10A84000013190FBF1F303FB1100284438BD0000F7
:10A8500010B504460DF034F8014B1C6010BD00BF6C
:10A86000F0000020024B1868013018600DF028B885
:10A87000F000002038B5451E15F8014F04B938BD69
:10A880000CF06AF923462044427802F00302012AC0
:10A8900008BF20332B70EFE72DE9F04106460DF09D
:10A8A0007CF930B3002734180CF056F914F8013C49
:10A8B000354618444378621E19070DD42F463B785D
:10A8C000A4EB050801355BB908F1010239463046B1
:10A8D000BDE8F0410CF098B904F8017C1446E3E7B8
:10A8E0000CF03AF915F8013C184443781B07E5D4FD
:10A8F000EAE7BDE8F08108B50DF03DF9B0FA80F067
:10A90000400908BDF8B50F4CD4F88032984723466B
:10A9100010F5617641F1000704F52072D3E908458E
:10A92000A04271EB050401DAC3E90801D3E9064549
:10A93000A64277EB050401DAC3E9066728339342A0
:10A94000ECD1F8BDC80E002010B5044618B9BB21E3
:10A950000748F8F73DFE074BD3F880329847D4E913
:10A960000623904271EB0304B4BF101A002010BDFF
:10A9700014C10108C80E00202DE9F84F064628B979
:10A98000BDE8F84FDC213448F8F722BE0023334AF3
:10A990001C469246D118097A2833B14208BF0134C7
:10A9A000B3F5207FF6D1002C54D0062E03D94021D8
:10A9B0002948F8F70DFE2A4B53F83650002D47D1A1
:10A9C000E7212548F8F704FE4FF0000B65430AEB3A
:10A9D0000B04227AB24235D16268002A32D0226951
:10A9E000012A03D1D0211C48F8F7F2FDD4E906234F
:10A9F00019461343104624D0D4E90889B0EB080067
:10AA000061EB09010BF0D4FA0746206901380BF01D
:10AA1000B5FA014638460BF0BDFB074628460BF059
:10AA2000ADFA39460BF002FB39460BF0F5F90BF0A5
:10AA3000E9FC18EB000249F1000310461946C4E98D
:10AA4000060125610BF1280BBBF5207FBFD101E08A
:10AA5000012DB9D1BDE8F88F14C10108C80E00203E
:10AA60003CBF01084FF47A73B0FBF3F341F6583260
:10AA7000A3F55223A3F6183393422DD81B4B1C4A3F
:10AA80000344934228D91B4B1B4A0344934223D9C6
:10AA90004CF24E32194B034493421DD9184B984245
:10AAA0001CD903F5371303F5D863984218D903F579
:10AAB000122303F5F863984214D903F5122303F522
:10AAC000F863984210D903F5DB2303F5BA63984283
:10AAD00094BF052006207047002070470120704772
:10AAE0000220704703207047042070473F373ACC5C
:10AAF0009E8601007F0F31CC3E0D0300AF312ACC82
:10AB000040DA8E332DE9F04385B0E0B1D0E9039807
:10AB10004FF47A740D4B4168D3F88C62037AB1FB21
:10AB2000F4F4062B96BF0A4A0A4D52F823500778D0
:10AB3000FFF70AFFCDF80080CDE901903B462A4699
:10AB400021460548B04705B0BDE8F083C80E002097
:10AB500074BF010894C00108A1C0010870B5134C6E
:10AB6000054694F894320E4623B94FF49671104876
:10AB7000F8F72EFD25B940F22D110D48F8F728FD04
:10AB800026B94FF497710A48F8F722FD00232822CE
:10AB900002FB03F0215CA94203D120444168B14289
:10ABA00003D00133102BF3D1002070BDC80E00205C
:10ABB00014C101082DE9F04F2E4F9A4697F89432B0
:10ABC00093B00191934623B940F241112A48F8F716
:10ABD000FFFC0025FFF796FEA9464FF0FF382C46F4
:10ABE000282303FB0576019AF368934218DBBBF137
:10ABF000000F10D13046FFF7A7FE80B3404536D393
:10AC00000ED1D4E90823D6E90801FFF710FC00288B
:10AC100018BF344604E000213046D8470028E9D167
:10AC20000135102DDCD1BAF1000F01D0CAF8008037
:10AC3000B8F1000F0FD1B9F1010F0CD909F1FF31B3
:10AC40004046FFF7F7FD12AB03EB8000282350F8D6
:10AC5000404C03FB0474204613B0BDE8F08F12ABE8
:10AC600003EB890343F8405C09F10109C6E780461C
:10AC70003446D5E7C80E002014C1010800000000CA
:10AC80002DE9F14F0D46044620B94FF4C27120481A
:10AC9000F8F79EFC236923B940F285111C48F8F7A8
:10ACA00097FCDFF87490D9F8803298478B4682463B
:10ACB0002069C4E908AB0BF061F929460BF0B6F93D
:10ACC00029460BF0A9F80AF019FD0FA3D3E90023D8
:10ACD0000AF096FE0AF054FA0BF02AF81AEB000676
:10ACE0004BF100078046C4E9066728460BF064FB79
:10ACF000D9F88C5202464346AC466168054801B01B
:10AD0000BDE8F04F604700BF0000000080842E4186
:10AD100014C1010890BF0108C80E00202DE9F041C0
:10AD20000E461746054620B94FF4C8711348F8F788
:10AD30004FFC26B940F291111048F8F749FC002168
:10AD400038460BF02FFB20B94FF4C9710B48F8F7C8
:10AD50003FFC0024DFF8288014F80830AB4207D10C
:10AD600008EB04004368B34202D13946FFF788FF7D
:10AD70002834B4F5207FEFD1BDE8F08114C101087B
:10AD8000C80E002008B5FFF76DFE003018BF012087
:10AD900008BD00002DE9F0473F4F94B097F894327A
:10ADA00006460D4623B94FF4D9713C48F8F710FC1C
:10ADB0002846FFF7E7FF044658B94FF47A71384840
:10ADC000D7F89032B5FBF1F19847204614B0BDE8B2
:10ADD000F08729463046FFF7C1FE0028F6D18046AD
:10ADE000282303FB0879D9F804202AB108F10108C7
:10ADF000B8F1100FF5D1E9E797F894321BB9772134
:10AE00002648F8F7E5FB1EB978212448F8F7E0FB5F
:10AE1000282200210DEB02000BF00FFF2846FFF760
:10AE200021FE062804468DF8300003D940211B4836
:10AE3000F8F7CEFB0B956D464FF0280A194B8DF8AD
:10AE4000286003EBC402526853F834300AACCDE9F1
:10AE50000D230FCC0FC50FCC0AFB087A0FC594E861
:10AE600003006E46544685E803000FCE0FC40FCE94
:10AE70000FC495E80300D7F88C3284E803004146FC
:10AE8000094898474846FFF73DFE9AF80800FFF743
:10AE900073FD48469AE700BFC80E002014C10108A0
:10AEA00044C001083CBF010873C001080D4B10B538
:10AEB00093F89432044623B94FF4EA710A48F8F73C
:10AEC00087FB6CB163685BB10848FFF761FB204604
:10AED000FFF718FE0023207A63602372FFF74CFD12
:10AEE000002010BDC80E002014C1010804C10108D3
:10AEF0002DE9F041124D074695F89432884623B962
:10AF00004FF4F6710F48F8F763FB27B940F2ED11E3
:10AF10000C48F8F75DFB002426462B5DBB4208D1A8
:10AF200028194368434504D1FFF7C0FF002818BF24
:10AF300006462834B4F5207FEFD13046BDE8F081D5
:10AF4000C80E002014C1010870B5114C064694F8D3
:10AF5000943223B94FF4FE710E48F8F739FB26B945
:10AF600040F2FD110B48F8F733FB0025635DB34257
:10AF700004D1601943680BB1FFF798FF2835B5F588
:10AF8000207FF3D1D4F88C320348BDE870401847D5
:10AF9000C80E002014C10108E8C001082DE9F843DB
:10AFA000154D06460F4690460024A946635DB34200
:10AFB00009D12B195A6832B1002398450DDC09EBF1
:10AFC0000400FFF773FF2834B4F5207FEED100248E
:10AFD000A04508DC0120BDE8F88357F823108A4219
:10AFE000F1D00133E9E757F824103046FFF7D2FEDD
:10AFF0000028F0D00134EBE7C80E0020014B93F895
:10B0000094027047C80E002010B5074C2378FA2B25
:10B0100004D94FF40D710548F8F7DAFA20780130B9
:10B02000C0B2207010BD00BFC40E002014C10108C2
:10B0300084B070B504AC84E80F001C4B93F89412F4
:10B040001C4631B1BDE87040D3F89032184804B0C6
:10B0500018474FF42672184604F5207504AE0BF01D
:10B06000ECFD0FCE0FC533682B6013B9114BC4F83C
:10B070009032D4F88C3213B90E4BC4F88C32D4F819
:10B08000883213B1D4F884324BB9D4F88C320A48E0
:10B0900098470A4BC4F88832094BC4F8843201231C
:10B0A00084F89432BDE8704004B07047C80E0020A8
:10B0B000D0BF010889A5000809C00108856B0108F7
:10B0C000756B01082DE930080F4B03F52072D3E9A9
:10B0D00008BC5BEA0C0405D01BEB00044CEB01053B
:10B0E000C3E90845D3E906BC5BEA0C0405D01BEBB9
:10B0F00000044CEB0105C3E9064528339342E6D131
:10B10000BDE83008FFF7FEBBC80E002070B504464E
:10B11000044E451814F8011B3046FFF739FAAC42CB
:10B12000F8D170BD7BE0010870B515460022C0E97A
:10B1300001150270C0E90332C0E90522C0E9072207
:10B140004262DDE90412044600F11C06F8F7FEFE37
:10B1500038B929460748FFF71BFA2B210648F8F7AC
:10B1600037FADDE9042331462046F8F7DCFE2046B5
:10B1700070BD00BFAB970108D69701082DE9F041DB
:10B1800000259DF81860C0E901120570C0E903357B
:10B19000C0E90555C0E907554562314604461746E2
:10B1A00000F11C08F8F7D6FC38B939460748FFF714
:10B1B000EFF920210648F8F70BFA324641462046BF
:10B1C000F8F7B6FC2046BDE8F08100BFAB97010858
:10B1D000D6970108F0B50125044608270E468DB024
:10B1E000564B574A2946009502A8FFF7C7FF02A908
:10B1F0002046FAF75DF802A8F4F7A8FF514BCDE915
:10B2000000671A460DEB07000421FFF78DFF0DEBD9
:10B2100007012046FAF74CF80DEB0700F4F796FF0C
:10B22000F319494A019700930DEB0700474B04219E
:10B23000FFF77AFF0DEB07012046FAF739F80DEB1F
:10B2400007001027F4F782FFF3190093404B019792
:10B250001A46042102A8FFF767FF02A92046FAF761
:10B2600027F8203602A8F4F771FF3A4B3A4A0096C5
:10B270000197042102A8FFF757FF02A92046FAF719
:10B2800017F802A8F4F762FF0C230026334A009354
:10B290000221334B02A8F5F71FF802A92046FAF75E
:10B2A00007F802A8F4F752FF2E4B2F4A29460095C3
:10B2B00002A8FFF763FF02A92046F9F7F9FF02A8E9
:10B2C000F4F744FF294B2A4A0096022102A8F5F719
:10B2D00003F802A92046F9F7EBFF02A8F4F736FFBE
:10B2E000244B254A0096022102A8F4F7F5FF02A993
:10B2F0002046F9F7DDFF02A8F4F728FF1F4B204A8C
:10B300002946009502A8FFF739FF02A92046F9F760
:10B31000CFFF02A8F4F71AFF06231A4A009302216E
:10B32000194B02A8F4F7D8FF02A92046F9F7C0FF8D
:10B3300002A8F4F70BFF0DB0F0BD00BFDFC101089C
:10B34000B8B40108F2C10108C9C50108B0C50108B7
:10B3500000C20108D1C50108FBC5010898B4010865
:10B3600007C2010860C20108A9D4010802C6010889
:10B370009BB4010840C60108A4B401087BC60108BB
:10B3800085A20108ADB4010897C6010870B504464E
:10B3900090B00146924A01A8F9F703FD914A21466F
:10B3A00004A8F9F7FEFC904A214607A8F9F7F9FC32
:10B3B0008E4A21460AA8F9F7F4FC8D492046F9F790
:10B3C000E7FC05468B48FFF7E3F8DDE901239B1A0C
:10B3D000082B06D08848FFF7DBF8B1218748F8F73B
:10B3E000F7F8DDE904239B1A082B06D08448FFF701
:10B3F000CFF8B5218148F8F7EBF8DDE90A239B1A6D
:10B40000102B06D07F48FFF7C3F8B9217B48F8F727
:10B41000DFF8DDE907135B1A102B0CD101234A1E5C
:10B4200001F10F0012F8016F002E18BF00239042A7
:10B43000F8D1002B53D07448FFF7AAF85DB37348D6
:10B44000FFF7A6F8674A21460DA8F9F7AAFC70484D
:10B45000FFF79EF808210198FFF758FE6D48FFF7A7
:10B4600097F808210D98FFF751FE6B48FFF790F809
:10B4700010210A98FFF74AFE6848FFF789F80D98EF
:10B480000A9A019900F076FF0DA8F8F727FF6448A3
:10B49000FFF77EF861E06348FFF77AF86248FFF74C
:10B4A00077F80A99019800F0C7FE6048FFF770F836
:10B4B000042101980844FFF729FE5D48FFF768F86A
:10B4C00010215C48FFF722FE5B48FFF761F810216E
:10B4D0005A48FFF71BFE5148FFF75AF8D7E71022EA
:10B4E0000A980BF077FB5649564B002818BF1946AF
:10B4F0005548FFF74DF8002D40D04448FFF748F875
:10B50000384A21460DA8F9F74CFC5048FFF740F89F
:10B5100008210198FFF7FAFD4D48FFF739F8082197
:10B520000D98FFF7F3FD4B48FFF732F8102107980D
:10B53000FFF7ECFD4848FFF72BF810210A98FFF7BA
:10B54000E5FD3648FFF724F80D98079B0A9A019904
:10B5500000F026FF0DA8F8F7C1FE3048FFF718F8F5
:10B560000AA8F8F7BBFE07A8F8F7B8FE04A8F8F792
:10B57000B5FE01A8F8F7B2FE10B070BD2948FFF77C
:10B5800007F83648FFF704F8079A0A99019800F07F
:10B5900095FE2648FEF7FCFF042101980844FFF7BA
:10B5A000B5FD2F48FEF7F4FF10212248FFF7AEFD4E
:10B5B0002C48FEF7EDFF10212B48FFF7A7FD2B4885
:10B5C000FEF7E6FF10212A48FFF7A0FD2948FEF705
:10B5D000DFFF1A481021FFF799FD104858E700BF18
:10B5E000F2C10108C9C50108FBC5010800C2010874
:10B5F000B8B4010892C20108A9C20108B9C2010881
:10B60000ECC20108FDC201080DC3010828C30108EE
:10B610002EC301083FC3010851C30108ACA30108B0
:10B62000F9C3010871C3010876C30108A8C3010862
:10B63000BAC3010894020020E6C30108C402002036
:10B640007BC20108ADA3010818C4010835C4010874
:10B6500047C401085AC401087AC40108C5C40108D6
:10B66000FFC401086BC50108A402002082C50108BF
:10B67000B402002099C5010810B5084CD4F8342252
:10B680001AB95A210648F7F7A3FFD4F83402002369
:10B69000BDE8104003222021F6F716BDF800002077
:10B6A00071CB0108F0B51F461446C7B005460E46DB
:10B6B000F122002109A80BF0C0FA09AA102138468E
:10B6C00003F00EFC20460CF068FA07461022002119
:10B6D00001A80BF0B2FA102F3A46214628BF1022DB
:10B6E00001A80BF086FA09AA05A901A803F072FCCB
:10B6F000324605A928460BF07CFA47B0F0BD0000A1
:10B7000037B5104C104D94F82F30022B15D123680B
:10B710000E48984794F8213094F8F3210093D4F818
:10B72000F4110823012003F08DFB6B6B0020984778
:10B73000042384F82D3003B030BDEB6A9847012311
:10B74000F7E700BFF80000204CEF0108A7CB010885
:10B75000044B5A7F22B993F8330080F00100704700
:10B7600000207047F8000020F0B570279DB0064615
:10B770000D463A46002168460BF05FFA08212B4639
:10B780000DEB010004AC0B4AFFF78CFF2B46204663
:10B79000094A102108ADFFF785FF94E80F0085E8FE
:10B7A0000F003A46694630460BF023FA30461DB08A
:10B7B000F0BD00BF62CB01086ACB010808B505489F
:10B7C000FEF7E6FE044A92F8F831013382F8F831C8
:10B7D00008BD00BFC0C90108F80000200022024BCC
:10B7E00083F8F821704700BFF8000020014B93F860
:10B7F000F9017047F800002084B070B58AB00EAC33
:10B8000084E80F00764C4FF4107225460021204644
:10B810000EAE0BF012FA0FCE0FC596E8030014AB74
:10B8200085E803000FCB04F1180585E80F000E9B97
:10B830000BB96C4B23600F9B0BB96A4B2360109BB9
:10B8400023B940F285116848F7F7C2FE129B23B96D
:10B8500040F289116448F7F7BBFE119B23B940F20F
:10B860008D116148F7F7B4FE139B23B940F2911193
:10B870005D48F7F7ADFEA36923B923685B48984795
:10B880000323A36102F09EFA94F8203013B9012338
:10B8900084F8203002F08EFA94F8213013B90E2388
:10B8A00084F82130636A0BB9514B636202F076FA77
:10B8B00006F0F6FEC4F830020138033008D94D48CE
:10B8C0006368984700200AB0BDE8704004B0704734
:10B8D000002204210120F7F78BF90322C4F83C026F
:10B8E00000210120F7F784F9C4F8380220B94FF499
:10B8F000DD713D48F7F76CFE002204210120F7F7C7
:10B9000077F9C4F83C0120B94FF4DF713648F7F7F6
:10B910005FFE002204210120F7F76AF9C4F8400114
:10B9200020B940F2C1113048F7F752FE4FF481635D
:10B93000A4F80032002384F83430012384F8043260
:10B94000FFF75CFB05AD68B9A3682269059323681E
:10B9500007920893E26863680692009395E80F00E7
:10B96000FFF766FBFFF750FB84F8320002F06AFA3B
:10B970002368214E0793636806F1A00208932369A8
:10B9800004960693E368F03605930AAB43F81C2D42
:10B9900093E803008DE8030095E80F0002F0BCFC7B
:10B9A0000196A3694FF4CD72009314490123144802
:10B9B000F5F71AFC012804D04FF4F3710A48F7F7A1
:10B9C00007FE002303220421D4F83402F6F77CFB9F
:10B9D0000C4823689847012084F8310073E700BFC2
:10B9E000F800002089A5000871CB0108F1C7010803
:10B9F00008E6D3333AC801083C0200206DC80108AC
:10BA0000B5BF000875C8010810B5124CD4F834321F
:10BA100023B940F2EF111048F7F7DAFD03220421B1
:10BA20000023D4F83402F6F74FFB23680B489847FD
:10BA300042F21071D4F83802F7F7EAFA0023D4F88A
:10BA400038021A461946F7F7F7F823680448BDE8A4
:10BA500010401847F800002071CB01082CC90108DC
:10BA600053C9010838B50E4DD5F8383223B94FF413
:10BA700000710C48F7F7ACFD0021D5F83802F7F754
:10BA8000C7FA0128044608D10023D5F838021A461F
:10BA90001946F7F7D1F8204638BD0020FCE700BF73
:10BAA000F800002071CB010810B5FFF7DBFF0B4C4D
:10BAB00078B1002303220821D4F83402F6F704FBFE
:10BAC000236807489847D4F83402BDE81040F5F7DA
:10BAD00039BD23680348BDE810401847F80000202E
:10BAE0006EC9010890C90108002313B502A941F8E5
:10BAF000043D4EF65E224EF66023441E94428CBFF7
:10BB000002461A46034BD3F84001F7F7EFF90198C4
:10BB100002B010BDF8000020F8B5FFF7A3FF1D4DDF
:10BB200020B16B681C4898470020F8BDD5F83C014F
:10BB3000F7F7FCFB074610B12B681848F3E70146FE
:10BB400002F0E6FC064610B92B681548EBE70770D3
:10BB500002F026F8044618B9304602F027FDE3E764
:10BB6000104A1368013313608BB9136801331360F3
:10BB7000636004232046237002F036F828B90A488F
:10BB80002B689847204602F01DF86068CDE71368DF
:10BB9000EEE700BFF800002092C80108BEC8010807
:10BBA000D5C8010860110020FBC801082DE9F04349
:10BBB0008DB08146884617460393FFF753FF604DCB
:10BBC00038B12B685F489847002420460DB0BDE887
:10BBD000F083D5F83C01F7F7A9FB044610B12B68B8
:10BBE0005948F0E72FB9B8F1000F08D02B68574833
:10BBF000E9E7E02F03D92B6855489847E5E7414628
:10BC0000484602F085FC064610B92B685148DAE731
:10BC10009DF80D30002B59D004230370FFF7CEFDA3
:10BC20000F2208A905A80DF088FC9DF80C303BB147
:10BC30000D230CA901F8203D012205A80DF08BFC75
:10BC40009DF80E303BB102230CA901F8203D0122E2
:10BC500005A80DF080FC95F82E2095F82F30934222
:10BC600003D195F83030934217D02023022A18BF11
:10BC700000228DF8103096F8783004A90BBF43F0FD
:10BC8000040343F001038DF811208DF8112005A85D
:10BC900086F8783002220DF05EFC95F81432079C8D
:10BCA00095F8F0011C44E4B2214602F085FA804583
:10BCB00002460ED995F8F031414600932D6823468F
:10BCC0002548A847304602F071FC7DE70223037047
:10BCD000A6E7079A62B1D2B20599304600F088FD16
:10BCE000044628B9304602F061FC2B681B4884E703
:10BCF0007777304601F054FF07460028E2D0002352
:10BD0000174A836013680133136083B913680133E2
:10BD100013607B60022338463B7001F065FF0446E8
:10BD200038B9384601F04EFF6B680E4865E7136876
:10BD3000EFE72B6879680C4898477C6845E700BFB7
:10BD4000F800002004CA0108BEC8010820CA010882
:10BD500044CA010864CA01089FCA0108E0CA010870
:10BD600060110020FBCA010815CB0108034B93F8B2
:10BD7000141293F8F00102F01FBA00BFF80000207F
:10BD80000E2808BF0120024BD87783F8F0017047D6
:10BD9000F8000020024B83F8200083F8F10170477F
:10BDA000F8000020014B83F821007047F8000020C4
:10BDB00008B5FEF7D9FC024BC3F8480108BD00BF27
:10BDC000F8000020034630B5054C00F1100522466E
:10BDD00018685968083303C2AB421446F7D130BD26
:10BDE000B4020020034630B5054C00F11005224690
:10BDF00018685968083303C2AB421446F7D130BD06
:10BE0000A4020020034630B5054C00F1100522467F
:10BE100018685968083303C2AB421446F7D130BDE5
:10BE200094020020034630B5054C00F1100522466F
:10BE300018685968083303C2AB421446F7D130BDC5
:10BE4000C402002010B50446FFF7BCFF2046FFF7F0
:10BE5000C9FF2046BDE81040FFF7D4BF30B510251C
:10BE6000C3B0224CF122002105A80AF0E6FE2A46C2
:10BE7000002101A80AF0E1FE94F85B3105AA8DF8D3
:10BE8000053094F85A3129468DF8063094F8593126
:10BE900004F5B6708DF8073094F858318DF80830F5
:10BEA00094F857318DF8093094F856318DF80A30EE
:10BEB00094F855318DF80B3094F854318DF80C30DE
:10BEC00003F00EF8052305AA04F5C67101A88DF844
:10BED000043003F07FF8062305AA04F5BE7101A81B
:10BEE0008DF8043003F076F843B030BDF800002040
:10BEF0000246024B0068516803C3704744020020A9
:10BF00000246024B0068516803C370474C02002090
:10BF1000034630B5054C00F11005224618685968F3
:10BF2000083303C2AB421446F7D130BD540200209F
:10BF3000034630B5054C00F11005224618685968D3
:10BF4000083303C2AB421446F7D130BD640200206F
:10BF5000014B9877704700BFF800002030B1044BC8
:10BF6000044A02280CBF1846104670470248704722
:10BF7000FCC9010859C10108F4C9010870B505469A
:10BF8000FFF7ECFF034C014626680348B04784F8EE
:10BF90002E5070BDF800002047CB010838B504468C
:10BFA00000680D46884203D008B101F00BFE256001
:10BFB00038BD00002DE9F041FEF754FC0123834C0D
:10BFC000DFF81082824E84F82D300A23814A4FF028
:10BFD000FF310020F6F72EF8012866D1D8F80000CE
:10BFE00043071DD5337833B106F0A6FA002006F0DA
:10BFF000F7FA00233370F6F7DDFB2368764898479D
:10C00000F6F7F8FB022384F82D300023D4F8380229
:10C010001A461946F6F710FE0020F5F7FDFCD4E7A6
:10C0200010F0080724D0337893B941F2883006F035
:10C03000AFFA18B99B216948F7F7CAFA684806F0C1
:10C04000CFFA01236748337023689847FFF758FBFE
:10C050000020F6F733F94FF4FA61D4F83802F6F716
:10C06000D7FF0028B1D1A2215C48F7F7B1FAACE7BD
:10C0700010F0200046D03378A3B194F82D30042B73
:10C0800010D1594D3A462946D4F83002F7F770F8E6
:10C09000012807D12B78072B24D1236853489847D0
:10C0A00001F0FCFC0020F6F709F93378002B8CD066
:10C0B00001F0AEFD0546002887D00378012B27D17B
:10C0C00094F82C10A26A01B1FAB9B2FA82F2484887
:10C0D0005209FEF75DFA284601F00EFE284601F0EF
:10C0E00071FD72E73A462946D4F83002F6F7FEFEB3
:10C0F0000128D7D1236829783E489847284606F07A
:10C1000075FACFE7F6F7DAF85FE701F05BFDA56AAD
:10C11000032384F82D302B782768052B98BF364AE7
:10C12000696894BF52F82320344A3548B8472B78C1
:10C13000052B46D8DFE803F003450A0A3A3AD52131
:10C140002648F7F745FAFFF7DBFA3EE729462D4880
:10C15000FFF724FFFFF7FCFA68B101F06BFD05461D
:10C1600018B9E1211D48F7F733FA022328462B704E
:10C1700001F09CFDE7E701F05DFD074618B9E821F5
:10C180001648F7F725FA3946284600F037F97B7E3E
:10C1900053B14FF47A70F5F7C1FB3946284600F0E9
:10C1A0002DF97B68002BF2D03846E1E715480021D5
:10C1B000FFF7F4FE284601F007F8284601F002FDDB
:10C1C000C1E7636810489847F7E700BFF800002010
:10C1D0006411002074110020E0C6010871CB010831
:10C1E00079B6000803C701086811002033C70108A9
:10C1F0006FC701084AC70108C8C6010859C101082C
:10C20000AFC7010820010020CDC7010813B50024E5
:10C21000074802AB90F8F11143F8044D054A90F835
:10C220003200FEF7C7FC2146019802B010BD00BFE6
:10C23000F8000020D5C3000830B50430C7B00D4663
:10C24000FFF7B6FD1B4B0DF1050203F10C0153F88E
:10C25000040B8B4242F8040BF9D11B880124138094
:10C2600000238DF81330022309AA102128468DF8E7
:10C27000043002F035FE09AA05A901A802F0AAFEC1
:10C2800005A8FFF7CFFD09AA102128468DF8044024
:10C2900002F026FE09AA05A901A802F09BFE05A846
:10C2A000FFF7D0FD1022044B5C771A7783F8442106
:10C2B00047B030BD1DC90108F800002030B504307A
:10C2C000C7B00C461546FFF773FD284B0DF105026C
:10C2D00003F10C0153F8040B8B4242F8040BF9D123
:10C2E0001B882046138000238DF81330022301247D
:10C2F00009AA10218DF8043002F0F2FD09AA05A95F
:10C3000001A802F067FE05A8FFF78CFD09AA10211D
:10C3100028468DF8044002F0E3FD09AA05A901A80A
:10C3200002F058FE05A8FFF74DFD032309AA05A951
:10C3300001A88DF8043002F04DFE05A8FFF752FD6C
:10C34000042309AA0DEB030005A98DF8043002F0BF
:10C3500041FE05A8FFF756FD1122054B5C771A77C1
:10C3600083F8442183F8FD4147B030BD1DC9010861
:10C37000F800002038B50D461446FFF7B9FD2846F1
:10C38000FFF7BEFD2046FFF7C3FD2046FFF7D0FDB7
:10C390000022024B5A7710221A7738BDF80000208D
:10C3A00070B50E4615461C46FFF7A2FD3046FFF756
:10C3B000A7FD2846FFF7ACFD2046FFF7B9FDBDE815
:10C3C00070400022024B5A7711221A77FFF746BDC0
:10C3D000F8000020002310B54168074C1A19106CB2
:10C3E000884202D192F83C0020B91033B3F5807F27
:10C3F000F4D1002010BD00BFF80000202DE9F04F5F
:10C40000064689B00C4619B918217148F7F7E0F8CB
:10C4100016B13378022B03D01A216D48F7F7D8F8FC
:10C4200033691BB91B216A48F7F7D2F833691B78C7
:10C43000042B05D0022B03D01D216548F7F7C8F85F
:10C44000644F3378644863703B6898470022D7F89C
:10C45000F43197F8F181029308AB43F80C2D414673
:10C460005E4A97F8320097F8F0B197F8F2A197F882
:10C47000F391FEF79FFB3D46024628B93B685848BA
:10C4800098470123237007E0059B43B101F014FF97
:10C4900003232370059B636009B0BDE8F08FB36888
:10C4A0000133012BB36013D1D7F8E41103900131AC
:10C4B0003069C7F8E411B7F8FE1187F82C30013164
:10C4C000A7F8FE1100F0FEF8306900F0BFF9039AFA
:10C4D000D5F8481133695960D5F8E411598195F8B8
:10C4E000F91141B1002185F8F911197A41F00401DF
:10C4F0001972B5F8FA11A3F87A10104601F0C8FCC9
:10C50000034695F8F02105EB00113069002780F80B
:10C510007D3080F87C2095F804224FF47A7312F075
:10C520000F0208BF01225A4307AB019306AB0093E9
:10C530003C3102F57A73069701F046F910B92B6881
:10C5400028489DE7F5F792F8F060D4F8A00027702E
:10C5500008B102F02BF8069B0798C4F8A030C4F885
:10C560000A0022463146204800F076F880223169E0
:10C5700004F120000AF03DFB0021029B0798636153
:10C5800095F83330C4F80A00C4F8881084F810B065
:10C5900084F8118084F812A084F813902170237617
:10C5A000B26895F80232D4F8A0009A4200D258B18D
:10C5B000617685F82C10003018BF0120617E009054
:10C5C0000A48FDF7E5FF67E701216176F3E700BF61
:10C5D000E2CB0108F800002015CC0108D5C3000803
:10C5E00039CC010873CC010820010020B3CC01082C
:10C5F00037B5164C10B10023A4F8FE31A37F1BB34E
:10C60000B4F8FE1194F8002291421DD994F8013239
:10C610008D1A95FBF3F003FB1050A8B90C48256860
:10C62000A84701F0D7FB20B901F0E2FB08B901F0FF
:10C63000EFFBE07F94F8F03194F8202094F8F111AA
:10C64000009024680348A04703B030BDF8000020E4
:10C650000CCD010862CD010870B5D2F8A0400646A5
:10C6600015460CB30021204601F086FEFFF7B6F810
:10C6700023782046052B01BF012386F8D131638939
:10C68000A6F8D231FFF7B4FFD5F80A10204600F023
:10C6900055FD237A5B0706D5084B61891B6808485E
:10C6A000984701232B7270BD2046FFF7A1FFD5F8F4
:10C6B0000A102046BDE8704000F040BDF8000020A0
:10C6C000F0CC010870B51F4C0546A37F002B38D075
:10C6D000037A94F8F02143F001030372E37F9A4256
:10C6E00008D194F83C3063B394F84C304BB394F8D1
:10C6F0005C3033B394F8013294F800222668B4F821
:10C70000FE111148B047B4F8FE2194F800329A4265
:10C7100017D994F8F021E37F9A4212D02B7A43F094
:10C7200002032B72FFF74AF82B7A256894F800224F
:10C73000B4F8FE11AC46BDE87040C3F340030348B3
:10C74000604770BDF800002091CD0108D1CD0108EF
:10C75000431EDBB21F2B96BF0D4A0023D35C0A2871
:10C760000BD8012202FA00F010F4A46F05D0094A98
:10C7700092F814221A440E2A07DC074A107818444B
:10C780000E28CCBF0020012070470020704700BF5A
:10C790000CCE0108F80000208711002070B5057844
:10C7A00004462846FFF7D4FF88B1094A094E13789A
:10C7B000F5540133137051B1074A247892F81432BA
:10C7C000D01880F805420846013382F8143270BD53
:10C7D0008711002078110020F800002038B100787F
:10C7E000032803D0431F5842584170470120704727
:10C7F000037A70B51B09D61804460F2E00F10C0001
:10C80000154618440E4E0DDC0AF0F3F9237A0D4854
:10C8100005EB131262F30713237229463368984716
:10C82000012070BDC3F10F020AF0E3F9237A064834
:10C8300043F0F00323722946336898470020F0E75D
:10C84000F800002029D4010848D4010873B5164E19
:10C8500005463278154CBAB11549FFF7C9FF0F22CA
:10C86000002113480AF0E9F90023337094F8FD31F0
:10C8700043B140F2011302A921F8043D02222846E7
:10C88000FFF7B6FF02B070BD94F814120029EDD086
:10C8900023680848984794F8142204F20521284692
:10C8A000FFF7A6FFE2E700BF87110020F800002095
:10C8B000781100206DD4010838B5064C00F00F0542
:10C8C00023682A4694F804120348984784F80452CF
:10C8D00038BD00BFF800002003D4010800000000AC
:10C8E0002DE9F04F002599B0CDE90C019DF888B0F5
:10C8F000904C11920E935D4518D20E9B8E485E1996
:10C900005B5D0493049A2368571EFAB21F2A96BFF0
:10C910008A498B4A51F82220049998470498FFF7D6
:10C9200017FF0A9028B98748FDF732FE19B0BDE815
:10C93000F08F1F2F00F2E283DFE817F02000E00302
:10C940002C0065030502E501B6024F036503F502FD
:10C95000E0036703B1018F039103E003E003E00309
:10C96000E003E003E003E003E003E003E003E003AF
:10C97000E003E003E003E003E003B503ABEB0503F2
:10C98000DBB2012B4FF0000700F0DB8184F8FD7172
:10C990000227D6E1ABEB0503DBB20B9307238DF83F
:10C9A0004C3000239A4607930B9A0AF104039A42EB
:10C9B00003DD16F80A30032B12D0079B43B123681E
:10C9C000614898479DF84C306FF300038DF84C3068
:10C9D0009DF84C30072B40F038814FF0000A2BE1D6
:10C9E00006EB0A03D3F801302768039314930AF186
:10C9F00005035FFA83FA9DF80C3054484FEA131987
:10CA000003F00F030593039B4946C3F30F230693DB
:10CA1000039B1B0EC3F3021203F00F030892019352
:10CA20000092DDE90523B847149BB9F1060F4FF0DA
:10CA30000007159304D9039B03F0F003F02B5FD19B
:10CA40004FF6FF72039B0699C3F3076303F070036D
:10CA5000602B18BF0A46002398461092099310993C
:10CA60005FFA88F001F0A0FA0F90A8B104EB081368
:10CA70001B6C8BB104EB081292F84420236802F07F
:10CA80000F01494537D8B9EB121F34D84246494601
:10CA90002F4898470F9B099308F10108B8F1100F30
:10CAA000DDD1099B0BB14FF00207059B072B2CD85A
:10CAB00047F00407089B1B01602B2ED147F00107AC
:10CAC000039BC3F3076313F0700305D0079A0A9919
:10CAD000602B18BF0A4607929DF84C30C7F34002FE
:10CAE00067F3000362F34103C7F3800767F3820330
:10CAF0008DF84C3058E74246494616489847CBE7F0
:10CB00002368494614489847CFE7059B0F2BCFD0A1
:10CB10002368059911489847CCE723B9069801F096
:10CB200021FA0028CAD12368089A06990C48984728
:10CB3000C6E700BFF8000020B4CE01082CCE0108E3
:10CB4000ACCE0108D5CE0108FFCF01080CCF0108FB
:10CB500057CF010879CF01089DCF0108B9CF01084F
:10CB6000D4CF010806EB0A03D3F801700AF10503DC
:10CB70005FFA83FA9DF84C30169703F00703072BF2
:10CB80005AD19DF85830B648C3F303135FFA83F9BE
:10CB900084F8F03149462368984707F00F030F2BBC
:10CBA0000DD033B901229DF8583062F303038DF89C
:10CBB00058309DF85830C3F3030384F8F1319DF8E1
:10CBC0005820236802F00F0294F8F111A548984705
:10CBD0009DF85B30C7F30F28C3F302131A46039383
:10CBE0004146A14823689847039B4A461946404658
:10CBF00001F0E0F920B940F275119C48F6F7E8FC25
:10CC000094F84431102B09D117F0706F01BF012245
:10CC10009DF85B3062F303038DF85B309DF85B7029
:10CC20003B0709D0C7F3030723683A4694F802127A
:10CC30008F48984784F802720B9A0AF104039A42CB
:10CC400003DD16F80A30032B8CD0BAF1000F16D092
:10CC5000032318A800F8083D0021FFF79FFD0021DD
:10CC600013A8FFF79BFD9DF84C10266801F0010307
:10CC70000093C1F38002C1F340037E48B04701F046
:10CC80001BFB05EB0A07FFB2BD4240F03E827A4B28
:10CC9000ABEB05021B6804997848984746E6ABEB76
:10CCA0000503DBB2052B40F2278233780D2B40F0D1
:10CCB0002382701CFDF75FFD96F905300021002BE3
:10CCC0001DDB63A3D3E90023002794F80462121844
:10CCD0004B4116EB020847EB0309119B022B03D1D2
:10CCE00018F1010849F100090C9923684246096FBF
:10CCF000634898470C9BC3E91C89062721E056A38B
:10CD0000D3E90023E0E73378062B40F0F58118A83B
:10CD100000F8103D0021FFF741FD0D9B18AF03F017
:10CD20001F0207F8082D94F8031256482668B047EA
:10CD300000215548FFF732FD38460021FFF72EFD50
:10CD400001272F449FE7ABEB0503DBB2042B40F236
:10CD5000D3813778052F40F0CF81D6F80110002617
:10CD60001691C1F3021105298DF84C60236857D83C
:10CD70000A46464894F8F21198479DF85830C3F394
:10CD8000021384F8F2319DF84C3043F004039DF80F
:10CD900058208DF84C3002F00F02062A236847D83D
:10CDA00094F8F3113A4898479DF85830C3F30303B9
:10CDB00084F8F3319DF84C3043F002030DF1590033
:10CDC0008DF84C306426FDF7D8FC46433046FDF71D
:10CDD000D9FF2368804698B33246D4F8F4112D4821
:10CDE00098479DF84C30C4F8F46143F001038DF886
:10CDF0004C30052318A800F8103D0121FFF7CEFCA8
:10CE0000012113A8FFF7CAFC9DF84C10266801F019
:10CE10000103C1F340022048C1F38001B04790E70D
:10CE200007221E4898479DF84C3066F38203AEE710
:10CE300011461B4898479DF84C306FF34103BDE7FE
:10CE40003146184898479DF84C3068F30003CEE708
:10CE50006E3DD512000000006F3DD51200000000AD
:10CE600017D0010838D0010851D001087AD0010844
:10CE7000AAD00108C3D00108F8000020CBD30108D4
:10CE8000F2D0010810D10108FB02002034D10108C2
:10CE90008FD10108DDD1010831D2010863D1010829
:10CEA000BBD101080AD20108ABEB0503DBB2052BAD
:10CEB00040F222813778072F40F01E8156F8010F8B
:10CEC000337916900DF159008DF85C3000F0D6FFE3
:10CED00080469DF85C309DF858101A09009203F0C6
:10CEE0000F03024626688A48B0479DF85C204146F9
:10CEF0009DF8580000F0E0FFC1B2C1F34002236882
:10CF00008DF84C0001F001018248984701F0D4F9F6
:10CF100018A800F8107D0021FFF740FC002113A89D
:10CF2000FFF73CFCE9E6ABEB0503DBB2042B40F278
:10CF3000E38033780A2B40F0DF80D6F801300DF122
:10CF40005900169300238DF84C3000F097FF0646E9
:10CF500002469DF858107048FDF71AFB3046FDF761
:10CF600011FF28B19DF84C3043F001038DF84C308F
:10CF70009DF858300F2B2ED801331B0103F12C02E2
:10CF8000234493F82C10224439B11B6B2BB19DF82C
:10CF90004C3043F002038DF84C309DF84C3018A80B
:10CFA00003F00303032B4FF00A0308BFD66000F819
:10CFB000103D0121FFF7F2FB012113A8FFF7EEFB63
:10CFC0009DF84C105548C1F3400201F00101FDF7F6
:10CFD000DFFA0527B5E60022DFE7ABEB0503DBB29E
:10CFE000012B00F089803778082F40F08580707819
:10CFF00000F00F00FFF760FC012118A800F8087D81
:10D00000FFF7CCFBC4E4AF1C3DE6ABEB0503DBB2A2
:10D01000012B71D037780C2F6ED14FF00109767843
:10D0200023684FEA161809FA08F806F00F06424678
:10D0300094F800123A4809FA06F9984794F8011250
:10D04000384884F8008223684A46984718A884F82C
:10D05000019200F8087D0021D2E7EF1C13E6ABEB4C
:10D060000503DBB2012B47D037780F2F44D1A368DB
:10D070007678984701222C4B8DF85020C3E90001A7
:10D08000330918A80A3302FA03F3002106F00F0649
:10D0900000F8087DC4F82032C4F82462FFF77EFB54
:10D0A000002114A8ACE7ABEB0503DBB2012B23D0C6
:10D0B0003378202B20D176780EB1022E1CD1304649
:10D0C0002768FEF74BFF01461848B84794F8300030
:10D0D000864203D123681648984759E42768FEF72B
:10D0E0003DFF80463046FEF739FF41460246114873
:10D0F000B84784F830604BE4002722E62368ABEBA6
:10D10000050204990C489847C1E53D46FFF7F3BB7B
:10D110006DD2010895D20108C4D20108E3D20108FA
:10D120000CD3010831D301081003002056D30108A5
:10D1300081D30108A4D30108CBD30108F0B585B091
:10D140000391044610B3FFF749FBF8B10020144BDC
:10D150009DF90E1083F8050283F81402207A93F8E3
:10D160001EC09DF80F200609677F257FBCF1000FC8
:10D1700005D010F0010018BF012083F8FC013EB17A
:10D18000009604F10C032046FFF7AAFB05B0F0BDA2
:10D19000002FFBD1002DF9D00095A36EF3E700BF5F
:10D1A000F8000020002310B54168064C1A19106CD5
:10D1B000884202D192F83C0018B91033302BF5D1D7
:10D1C000002010BDF80000202DE9F04F054689B081
:10D1D00018B10378043B012B03D91E215448F6F7FC
:10D1E000F7F92B690BB11B781BB11F215048F6F7DB
:10D1F000EFF9504E50483368984796F8F33196F857
:10D20000F1810393D6F8F43196F8F0B1029396F8D1
:10D21000F2A100F0CFFD00F0D5FD002208AB43F8ED
:10D220000C2D4146454A96F83200FDF7C3FC3446C2
:10D2300040B9434833689847284600F05DFD09B07F
:10D24000BDE8F08F00F024FE059B07469BB101F07E
:10D2500033F800F0EFFC044618B93B213448F6F7E8
:10D26000B7F92B782046637003232370059B636016
:10D2700000F01CFDE3E7AB68327F0133102AAB609E
:10D2800036D1012B09D1D6F8E4310133C6F8E431A7
:10D290002C4B5B699847A6F8DC01B4F8DC3101330C
:10D2A000A4F8DC3100262368B4F8DC11264898473E
:10D2B00007AB94F8F39184F8F361019306AB009304
:10D2C00004EB071141F2707341F288323C31286956
:10D2D000069600F079FAC8B923681C489847284692
:10D2E00000F00AFD069801F061F984F8F391A6E7D1
:10D2F000112A06D1736906F5A6709847A6F8DC01D5
:10D30000D0E74E210A48F6F763F9CBE7069A84F88E
:10D31000F391236812B11278012A1BD00C48984768
:10D32000284600F0E9FC069801F040F987E700BFC5
:10D330004DD50108F80000207ED50108A5D10008D0
:10D340009ED501084CEF0108C3D50108D8D50108C6
:10D35000FDD5010899489847277F102F40F0D680C7
:10D3600023689748984784F84471069BD4F848117D
:10D37000DA6894482368C4F848219847069B002E31
:10D3800000F0D8801122904F84F8442103F1630CFF
:10D3900003F153023E4610685168083203C66245E5
:10D3A0003746F7D1894F03F1230203F1330C3E4690
:10D3B00010685168083203C662453746F7D1844F7A
:10D3C00003F1330203F1430C3E4610685168083202
:10D3D00003C662453746F7D17E4F03F1430253330C
:10D3E0003E4610685168083203C69A423746F7D164
:10D3F000236894F8DB2194F8CC1177489847236888
:10D4000094F8CB2194F8BC1174489847236894F899
:10D41000BB2194F8AC1172489847236894F8AB216B
:10D4200094F89C116F4800269847069BA16B9A6858
:10D430006D48A26323689847069B94F8F3111A7C01
:10D440006A48C2F3030284F8F32123689847069BD5
:10D4500094F8F2111A7C6648C2F3021284F8F221A1
:10D4600023689847069B587CFFF726FAD4F8E41106
:10D47000C4F8EC61C4F8E861C4F8E46123685D486D
:10D48000984723685C48984794F82E30069813F024
:10D49000FD0F00F1120018BF84F82E6084F82F6091
:10D4A00084F8306000F0E2FD23685448984700F0AB
:10D4B00003FF012384F8333000F0BCFB064618B9A3
:10D4C000CA214F48F6F784F88022296906F1200026
:10D4D00009F08FFB0023069A0798C6F8A02094F85D
:10D4E0003320C6F8883032769DF80C203370F27401
:10D4F0002B78029AC6F80A0086F810B086F81180D8
:10D5000086F812A0726173703046B1E6112F0CD10B
:10D51000069B93F8226023680EB13A4822E73A4806
:10D520009847102384F844311FE77C213448F6F7EC
:10D530004FF81AE71022244F84F8442103F1630CBA
:10D5400003F153023E4610685168083203C6624533
:10D550003746F7D11D4F03F1230203F1330C3E464A
:10D5600010685168083203C662453746F7D1184F34
:10D5700003F1230203F1330C3E4610685168083270
:10D5800003C662453746F7D1124F03F12302333306
:10D590003E4610685168083203C69A423746F7D1B2
:10D5A000236894F8DB2194F8CC1118489847236835
:10D5B00094F8CB2194F8BC11154834E722D6010821
:10D5C00049D60108DCD60108C4020020B4020020BC
:10D5D000A4020020940200200AD701084CD70108B9
:10D5E0008ED70108D0D701088ED80108BBD8010812
:10D5F000E9D801081AD901084AD9010873D90108E4
:10D600004DD5010869D6010889D6010812D801084C
:10D6100050D801082DE9F04385B007460C468DF837
:10D620000F202BB101220DF10F01002005F0C2FBEC
:10D63000F4F71CF81D4B1E4D1E4E9DF80F10804632
:10D640009B6A2046984741F288322946D6F8300234
:10D65000F5F74CFC40B32B78012B20D12846AC6861
:10D6600004F0C4FF4FF47A70A4EB080909FB000032
:10D6700008F084FC7968024696F83200FDF74EFB0C
:10D6800000F01AFECDE900499DF80F1035684346B9
:10D690007A680948A847204605B0BDE8F0832846C7
:10D6A00004F0A4FF0024F6E70446F4E74CEF010879
:10D6B00088110020F8000020D1DC01082DE9F84F86
:10D6C000394E9846736B0546894614464FF47A7A6C
:10D6D0009847DFF8DCB0354F0AFB05F202F59C32C3
:10D6E0008032B2FBFAF23249D7F83002F5F7FEFB8E
:10D6F00020B9336B98474FF0FF302FE09BF8003094
:10D70000072B07D1584604F071FF4FF47A6505F0F6
:10D71000E1FAE1E7032B366B22D1DBF804502879DC
:10D720002968844228BF04464846224609F061FA27
:10D730003F6895F90830B5F90620A9881D48B84713
:10D74000B8F1000F05D0EB88A8F800302B7A88F8E4
:10D750000230174804F04AFFB0472046BDE8F88F72
:10D76000042B0BD1124804F041FFB0473C68F3F79B
:10D770007DFF01461048A0470020EFE7052B09D1A7
:10D780000B4804F033FFB0473C68F3F76FFF0146E6
:10D790000A48F0E7F2210A48F5F71AFF044804F0B6
:10D7A00025FFB047A7E700BF4CEF0108F8000020B5
:10D7B000941100207ADB0108A4DB0108BCDB01081E
:10D7C000D2DB0108000000002DE9F04FA44EC9B0E3
:10D7D00002938946924696F84431FF2208A983466F
:10D7E000539F00F0FBFE3546044630B933689D4830
:10D7F0009847002049B0BDE8F08F96F8F01196F8F0
:10D80000F281D9F80420884598BFA1EB08080846A2
:10D8100094BF5FFA88F84FF00008366805920491CB
:10D8200000F076FC039095F8F10100F087FCDDE94B
:10D830000412039B00908C48B047D9F80C20404656
:10D840002E68039200F064FC039A03464146874821
:10D85000B04795F8F311D5F8F42108462E680492E4
:10D86000039100F055FCDDE9031203468048B04700
:10D870002B68029A51467F4898470121584600F08C
:10D880007BFD95F8211095F8F13195F8F021009184
:10D89000D9F80410002008AE01F0D4FA2246002383
:10D8A00031464846FFF7B6FE044610B92B68724869
:10D8B0009EE79BF878306A4D13F0050F11D013F0F6
:10D8C000040F0CBF0020022095F82F30834208D0AF
:10D8D00085F82F00D5F800B0FEF740FB01466748F9
:10D8E000D847FF220021304609F0A7F995F82130EA
:10D8F00042460093D9F80C100823012001F0A2FA47
:10D90000AAF1140007F0D8FE51A3D3E9002307F0D1
:10D910004DFF08F00DFA81460AF2AB2007F0CCFE6D
:10D920004DA3D3E9002307F041FF08F001FA029B61
:10D930008046A3F1140007F0BFFE45A3D3E90023FE
:10D9400007F034FF08F0F4F9A0F1140BC34594BFBD
:10D95000C9EB0B0BC9EB080B4FF47A7808FB09F104
:10D960008246B1FBF8F107A80794F3F797FF3B460F
:10D97000FF2231465846FFF7A1FEB0F1FF3F814636
:10D9800002D12B683E4833E7002829DD2D68F3F7E4
:10D990006DFE2346024649463A48A8470FB1012387
:10D9A000FB700024529BA1451C6017DD2C4D5FFAD3
:10D9B00089F195F84421304601F0B6F9529B324F77
:10D9C00018602B6831489847315D2B683846013420
:10D9D0009847A145F8D12B682D489847012009E7C1
:10D9E00095F8213095F8F3210093D5F8F411082328
:10D9F000012001F027FA08FB0AF107A8B1FBF8F1B2
:10DA00000794F3F74BFF029B03F2AB2007F054FEA1
:10DA100011A3D3E9002307F0C9FE08F089F93B46BA
:10DA2000FF223146A0EB0A00FFF748FEB0F1FF3FAE
:10DA3000814602D12B681748DAE60028B1DD01469D
:10DA40002B6815489847002FABD00223A8E700BFEA
:10DA50000AD7A3703D0AEF3FA4703D0AD7A3F03F59
:10DA6000F800002002DA01081FDA010851DA010883
:10DA700077DA01089DDA0108B8DA0108D7DA010877
:10DA8000FDDA010811DB01087BE0010868DB010811
:10DA9000ACA301083CDB010850DB01082DE9F04193
:10DAA000344EC2B033684FF47A61334802AF9847BE
:10DAB0006B46FF2239464FF47A60FFF7FFFD051EE3
:10DAC000344653DD336829462C48984733682C4840
:10DAD00098470026DFF8C480B95D236840460136C8
:10DAE0009847B542F8D12368264898470023D4F8D0
:10DAF00048210193E9B294F84431384600F0B6FE6B
:10DB0000019038B303782668052B27D0032B27D143
:10DB10001D49427F037F1D48B04723681848984736
:10DB2000019B197F986EFCF799FD2368154898476B
:10DB30000021019800F020FC0198FEF759FDDDE975
:10DB40000010FFF7FBFA0023012201A9D4F83C02E0
:10DB5000F5F772F8284642B0BDE8F0810C49D8E7E5
:10DB60000C48B047019800F021FDF3E733680A48FC
:10DB70009847EFE7F800002009DC010836DC0108CF
:10DB800068DB0108ACA3010806DC01084FDC0108D2
:10DB9000ADA301089ADC0108C0DC01087BE00108A4
:10DBA00038B5074B0546DB6814209847044620B17A
:10DBB0001022002109F041F82561204638BD00BF40
:10DBC000F800002010B5044650B1006900F0EEFCEA
:10DBD00000232361034B2046BDE810401B69184712
:10DBE00010BD00BFF8000020002307B502A941F8CE
:10DBF000040D06481A46D0F83C01F5F71DF8431EFF
:10DC00005842584103B05DF804FB00BFF800002003
:10DC1000002307B50193064B93F8342022B901A9DC
:10DC2000D3F83C01F5F762F9019803B05DF804FB05
:10DC3000F8000020064B10B5DB68A8209847044682
:10DC400018B1A822002108F0F8FF204610BD00BF3F
:10DC5000F800002070B50446104D11482B68984715
:10DC6000DCB1D4F8883033B10E482B68984704F102
:10DC7000200000F085FCD4F8A0304BB12B680A4896
:10DC80009847D4F8A00000F091FC0023C4F8A0301D
:10DC90002B692046BDE87040184770BDF800002091
:10DCA000BBD90108D4D90108EBD901081FB5104C24
:10DCB0000190D4F84001F5F74BFB024640B903A9A7
:10DCC000D4F84001F5F712F910B10398FFF7C2FF3D
:10DCD000002301A91A46D4F84001F4F7ADFF20B99A
:10DCE00040F275110348F5F773FC04B010BD00BF96
:10DCF000F8000020D2DB010838B50546FFF79AFF8F
:10DD0000044620B94FF4BD710548F5F761FC0123C5
:10DD100023702B7820466370BDE83840FFF7C6BFFC
:10DD2000D2DB010810B50D4C031D04EB0313197170
:10DD30009A600123013004EB0010026380F82C305C
:10DD4000114694F83200FDF725F828B9BDE81040D7
:10DD50000B210348F5F73CBC10BD00BFF8000020C4
:10DD60004BDD0108002301460B4870B41A460646F5
:10DD70001D1895F83C401CB12D6C8D4208BF224601
:10DD80001033B3F5807FF3D122B996F8320070BC1E
:10DD9000FDF7AEB870BC7047F8000020044B93F854
:10DDA000222083F8F3215A6AC3F8F421704700BF98
:10DDB000F8000020024B93F8202083F8F1217047EF
:10DDC000F8000020024BDA7F83F8F021704700BF93
:10DDD000F8000020054B93F8202093F8F1119142B0
:10DDE0003ABF012083F8F12100207047F80000209D
:10DDF000064A92F8F031D17F99423DBF03F1FF33DB
:10DE0000012082F8F0310020704700BFF8000020A8
:10DE100010B55024084A21460020FFF783FF214611
:10DE2000064A0120FFF77EFF2146BDE81040044A64
:10DE30000220FFF777BF00BFA027BE33E034C13315
:10DE40002042C43310B50C4CFFF7A8FF94F8320001
:10DE5000FDF77AF8FFF7DCFF5021002204F174038C
:10DE600004F5A274197043F8042C5A6003F8082CC6
:10DE70001033A342F6D110BDF80000204378827819
:10DE80001B02007843EA024303436420584370476F
:10DE9000002330B54168074C04EB0312156CD8B26F
:10DEA0008D4202D192F83C201AB90133102BF3D1E4
:10DEB000002030BDF80000202DE9F8439046C31E35
:10DEC0000C2B05460E46C8F303124FF0000401D98F
:10DED00020460CE069B9204B013503EB0515286B92
:10DEE00085F82C10FFF73EFF4FF003002E63BDE8CE
:10DEF000F883062A2AD9184B08F00F011B68174827
:10DF000098474FF000093046FCF73CFF074600BB3E
:10DF10004FF47A72104BB6FBF2F21B682946104898
:10DF2000984769F3000467F3410404F00303032BEB
:10DF3000CED1094B284603EB05131F6C32464146F0
:10DF4000FFF7F0FE3846FFF70DFFC1E74FF001097C
:10DF5000D9E70127E5E700BFF8000020E2DD01086E
:10DF600002DE0108002110B50C460C4BC20709D592
:10DF700003EB0112146C24B90948FCF709FB204695
:10DF800010BD0124013110294FEA5000EED1002CC0
:10DF9000F5D10448FCF7FCFAF1E700BFF8000020D7
:10DFA00023DE01083FDE010841FA00F000F0010025
:10DFB000704700002DE9F04F274D062991B0074624
:10DFC00090462B6825D14FF6FF71244898474FF6AD
:10DFD000FF7700242646A146DFF87CA0DFF888B052
:10DFE000DAF8401019B147FA04F101F0010105EB2C
:10DFF000041090F844002A6800F00F0CC44502D8C1
:10E00000B8EB101F09D98AF83C9021461448904774
:10E0100013E0014613489847DBE78AF83C100029D3
:10E02000F3D021465846904710ABDAF84000711CF7
:10E0300003EB860646F8400CCEB20134102C0AF1F0
:10E04000100ACDD13246694695F83200FCF7A6FF9A
:10E0500011B0BDE8F08F00BFF80000207EDD0108A0
:10E06000CADD01089DDD0108B3DD010838B50446AD
:10E07000FFF704FF0546FCF785FE28B12A464FF05E
:10E0800050010320FFF74EFEE01CFFF7F7FE0546A8
:10E09000FCF778FE28B12A464FF050010420FFF724
:10E0A00041FEA01DFFF7EAFE0546FCF76BFE28B116
:10E0B0002A464FF050010520FFF734FE04F1090015
:10E0C000FFF7DCFE0546FCF75DFE28B12A464FF05F
:10E0D00050010620FFF726FE04F10C00FFF7CEFEEC
:10E0E0000446FCF74FFE38B12246BDE838404FF0F9
:10E0F00050010720FFF716BE38BD00000738C0B238
:10E1000005289ABF014B185C0E20704704DD0108FA
:10E1100007289ABF014B185C002070470ADD0108F0
:10E12000052804D90628034818BF00207047024874
:10E13000704700BF90D0030048E80100072810B5E1
:10E14000044604D940F277110348F5F741FA034B2E
:10E1500013F9240010BD00BF4BDD010814DD0108D8
:10E16000142810B5044613DD4FF4BE711148F5F7BD
:10E170002FFA062C14DD082C14DD0A2C14DD0C2CCF
:10E1800014DD0E2C14DD152CB4BF0020082010BDAA
:10E19000022803DD0428ECDC0620F8E70720F6E778
:10E1A0000520F4E70420F2E70320F0E70220EEE781
:10E1B0000120ECE74BDD01080F2938B505460C4678
:10E1C00004D940F2A7111348F5F702FA0F2D12D81F
:10E1D000DFE805F00808080B0E0E0E0E11111111E4
:10E1E00011111D1DC4F1330038BDC4F17300FBE7EC
:10E1F000C4F1F200F8E740F2BF110648F5F7E8F97C
:10E20000054B064A4FF4E071024808F0D5FA0020A9
:10E21000EAE700BF4BDD0108D39F010834DD0108A8
:10E220002DE9FF410446002838D000211D4B03EBA7
:10E23000011294422DD1CDB2616879B31A4B93F893
:10E240003200FCF78BFC94F80080DFF868E00646AB
:10E2500016484FF47A72B8F1000F08BF7046217A61
:10E260006768E36801F00F0C0909CDE90110B3FB01
:10E27000F2F3CDF800C0B7FBF2F229460C48FCF7E8
:10E2800087F9237853B1304604B0BDE8F041FCF77C
:10E2900039BC01311029CAD1FF25CDE704B0BDE852
:10E2A000F08100BF34010020F800002094DE010856
:10E2B000A5DE01089CDE010838B50848FCF768F9BE
:10E2C0000024074D28191034FFF7AAFFB4F5807F0A
:10E2D000F8D10448BDE83840FCF75AB969DE0108B6
:10E2E00034010020ACA301080068704782B00346E7
:10E2F00060B16A4659680068013B03C207221DF8F5
:10E30000021012F1FF3203F8011FF8D202B0704779
:10E310000FB404B07047000030B585B06D4685E895
:10E320000F00104C95E80F0084E80F0004F1100274
:10E3300008A903C982E803000BB90B4BE360A3688B
:10E340000BB9094BA36063680BB1236833B9A368A9
:10E3500006489847064B6360064B236001232376EB
:10E3600005B030BDA011002011E30008D9E001087C
:10E37000856B0108756B01082DE9F34105464E4C8C
:10E380004E4A4F48A3680E4600290CBF014611466D
:10E390004C489847A3684C489847696EA3684B4817
:10E3A00098472B784A48072B96BF4A4A4A4952F861
:10E3B0002310A7686A78B847A36848489847A368B5
:10E3C000697F47489847A368297F46489847A368CC
:10E3D000698945489847A368696844489847297AF5
:10E3E0000B090193C1F3C0030093002E32D0C1F397
:10E3F0008003C1F34002A66801F001013C48B04728
:10E400002B7A13F0F00F11D0A3683A486FF00B0786
:10E410009847DFF8F48005F10C067F1B297ABA19BA
:10E42000B2EB111FA36810DB33489847A368334849
:10E4300098472B7F002B3AD1A36831489847A368AF
:10E440002D4802B0BDE8F041184716F8011B4046C0
:10E450009847E3E7C1F38003C1F34002A66801F0E7
:10E4600001012848B0472B7A13F0F00FDED0A368E3
:10E4700020486FF00B079847DFF88C8005F10C06F9
:10E480007F1B297ABA19B2EB111FA368CCDA16F8F0
:10E49000011B40469847F4E7AB6E4046995DB8478C
:10E4A00001362A7FB3B29A42A768F5D8C7E700269B
:10E4B000DFF85880F5E700BFA0110020F0DE01086A
:10E4C000F7DE010800DF01081CDF010832DF010868
:10E4D00043DF0108D0DE010859C1010857DF0108F8
:10E4E00064DF01087ADF010899DF0108B1DF010864
:10E4F000CCDF010811E00108ACA3010863E00108CA
:10E5000072E0010821E001087BE001087AE00108DF
:10E510002DE9F041184D80462B7E0E461BB9D121C6
:10E520001648F5F755F8F22E03D9D2211348F5F71E
:10E530004FF82B6880209847044680B18022002144
:10E5400008F07BFBB8F1000F12D08EB12B6830467B
:10E550009847074630B920466B6898473C462046A6
:10E56000BDE8F0813246414608F043FB2677A766B6
:10E5700000236370F3E700BFA0110020A7E00108AB
:10E5800038B5084D04462A7E1AB9EC210648F5F73D
:10E590001FF834B1A06E20B16B6898470023A366C2
:10E5A000237738BDA0110020A7E0010870B5094C01
:10E5B0000546227E1AB9F7210748F5F709F83DB15B
:10E5C0002846FFF7DDFF63682846BDE8704018471E
:10E5D00070BD00BFA0110020A7E001082DE9F04F99
:10E5E00099469F4B17461A7E93B005460E469846AD
:10E5F00022B94FF485719B48F4F7EAFF032F01D845
:10E600000024D8E02A786B7843EA421333702B78E1
:10E61000022B02D0042B40F08D800023042F8DF8B4
:10E620002630EDD06B6873706B681B0AB370EB8893
:10E63000F370EB7933716B68CDF822309DF826309A
:10E64000002B40F0C180052FDAD006242A7AC2F3CD
:10E65000400302F001019B0143EAC11343EA121394
:10E66000C2F3800243EA4213737195F808A04FEA9F
:10E670001A1A631C9F42C3DD6A89DBB232556A896C
:10E680000234120AF254D8F810301A886B899A4270
:10E6900004D040F269117348F4F79AFFD8F81030AB
:10E6A000B9F1100F1B680A930FD9D8F81420029300
:10E6B0000DF1220301930123297A0093583200239C
:10E6C000090905F10C0000F0D9FFBAF1000F0BD0D9
:10E6D00004EB0A0B5F4593DB3019524605F10C0140
:10E6E00008F087FA5FFA8BF42B7F002B77D0BC42BF
:10E6F00086D26B7F04F1010A33556A7F5FFA8AFA8A
:10E70000D8F81430002A68D158330693AB6E06A9A6
:10E7100007932B7F06EB0A00ADF8203000F0A1FE36
:10E720005044C4B2A7425AD240F297114D48F4F770
:10E730004FFF65E7032B01D0052B01D101236DE7C6
:10E74000002B3CD1082F7FF65BAFD8F81440701C2B
:10E75000224652F8083FC6F8013053684360FFF77D
:10E76000C5FD102F7FF64CAF224652F8103F06F140
:10E770000900C6F8093053684360FFF7B7FD122F50
:10E780007FF63EAFB4F8983006A97374B4F89830A9
:10E7900005A81B0AB37413232834CDE90646ADF847
:10E7A000203000F028FE162F7FF62AAF1724059B95
:10E7B000C6F813306B66204613B0BDE8F08FD8F86A
:10E7C0000C30294898471BE740F25F112548F4F7C1
:10E7D000FFFE4FF0000A05244BE7883395E7E31C62
:10E7E0009F427FF70DAFB9F1100F0FD1D8F8143059
:10E7F00006A9783305A8CDE90636ADF8204000F02B
:10E8000061FD059B33510434E4B2D4E7B9F1110F33
:10E810001FD1D8F814300BA903F1780268330B9399
:10E820000DF122030F930A9B05A81093B5F87A30D7
:10E830000C92ADF8443095F87C300D968DF846304A
:10E8400095F87D30ADF838408DF8473000F072FD16
:10E85000D7E74FF4DD710348F4F7BAFEABE700BF2A
:10E86000A0110020A7E0010880E001082DE9F04F89
:10E87000904D9B462B7EA5B006460F46904623B989
:10E8800040F2C7118C48F4F7A3FE022F29D90021CA
:10E890000846FFF73DFE044630B9EB6887489847C5
:10E8A000204625B0BDE8F08F33785B0903703278DD
:10E8B000072B02F00302427003D1EB6880489847AF
:10E8C0000CE0B8F1000F00F01D82012B40F0F38145
:10E8D000AB687C48F3E742467B4898472046FFF701
:10E8E00065FE0024DCE70AF18801A6E1886873462A
:10E8F000B7E148680023B4E102EB084806EB0900E1
:10E900000593CDF83880FFF7EFFC0AF168020DF1AE
:10E91000900A4AF8682D6066514609A800F0D2FCBA
:10E92000099A616E059B8A420FD0EB686748984749
:10E930000E99ED68DDF83230BDF830206448A84704
:10E9400000212046FFF718FDC8E72A6908F10101F8
:10E95000002B3CD09160227A079304F10C030593BD
:10E9600013091A4606F108010598069308F041F9C3
:10E97000BBF1100F079B0CD90DF132016A690191AF
:10E980000021CDF8088000915832DDE9050100F042
:10E9900075FE237A1B0903F10C02974238D903F163
:10E9A0000D02974215D100234A482377EB68984718
:10E9B000667F002E7FF474AF237A1B093FF470AF9B
:10E9C000237F002B3FF46CAFEB68434877E751603F
:10E9D000C1E70933A9EB0300617FC0B220776A6900
:10E9E00061B958321E440A920B96ADF830002B687C
:10E9F0009847A06620B9EB68384860E78832F1E7AD
:10EA0000514600F02EFD0028D2DCEB68344856E772
:10EA100000232377A366CBE7212F01D1012354E103
:10EA2000EB6830484BE79DF84730043F09EB07009F
:10EA3000DB09FFF759FC6E696066A3B30DF1600A4C
:10EA400000213022504608F0F8F8FF2332468DF8B6
:10EA5000603052F8083F0DF16100CDF86130536825
:10EA60003836CDF86530FFF741FCB6F860303A46ED
:10EA70008DF8693049461B0A0DF16B008DF86A303C
:10EA800008F0B7F8CDE90A6A08F107080AA909A849
:10EA9000ADF8308000F0AFFC636E099A9A4225D041
:10EAA000EB6811480BE72836CDE90A69A8F104089C
:10EAB000ECE700BFA0110020A7E0010806E1010873
:10EAC00011E101083CE101088BE101082AE201089B
:10EAD00069E2010882E20108FDE20108B3E20108EF
:10EAE000D7E2010835E3010892E301089DF83F6091
:10EAF0009DF83E30360446EA03269DF83D300DF180
:10EB000043001E4366609DF842709DF841303F040B
:10EB100047EA03279DF840301F43A760FFF7E4FB57
:10EB2000E0609DF84720237CD10961F3C7131109E8
:10EB300061F3061362F3030323749DF84830637492
:10EB400094F8213003B324AB33F8472D9B786282CD
:10EB5000237524AB33F8442D9B78A4F81520E37576
:10EB600024AB33F8412D9B782283A37624AB33F872
:10EB70003E2D9B78A4F81B20637724AB33F83B2D04
:10EB80009B78E28384F820306D6994F9102005F1B8
:10EB9000280C002AB5F8981004F1230004F153035F
:10EBA000CDF860C018AA12DA05F11807ADF8701098
:10EBB0000092083504F1430204F13301CDE91976DE
:10EBC0001B9500F0E9FC012384F8223068E6ADF8DB
:10EBD0006C101946CDE9196700F09DFC0023F3E79E
:10EBE000EB684D486BE6701CFFF77EFB80450146E5
:10EBF0006060EB687FF46FAE414648489847002359
:10EC0000052F6377A7F1040907D9737903F00F0380
:10EC100008339945C4BFF35C637796F80780B279EF
:10EC2000637F42EA082296F805C0D5F814A06281F5
:10EC3000002B7FF458AE0AF158014FF0010ECDE9D8
:10EC40000A166168BBF1100FCDF83210ADF83090A4
:10EC50008DF836E029697FF64CAE002B7FF446AE86
:10EC60004868217A4FEADC1E6EF300014FEA5C1E11
:10EC70006EF382014FEA1C1E6EF3C3014FEA104887
:10EC80006CF3071180B22172411E8A42BCBF08F1A9
:10EC900001081FFA88F8BBF10F0F7FF62DAE111A8D
:10ECA000B1F5804F7FF728AE0346ED684FF4804101
:10ECB0001B48A84712E6032B95D0052B93D0012BB8
:10ECC0008ED1112F7FF4A8AE002384F821306B6918
:10ECD0001FFA87F828330A93731C0B9308F1FF334C
:10ECE000ADF8303033780AA90DF13D008DF83C3095
:10ECF00000F099FB00280DF13C093FF794AEEB685A
:10ED00000848DCE5032B01D0052BD8D1701CFFF798
:10ED1000EBFA606073E700BFBEE301085EE1010843
:10ED2000C3E1010872E3010813460022FFF79EBD0C
:10ED30002DE9F04F8DB01F46DDF85880394B8346E2
:10ED400098458A460B9246D0374B984504D0374BAE
:10ED500098453BD1002600E00226354D0024EB6AA1
:10ED60009847EB6850469847BBF1010F0A95DFF8CA
:10ED7000D09032D108230A22CDE90132AB693A465C
:10ED8000CDE90644CDE90444039400941D46314680
:10ED90005B460220CDE908BBA8472146FF2003F0CF
:10EDA000A1FCCDF800A0D9F80040334642463946D0
:10EDB0002048A047082003F08BFC342139200A9B0F
:10EDC0001B6C0A930DB0BDE8F04F1847AC211A48F0
:10EDD000F4F7FEFBBEE70126BFE74FF47A634FF07E
:10EDE000010BCDE907430823CDE901B30A9B224675
:10EDF000DB69CDE90544CDE9034B1D460B9933464C
:10EE000000970220A8475946FF2003F06BFC0B9B9C
:10EE1000D9F80040CDE900A34246334639460748B9
:10EE2000A047C7E790D0030020A1070048E80100F1
:10EE30004CEF010867E4010837E401089EE401088B
:10EE4000F80000202DE9F0470446104615460F460D
:10EE500099469DF82060FFF763F980462846FFF742
:10EE600057F9C5B21DB9CB210A48F4F7B1FB7CB9FB
:10EE70004846FFF763F90246B242C8BF72B2CDF806
:10EE800020802B4639462046BDE8F047FFF750BFAB
:10EE90000022F1E737E401080A6803685340036081
:10EEA0004A684368534043608A688368534083607C
:10EEB000CA68C3685340C36070470B6810B51468D4
:10EEC0006340036054684B686340436094688B6898
:10EED00063408360CB68D2685340C36010BD0000BC
:10EEE000A1F11003DBB2102B2DE9F0470C461546BB
:10EEF00008D84FF0010909FA03F303F0013323F0B6
:10EF000080732BB90023FF2085F8F030BDE8F0872F
:10EF10000A460146284607F06CFE04F11C0E4FEA33
:10EF20008E0E5FFA8EFE4FEA1E13013B85F8F0301D
:10EF300023462749B3FBF4F204FB1232E81812F01F
:10EF4000FF0210F804AC10F803CC10F8027C10F8A3
:10EF5000016C32D111F80C804FEAD91289EA080805
:10EF600011F807C08F5D11F80A604FEA420A524457
:10EF7000C24602EBC20282EA49025FFA82F91A1B18
:10EF8000D2B215F802802A448AEA080A05F803A0DA
:10EF900092F8018004338CEA080C80F801C092F8E2
:10EFA00002C0DBB287EA0C078770D2789E4586EAFA
:10EFB0000206C670BED80020A8E7182CDFD9102A98
:10EFC00001BF11F80AA011F80CC0CF5D8E5DD6E725
:10EFD000E0E601082DE9F04F92F8F030A1B01A9167
:10EFE0001892002B00F05D8101461CA8FFF765FF19
:10EFF0004FF00108AC4CAD4DAD4E189B9DF875E03F
:10F0000003EB081319939DF870309DF87AA00093D4
:10F01000009A9DF87F90A05C9DF8742014F80A1067
:10F020000192019F9DF87920E75D02920697029F69
:10F030009DF87E20E75D03920797A25C9DF87870AB
:10F04000049208979DF873209DF87D70059214F83E
:10F05000093014F80EC0A25C09979DF872700A97E7
:10F06000E75D0B979DF877700C97E75D0D97089F0C
:10F07000E75D0E97099FE75D0F979DF87C701097ED
:10F080009DF8717011979DF876701297E75D139750
:10F090009DF87B701497E75D1597109FE75D1697B5
:10F0A000119FE75D1797189F97F8F07047453ED876
:10F0B0008DF870009DF818008DF872108DF87400AE
:10F0C0009DF82C109DF838008DF87A108DF8780096
:10F0D0009DF810109DF858008DF876108DF87C0082
:10F0E0009DF84C109DF81C008DF87E108DF8750071
:10F0F0009DF854109DF83C008DF87F108DF8790034
:10F100009DF834109DF85C008DF87B108DF87D0023
:10F110008DF877201A98199A1CA98DF871C08DF86E
:10F120007330FFF7CAFE002021B0BDE8F08F81EAFE
:10F1300003071B97009F434015F807B01B9F80EA09
:10F140000C008BEA070716F80EB081EA0C0187EA7B
:10F150000B078DF8707015F80E707B4016F80A706A
:10F160007B408DF8713015F80A30584016F8093098
:10F170005840009B8DF8720016F803C0049B8CEA7F
:10F18000010115F809C0534081EA0C018DF8731094
:10F1900001991CA8695C4B400299715C4B408DF849
:10F1A0007430069B5A40029BEB5C5A40039BF35C15
:10F1B0005A408DF87520DDE906325340039AAA5C67
:10F1C0005340059AB25C53408DF87630079A049B01
:10F1D0005340019AB25C5340059AAA5C53408DF8A3
:10F1E00077300D9A0B9B5340089AAA5C5340099ABA
:10F1F000B25C53408DF87830DDE90D325340099A06
:10F20000AA5C53400A9AB25C53408DF87930DDE92C
:10F210000E3253400A9AAA5C53400C9AB25C534097
:10F220008DF87A300B9B0F9A5340089AB25C53408A
:10F230000C9AAA5C53408DF87B30159A139B53406F
:10F24000109AAA5C5340119AB25C53408DF87C30FE
:10F25000DDE915325340119AAA5C5340129AB25C10
:10F2600053408DF87D30DDE916325340129AAA5C86
:10F270005340149AB25C53408DF87E30179A139B1A
:10F280005340109AB25C5340149AAA5C19995340A7
:10F290008DF87F30FFF700FE08F101035FFA83F875
:10F2A000ABE6FF2040E700BFE0E60108E0E401082C
:10F2B000E0E501080B0A017043700B0C090E837026
:10F2C000C170704770B51025CEB00C462A46064670
:10F2D0000021684607F0B1FC49238DF80030A37B7C
:10F2E000D4F80A100DF106008DF80530FFF7E2FFA3
:10F2F00021690DF10A00FFF7DDFF238908A88DF8C9
:10F300000F3000F0FFF9216808A800F00BFA2A4638
:10F31000694608A800F00CFA2289616808A800F084
:10F3200007FA08A90DEB050000F06DFA049B3360A5
:10F330004EB070BD492370B500250C460646CEB0D0
:10F340008DF800300B8BCDE901558DF801301B0A8B
:10F350008DF802308B7E03958DF80330CB7E0DF156
:10F3600006008DF804300B691968FFF7A3FF616987
:10F370000DF10A00FFF79EFFA38908A88DF80F3052
:10F380008DF80E5000F0BEF9216808A800F0CAF907
:10F39000694608A8102200F0CBF9A289A16808A844
:10F3A00000F0C6F908A904A800F02DFABDF8103045
:10F3B00008A833808DF804508DF803508DF8025062
:10F3C0008DF8015000F09EF9616808A800F0AAF9D4
:10F3D000694608A8102200F0ABF9A289A16808A824
:10F3E00000F0A6F908A904A800F00DFABDF8103045
:10F3F00073804EB070BD30B50C46CBB0054604A846
:10F4000000F080F9216804A800F08CF92289616875
:10F4100004A800F08DF904A9684600F0F4F9009BF7
:10F420002B604BB030BD70B50C89BEB006460D46A2
:10F43000A4B114F00F0411D101AA10212868FFF71C
:10F440004FFD2889A04201DC3EB070BD68683119CB
:10F45000204401AAFFF7BEFD1034F2E74FF0FF3061
:10F46000F2E72DE9F0430F89C7B081460D46002F22
:10F470004ED0012410224FEA1718002117F00F0771
:10F4800001A818BF08F1010807F0D7FBAB7BD5F83E
:10F490000A100DF10A008DF809308DF80440FFF7CD
:10F4A00009FF29690DF10E00FFF704FF6E68013EA8
:10F4B000444503DD288947B0BDE8F08309AA10213F
:10F4C00028688DF81340FFF70BFD09AA05A901A8CC
:10F4D000FFF780FD444510DB002F14BF3B4610238F
:10F4E00030464A464B440DF1130C934207D8013481
:10F4F000A4B209F110091036DAE71023F0E710F88A
:10F5000001EF1CF8011F81EA0E0102F8011BECE774
:10F510004FF0FF30CFE770B5C2B0144606460D4637
:10F52000F122002105A807F088FB0023CDE9033371
:10F53000636810218DF805301A0A1B0C8DF807300E
:10F54000A3688DF806208DF808301A0A1B0C8DF878
:10F550000A30A3898DF809208DF80B301B0A8DF82D
:10F560000C30012305AA20688DF80430FFF7B8FCA1
:10F5700005AA314601A8FFF72DFD022305AA102197
:10F5800020688DF80430FFF7ABFC05AA294601A8D6
:10F59000FFF720FD42B070BD2DE9F0431025C3B048
:10F5A0004A9C80460F4616460021F12205A899463E
:10F5B00007F043FB2A46002101A807F03EFBA268A2
:10F5C00029468DF80520130AEA408DF80720E268E5
:10F5D0008DF80630D37920688DF8083093798DF84E
:10F5E000093053798DF80A3013798DF80B30D378C0
:10F5F0008DF80C3093788DF80D3053788DF80E30EF
:10F60000137805AA8DF80F30238A8DF810301B0A65
:10F610008DF8113001238DF80430FFF761FC05AA45
:10F62000414601A8FFF7D6FC022305AA29466068D7
:10F630008DF80430FFF754FC05AA494601A8FFF7EE
:10F64000C9FC032305AA294620688DF80430FFF77A
:10F6500047FC05AA394601A8FFF7BCFC042305AA0C
:10F66000294620688DF80430FFF73AFC05AA314698
:10F6700001A8FFF7AFFC43B0BDE8F083F0B50F2958
:10F68000C7B004460D4616461F4604D94FF4A17173
:10F690001B48F3F79DFF0123002F019318BF02239E
:10F6A0008DF808309DF830310DF10A0083F0010328
:10F6B0008DF809304D9B1968FFF7FCFD4E990DF14F
:10F6C0000E00FFF7F7FD4FF4807309AA10213046B2
:10F6D00005AEADF81230FFF703FC09AA314601A8C8
:10F6E000FFF778FC0023601EDAB2954201D847B0DC
:10F6F000F0BD10F8012FF15C01334A400270F3E7CE
:10F70000E0E7010810B5102204460021F13007F0AF
:10F7100094FA00212046C4F81411F022BDE81040EC
:10F7200007F08BBA0B46024610211846FFF7D8BBEC
:10F730002DE9FF470446D0F814010E46154604F2A1
:10F74000011920B3C0F110089045474628BF17465D
:10F7500048443A4607F04DFAD4F814313B440F2B95
:10F76000C4F814311ED9A8451CD204F1F10319467E
:10F7700013F8012BD87B4B4582EA000203F8012CD9
:10F78000F6D122460846FFF725FC3E44ED1B0DF15D
:10F79000100A102D09D82A463146484607F029FAA2
:10F7A000C4F8145104B0BDE8F08704F1F002731EF0
:10F7B00006F10F0013F8017F12F8011F834281EA5E
:10F7C00007011170F6D16A4604F1F1039846174615
:10F7D0009446186859680833ACE803004B45624604
:10F7E000F6D1224639463846FFF7F4FB43463A46FF
:10F7F00003CA524518605960174603F10803F6D151
:10F800001036103DC5E7F0B50C4689B01022002136
:10F810000546684607F011FA224669466846FFF732
:10F82000D9FB9DF900306A46002B0DF10F0140DA3B
:10F83000137812F8010F5B005BB243EAD0139142D8
:10F8400002F8013CF4D19DF80F305B0083F0870390
:10F850008DF80F30D4F81431102B39D1002304F275
:10F86000011211781DF8030001334140102B02F8FA
:10F87000011BF6D104F1F102134604F2011712F84C
:10F88000011BD07B974281EA000102F8011CF6D1EE
:10F8900004AA9446164618685968083303C6BB4242
:10F8A0003246F7D1224629466046FFF793FB09B05E
:10F8B000F0BD137812F8010F5B005BB243EAD0137E
:10F8C0008A4202F8013CF4D19DF80F305B00BFE79B
:10F8D0009DF900206846002A28DA027810F8016FA6
:10F8E000520052B242EAD612814200F8012CF4D101
:10F8F0009DF80F20520082F0870280218DF80F20A2
:10F90000E21882F80111002201330F2B1DD9C4F82F
:10F910001431002304F2011211781DF803000133A1
:10F920004140102B02F8011BF6D1A3E7027810F832
:10F93000016F520052B242EAD612814200F8012C05
:10F94000F4D19DF80F205200D7E7E11881F801218A
:10F95000DAE70000002103E00A4B5B584350043112
:10F9600009480A4B42189A42F6D3094A02E000239A
:10F9700042F8043B074B9A42F9D300F00DF8F1F737
:10F9800021FA7047C4F5010800000020BC050020E2
:10F99000C0050020E0180020314B82B01A6842F404
:10F9A00080721A6099682F4A0A409A601A6822F099
:10F9B000885222F001121A601A6822F480221A601A
:10F9C0009A6822F47D029A600022DA6001921B6834
:10F9D00013F4007318BF01230193019B012B37D14E
:10F9E0004FF48051204B1A68A3F5806322F0010286
:10F9F000C3F80024D3F8002422F00202C3F8002444
:10FA0000D3F8002422F00402C3F800245A6A42F01A
:10FA100080525A62154A11605168C906FCD49A682E
:10FA20009A609A689A609A689A605A6822F460426A
:10FA30005A605A6842F440425A609A6822F00302BF
:10FA40009A609A689A60064A936813F00C0FFBD18B
:10FA50004FF00062064B9A60064ADA6002B07047C7
:10FA6000003802400CC0FF88003C0240007000409B
:10FA700000ED00E00003FA0570B5064688B02E4898
:10FA800001F076FB2D4B1A680092009A91073CD545
:10FA900001214FF4007001F0C5FD012001F0B8FB19
:10FAA000274A536843F400335360A2F53742536842
:10FAB0001B07FCD50024012502A801F093FB02A935
:10FAC0001D488DF80D4006948DF81C508DF80C40A3
:10FAD00001F062FB2A4606233146174801F0A4FBD9
:10FAE0002946154801F08AFB0221134801F02EFC3B
:10FAF000114801F01DFC134D01940F4C02212046CA
:10FB000001F01EFC58B108B070BD1A6842F0010245
:10FB10001A60009A9207BBD41A680092F9E7019B19
:10FB200001330193019BB3F5805FE7DB3821284661
:10FB3000F3F74EFDE2E700BF002401400038024029
:10FB40000027014018E8010808B5002001F060FB1B
:10FB50000021074801F052FB00214FF4007001F032
:10FB600061FD044A136823F00103136008BD00BF60
:10FB7000002401400038024013B50723012201464A
:10FB8000114801F051FB02210F4801F0DFFB0E4844
:10FB900001F0CEFB00230D4C019302210A4801F035
:10FBA000CFFB28B1084802B0BDE8104001F0C5BB4A
:10FBB000019B01330193019BB3F5805FEDDB4C2189
:10FBC0002046F3F705FDE8E70024014018E80108A6
:10FBD00070B506460825FFF74FFF00243046FFF7B3
:10FBE000CBFF013D0444F9D1FFF7AEFFC4F3CF00D2
:10FBF00070BD00000000000008B51120FFF7E8FF0D
:10FC000006F0BCF90146084806F0C4FA05F076FD96
:10FC100003A3D3E9002305F0C9FD06F0A9F808BD48
:10FC20002FDD24068195F33F00F07F450F4A536A8C
:10FC300043F0805353620E4B1A465968C906FCD4F0
:10FC40001B68022823F4C05306D143F4C053136049
:10FC50005368DB06FCD47047012802D143F480537B
:10FC6000F5E70028F3D143F40063F0E700380240E1
:10FC70000070004010B50C4B5A68D206FCD41C68CA
:10FC800014F4C05F0BD114F480500AD114F4006452
:10FC900004D106482A21F3F79BFC204610BD022020
:10FCA000FCE70120FAE700BF0070004054E80108BB
:10FCB00038B50546012001F059FB022D01BF154A58
:10FCC000136843F001031360134B1A6842F4803247
:10FCD0001A601A689203FCD542F690529A609968AD
:10FCE0009142FCD19A6842F002029A600A4B9C68E9
:10FCF00014F00804FBD14FF480321A60074B084A15
:10FD000028461A60FFF792FF2046BDE8384001F010
:10FD100021BB00BF003C02400038024038030020F5
:10FD200000093D0038B50546012001F01FFB022DFA
:10FD300001BF144A136843F001031360124B1A68A1
:10FD400042F480721A601A689205FCD55A6822F44F
:10FD5000604242F440425A6000229A600A4B9C681A
:10FD600014F00C04FBD14FF480721A60074B084A60
:10FD700028461A60FFF75AFF2046BDE8384001F0D8
:10FD8000E9BA00BF003C02400038024038030020BE
:10FD9000D0FE3F000C4B5A6B900513D45A6A42F0C8
:10FDA00080525A62094A116841F480711160596B9E
:10FDB00041F480715963596B8905FCD5136823F4AC
:10FDC00080731360704700BF00380240007000402D
:10FDD000054B5A6B910706D45A6B42F001025A63E5
:10FDE0005A6B9207FCD5704700380240094B5A6A9B
:10FDF00042F020025A629A6942F020029A619A699E
:10FE000022F020029A610022A3F509331A801A8594
:10FE10005A627047003802401521023800224843D8
:10FE20000121064B1A85D86299825A621A8219807A
:10FE30001A8AD207FCD500221A80704700140040AD
:10FE4000002349F6FE7282B00193019B934201DDCB
:10FE500002B07047019B01330193F6E7002340F69F
:10FE6000FE7282B00193019B934201DD02B07047A4
:10FE7000019B01330193F6E7002382B00193019BBC
:10FE8000B3F5CC7F01DD02B07047019B0133F5E78C
:10FE9000D0B1012801D1FFF7EFBF0C4B00211A6848
:10FEA0004FF47A73B2FBF3F2094B013A92B21A851E
:10FEB00001220138D8629A82596219821A801A8AFC
:10FEC000D207FCD500221A80704700BF38030020FB
:10FED0000014004000F1774303F57803B3F5804F39
:10FEE0002DE9F04106460C4617462DD202F1F733B4
:10FEF00003F608030344B3F5804F25D2FFF7BAFE9B
:10FF0000804610B10020FFF791FE01F047FA01256D
:10FF10002744361BA7420AD101F050FAB8F1000F6E
:10FF200002D04046FFF782FE2846BDE8F08141F648
:10FF3000027001F04BFA301914F8011B01F0A2FA1B
:10FF4000042818BF0025E5E70025EDE710B50C46AD
:10FF500000F1774101F57801B1F5804F0DD202F142
:10FF6000F73303F608030344B3F5804F05D2014687
:10FF7000204606F03EFE012010BD0020FCE70000F8
:10FF800008B5114B984215D003F58063984213D001
:10FF900003F58063984211D003F5806398420FD037
:10FFA00003F5006398420DD0084B094A1421094813
:10FFB00006F002FC002008BD0120FCE70220FAE761
:10FFC0000320F8E70520F6E700000240D9E8010821
:10FFD00093E80108F2E801080F2808B505D9094B94
:10FFE000094A3B21094806F0E7FB012303FA00F028
:10FFF000C043074A516801405160136818401060BF
:020000040801F1
:1000000008BD00BF31E901089DE80108F2E80108D8
:10001000000401400F292DE9F84F82460D46934612
:100020001F4605D95A4B5B4A54215B4806F0C4FB76
:100030004FF0010909FA05F900F0B8F86FEA090371
:10004000564E032D7268564C02EA03027260326803
:1000500003EA0203534A3360136A43F00103136255
:100060002ED80F22A3684FEA850802FA08F223EA85
:100070000203A3605046FFF783FFA36800FA08F06D
:100080001843A0601BF0020F18BFB368464A1CBF9C
:1000900043EA0903B3601BF0040F1EBFF36843EA91
:1000A0000903F360336843EA090333603B01DBB2C1
:1000B000002D45D182F8063340231360BDE8F88F48
:1000C000072D13D80F22A5F10408E3684FEA88082A
:1000D00002FA08F223EA0203E3605046FFF750FFFA
:1000E000E36800FA08F01843E060CBE70B2D13D863
:1000F0000F22A5F1080823694FEA880802FA08F2DE
:1001000023EA020323615046FFF73AFF236900FA0E
:1001100008F018432061B5E70F22A5F10C086369C8
:100120004FEA880802FA08F223EA020363615046A4
:10013000FFF726FF636900FA08F018436061A1E742
:10014000012D03D182F807338023B6E7022D04D1B5
:1001500082F808334FF48073AFE7032D04D182F89F
:1001600009334FF40073A8E7042D04D182F80A3351
:100170004FF48063A1E7092D04D882F817334FF4B8
:1001800000039AE782F828334FF48073536095E7B1
:100190003DE90108B8E80108F2E80108000401405F
:1001A000000001400038024000E100E0144B98429A
:1001B00005D1144AD36943F00103D3617047124B50
:1001C000984204D10F4AD36943F00203F5E70F4B7D
:1001D000984204D10B4AD36943F00403EDE70C4B7A
:1001E000984204D1074AD36943F00803E5E7094B75
:1001F0009842E3D1034AD36943F02003DDE700BF0F
:1002000000000240003802400004024000080240A2
:10021000000C0240001402400323490010B584681A
:100220008B4024EA030484600124022A04FA01F4C6
:1002300007D0032A0DD0012A07D1836823438360A6
:1002400003E083688A401A43826083681C438460A9
:1002500010BD82681343F2E70F29F8B504460F4634
:1002600015461E4603D94B211948F3F7B1F920462C
:10027000FFF79CFF03237A009340DB43216819407A
:1002800021600121D4F800C001FA02F04CEA000C10
:10029000B940C4F800C009B266B1A688314389B23A
:1002A000A180E168012D03EA0103E36006D0022D7D
:1002B00008D0F8BDA68826EA0101F1E7E368034308
:1002C000E360F6E7E36805FA02F21A43E260F0E75A
:1002D0008DE901080F2970B505460C46164603D96D
:1002E0006B210E48F3F774F92846FFF75FFF0323ED
:1002F00061008B40DB43EA68012E02EA0302EA60F8
:1003000005D0022E03D02A6813402B6070BDEA6826
:1003100006FA01F11143E960F5E700BF8DE9010834
:100320000F2910B505D9074B074A8121074806F068
:1003300043FAFFF73BFF4B0003210268994011434A
:10034000016010BD31E9010849E901088DE90108A2
:100350000F2938B50446154605D987211B4B1C4A81
:100360001C4806F029FA0F2A03D91B4B184A88218A
:10037000F6E7FFF71BFF07294FF00F0318D8006AB5
:100380008A00934020EA03032362236A05FA02F2FB
:100390001A4322620322236849008A4023EA0203A7
:1003A00023600223226803FA01F11143216038BD62
:1003B000A1F10802406A9200934020EA03036362BD
:1003C000636A95401D436562E4E700BF31E90108B7
:1003D0005CE901088DE901087AE90108012303FAC3
:1003E00001F189B201837047012303FA01F189B257
:1003F00041837047012303FA01F189B20AB10183F5
:10040000704741837047008A084100F0010070473F
:100410000F2938B505460C4603D9B4210548F3F732
:10042000D7F828686400E04000F00300431E5842FB
:10043000584138BD8DE90108808A084100F001006B
:100440007047000010B5084C23681BB90120F2F773
:1004500097FC206023682BB9BDE810403621034883
:10046000F3F7B6B810BD00BFBC110020CAE90108FF
:1004700010B50B4C22681AB93C210A48F3F7A8F8CA
:10048000206842F21071F2F7C3FD01280CBF01246D
:10049000002403D040210348F3F79AF8204610BD0A
:1004A000BC110020CAE9010810B5074C22681AB92E
:1004B00051210648F3F78CF8002320681A46BDE85E
:1004C00010401946F2F7B8BBBC110020CAE9010878
:1004D00010B50446FFF7B6FFFFF7CAFF214610220A
:1004E000034801F09FFD0446FFF7DEFF204610BDE4
:1004F0000054004010B5FFF7A5FFFFF7B9FF01F06A
:1005000049FD0446FFF7D0FF204610BD08B513464D
:100510000A460146034801F07DF9003018BF01206A
:1005200008BD00BF0054004008B513460A46014606
:10053000034801F06FFA003018BF012008BD00BF6A
:100540000054004008B513460A460146034801F02E
:100550003DFB003018BF012008BD00BF0054004023
:1005600008B513460A460146034801F0BFFB0030B8
:1005700018BF012008BD00BF0054004008B5134655
:100580000A460146034801F009FC003018BF01206B
:1005900008BD00BF005400400123064A8340516952
:1005A000194205D05361044B53F8203003B118476A
:1005B000704700BF00040140C01100200F2838B56B
:1005C00004460D4603D926210348F3F701F8034BEF
:1005D00043F8245038BD00BF06EA0108C0110020CE
:1005E0000020FFF7D9BF0120FFF7D6BF0220FFF799
:1005F000D3BF0320FFF7D0BF0420FFF7CDBF08B55E
:100600000920FFF7C9FF0820FFF7C6FF0720FFF703
:10061000C3FF0620FFF7C0FFBDE808400520FFF735
:10062000BBBF08B50F20FFF7B7FF0E20FFF7B4FFE1
:100630000D20FFF7B1FF0C20FFF7AEFF0B20FFF7F7
:10064000ABFFBDE808400A20FFF7A6BFFEE7FEE7C4
:10065000FEE7FEE7FEE7FEE7FEE7FEE7FEE7FEE772
:10066000FEE7FEE7FEE7FEE7FEE7FEE7FEE7FEE762
:10067000FEE7FEE7FEE7FEE7FEE7FEE7FEE7FEE752
:10068000FEE7FEE7FEE7FEE7FEE7FEE7FEE7FEE742
:10069000FEE7FEE7FEE7FEE7FEE7FEE70A23B0FB24
:1006A000F3F203FB120040EA0210C0B270470000F0
:1006B000CA22024B5A6253225A62704700280040F5
:1006C000014B1860704700BF001200204FF4003249
:1006D0000F4B10B50F4C5A61E368DB0503D4302192
:1006E0000D48F2F775FFFFF7E3FF4FF40072A368C0
:1006F00023F48853A360094BC3F88420FF2363626B
:10070000074B1B6813B1BDE81040184710BD00BF70
:10071000000401400028004042EA010800E100E036
:10072000001200202DE9F04F9846374B85B01B781A
:10073000824691469DF838709DF83C602BB9334B4A
:10074000334A8C21334806F037F8431E1E2B59D804
:100750000C2957D8A2F5FA63632B53D8B8F1170FB9
:1007600050D83B2F4ED83B2E4CD802F13000C0B2AF
:10077000FFF794FF83460846FFF790FF0446504674
:10078000FFF78CFF40F400554046FFF787FF45EA2E
:100790000B4545EA042504463846FFF77FFF000273
:1007A00040EA04443046FFF779FF20431A4CFFF734
:1007B0007FFFE36843F08003E360E3685B06FCD5FA
:1007C00065602060E36823F08003E360124BDA6821
:1007D0009206FCD5FF2204A85A6200F80C6D8DF831
:1007E00007A08DF80810ADF809908DF806808DF8F7
:1007F0000570F9F7F8FD094BC3E90001012005B0C8
:10080000BDE8F08F0020FAE704120020B1EA0108E9
:10081000A5EA010842EA0108002800400812002069
:1008200037B50578C4788378B0F80520017901954B
:10083000407800902046FFF775FF03B030BD000000
:1008400038B52B4B04461B781BB9E4212948F2F735
:10085000BFFE294AD36823F02003D360D3689B06E8
:10086000FCD513685268C2F30741080900EB800009
:1008700001F00F0101EB4001C9B201F5FA61A4F8E2
:100880000510C2F30721C1F300108500284401F0D0
:100890000F0101EB4001D2B22171C2F3011101EB52
:1008A000810102F00F0202EB4102E270C3F3074242
:1008B000C2F3011101EB810102F00F0202EB4102D0
:1008C000A270C3F30722C2F3021101EB810102F00F
:1008D0000F0202EB4102DBB26270C3F3021202EBC1
:1008E000820203F00F0303EB4203237038BD00BF05
:1008F0000412002042EA0108002800401FB501A8A8
:10090000FFF79EFF01A8F9F76EFD05B05DF804FB47
:1009100008B5FFF73FFA1B4A136843F4807313606E
:10092000FFF7C6FE184A536B23F4403343F48203A7
:100930005363164BDA6842F08002DA60DA685106D7
:10094000FCD5FF221A611A6942F4FE021A619A6804
:1009500022F040029A609A6822F44C529A60DA6857
:1009600022F08002DA60094BDA689206FCD5FF2299
:100970005A620122064B1A70FFF7C0FF054BC3E90C
:10098000000108BD0070004000380240002800400F
:10099000041200200812002008B5094B1B7823B967
:1009A00040F21F110748F2F713FEFFF781FE064BD6
:1009B0009A6822F480729A60FF225A6208BD00BFD2
:1009C0000412002042EA01080028004008B5144B38
:1009D0001B7833B9134B144A40F22711134805F022
:1009E000EBFEFFF765FE124BDA6822F48072DA60E4
:1009F000104A916841F400319160116841F400316E
:100A00001160F0210C4A82F829134FF400715160F3
:100A10009A6842F488529A60FF225A6208BD00BF69
:100A200004120020B1EA01087EEA010842EA010846
:100A3000002800400004014000E100E0F8B51E4637
:100A4000194B17461B7833B9184B194A4FF4A57147
:100A5000184805F0B1FE184CFFF72AFEA56825F4EA
:100A60008075A560E56825F48075E560FFF716FEE2
:100A700005460846FFF712FE000440EA05613846C5
:100A8000FFF70CFE05463046FFF708FE084340EA34
:100A90000520E368DB07FCD5FF23E0616362BDE866
:100AA000F840FFF793BF00BF04120020B1EA01082D
:100AB00093EA010842EA01080028004003784278DE
:100AC0008178C078FFF7BABF38B50D460446F1F714
:100AD00071FE1F4A136823F001031360F1F78AFEC9
:100AE00025B11C4A536843F00603536072B6BFF346
:100AF0004F8FBFF36F8F184A0120136823F0030351
:100B000043F4007343F00103136000F03BFC134B0C
:100B10001A6942F004021A6130BF1A6922F0040215
:100B20001A610F4B0F4A1B6893420AD10220FFF74C
:100B3000F9F8074A136843F00103136004B162B681
:100B400038BD094A9342F4D10220FFF7B1F8F0E72B
:100B500010E000E0002004E00070004000ED00E044
:100B600038030020D0FE3F0000093D0062B6704708
:100B700000220E4B10B51A700D4A0E4C13882046F9
:100B800023F040031B041B0C13800D210222FFF7EE
:100B9000A1FB204602220E21FFF79CFB2046BDE868
:100BA000104002220F21FFF795BB00BF101200205A
:100BB0000038004000040240284A38B5136A054650
:100BC00043F480531362052225480C461146FFF773
:100BD000BFFB052206212248FFF7BAFB05220721A9
:100BE0001F48FFF7B5FBC5B1022205211C48FFF7DE
:100BF00013FB022206211A48FFF70EFB02220721EF
:100C00001748FFF709FB012C21D144F4517401224C
:100C1000144B1C80144B1A7038BD2A46052110480D
:100C2000FFF7FAFA2A4606210D48FFF7F5FA2A4699
:100C300007210B48FFF7F0FA012C05D0022C03D056
:100C4000032C14BF0024032444F45974DFE7022C5E
:100C5000DBD0032C0CBF03240024D6E7003802406D
:100C600000000240003001401112002000220E4B13
:100C700010B51A700D4A0E4C1388204623F040031D
:100C80001B041B0C138005210222FFF723FB2046C7
:100C900002220621FFF71EFB2046BDE8104002227B
:100CA0000721FFF717BB00BF1112002000300140E1
:100CB00000000240064B074A988111781A461889AD
:100CC000C00701D40029FAD19089C0B2704700BF93
:100CD0000030014011120020054AD36823F4E0637C
:100CE0001B041B0C43F0BF6343F40033D360704715
:100CF00000ED00E020220021114B10B5C3F8842044
:100D0000104B114C1A6A204642F480421A625A690A
:100D100042F480425A615A6922F480425A610B4A75
:100D200091811A6A092122F480421A620222FFF795
:100D3000D1FA2046BDE8104002220A21FFF7CABAC4
:100D400000E100E0003802400000024000380140AD
:100D500010B50B4C40F22551204600F034FD48B14F
:100D6000204600F00EFD074BC0B21B6833B1BDE852
:100D700010401847A388044ADBB2137010BD00BFAF
:100D800000380140141200204018002010B504461D
:100D90008021084800F011FD0028F9D021460548BF
:100DA00000F0EBFC034C4021204600F006FD00283B
:100DB000F9D010BD0038014010B5441E14F8010FE1
:100DC00000B910BDFFF7E2FFF8E7000008B50248E0
:100DD00000F0D7FCC0B208BD003801402DE9F04357
:100DE0008846012189B08146084614461D4600F018
:100DF0000DFC01214FF4804000F014FC4FF4C0675B
:100E000002230122002602A93F488DF80C308DF8FC
:100E10000D308DF80F2002978DF80E6000F058FB12
:100E200007220921384800F095FB07220A2136489D
:100E300000F090FBB8F1450FCDF810903CD14FF485
:100E40008063ADF81830072C42D10023ADF8143080
:100E5000052D4ED14FF48053ADF816300023ADF878
:100E60001C300C2304A92948ADF81A3000F02AFCE4
:100E7000274B1A6802B1012240F22551234800F0A5
:100E800084FC0121214800F06DFCFFF79FFF252322
:100E90008DF804309DF840308DF8053000238DF832
:100EA000063001238DF80730FFF716FF01A800F088
:100EB00043F909B0BDE8F083B8F14F0F02D1ADF8A6
:100EC0001870C0E7072CADF818600DD1592107E064
:100ED000082C02D14FF48053B8E7092CB8D1542123
:100EE0000C48F2F775FBB3E7082CAED0092CAFD154
:100EF000F0E70F2D02D14FF44053ADE7022D0CBFA8
:100F00004FF400530023A7E70000024000380140DF
:100F100014120020BAEA01080E2307B50822009334
:100F20004E210123FFF75AFF03B05DF804FB0000D8
:100F300070B5134C40F22551204600F044FCC0B17E
:100F4000104B1D6825B1204600F01BFCC0B2A8471D
:100F500040F226610A4800F036FC78B140F2266182
:100F6000074800F04FFC084B1B683BB1BDE87040E0
:100F70001847A388054ADBB21370E9E770BD00BFCC
:100F800000440040181200201C12002040180020CD
:100F9000BFF34F8F0449054BCA6802F4E062134364
:100FA000CB60BFF34F8FFEE700ED00E00400FA05D1
:100FB00010B5441EE3B2052B03D917211148F2F7EF
:100FC00007FBFEF705FF45F255520F4B1A60DA6832
:100FD000D207FCD4052C06D8DFE804F003090B0D7A
:100FE0000F1101225A604CF6CC421A6010BD022249
:100FF000F8E70322F6E70422F4E70522F2E70622E7
:10100000F0E700BF79EB01080030004038B5224C12
:10101000236853B95F2000F01DFB204D38B1204BF1
:10102000236001232B7000F025FB206838BD5E2073
:1010300000F010FB18B11B4B23600223F2E75D2088
:1010400000F008FB18B1184B23600323EAE75C208B
:1010500000F000FB18B1154B23600423E2E75B208E
:1010600000F0F8FA18B1124B23600523DAE75A2092
:1010700000F0F0FA18B10F4B23600623D2E7592095
:1010800000F0E8FA18B10C4B23600723CAE70B4BBA
:101090002360FF23C6E700BF24120020281200208F
:1010A000F7EA010807EB01081DEB010838EB01081E
:1010B00047EB010856EB01086FEB010859C1010825
:1010C00008B5FFF7A3FF014B187808BD28120020D0
:1010D00038B5084B084D1A7852B9012420461C70C7
:1010E00000F0E0FA287020F0FF01204600F0CAFA74
:1010F000287838BD201200202112002010B50446A7
:10110000012000F0CFFA20F0FF0121430120BDE8CB
:10111000104000F0B7BA08B5FFF7F0FFFFF738FF4F
:1011200008B5012000F0BEFA10F0FF0F02D1012037
:10113000FFF7F1FFFFF72CFF30B5012403780A4DCC
:1011400003F01F029440C278590952B1074A2B4458
:10115000D26842781201D2B283F8002345F82140C8
:1011600030BD2031FAE700BF00E100E000ED00E013
:1011700008B5084B98420BD101214FF4007000F0E4
:101180005DFABDE8084000214FF4007000F056BA47
:1011900008BD00BF0024014043680A7923F0407372
:1011A00023F4807343EA02230A6810B513434360B3
:1011B000D1E9032313438A6884681343084A224011
:1011C00013434A7943EA420383600A7D036B013A81
:1011D00023F0F873D2B243EA0253036310BD00BF99
:1011E000FDF7FFC000234FF04072036003714371AD
:1011F0008360C0E90323012303757047836819B135
:1012000043F001038360704723F00103FAE7000015
:10121000044B5A6818B142F400025A60704722F435
:101220000002FAE7002701401D2970B51BD90725E8
:10123000A1F11E06C46D06EB4606B54024EA05047E
:1012400003FA06F62643C665062A38D81F24013A53
:10125000036C02EB8202944023EA040301FA02F2D7
:101260001A43026470BD13290DD90726A1F1140594
:10127000C46805EB4505AE4024EA060403FA05F50B
:101280002543C560E0E709290DD90726A1F10A0425
:10129000056904EB4404A64025EA060503FA04F4B4
:1012A0002C430461D0E70726446901EB4105AE40B9
:1012B00024EA060403FA05F626434661C4E70C2A2D
:1012C0000CD81F24073AC36B02EB8202944023EA36
:1012D000040301FA02F21A43C263C3E7122A0CD8CC
:1012E0001F240D3A836B02EB8202944023EA04032D
:1012F00001FA02F21A438263B4E7182A0CD81F24B9
:10130000133A436B02EB8202944023EA040301FA8E
:1013100002F21A434263A5E71F24193A036B02EB5A
:101320008202944023EA040391401943016399E740
:10133000836843F0804383607047806D80B270475C
:101340000368194214BF012000207047C94301609F
:1013500070470000044B1A6818B142F002021A608C
:10136000704722F00202FAE7003C0240044B1A6880
:1013700018B142F004021A60704722F00402FAE742
:10138000003C0240044B1A6818B142F008021A608F
:10139000704722F00802FAE7003C0240044B5A680A
:1013A000D20741BF034ADA60034ADA60704700BFE0
:1013B000003C0240EFCDAB8905040302024A5368AA
:1013C00043F0010353607047003C0240014B9861B9
:1013D000704700BF003C0240084B9A69D10709D40E
:1013E0009A69D20508D49B6913F4F05F14BF0320F7
:1013F000042070470120704702207047003C0240E3
:10140000042313B504468DF80730FFF7E5FF8DF888
:1014100007009DF80730012B0AD11CB905238DF870
:10142000073007E0FFF7D8FF013C8DF80700F0E731
:10143000002CF3D09DF8070002B010BD10B5044693
:101440004FF40040FFF7DCFF042804BF00232360B3
:1014500010BD000038B504464FF400400D46FFF7BC
:10146000CFFF04280BD1064A4FF40040536823F401
:10147000807353602560BDE83840FFF7C1BF38BDB9
:10148000003C024038B504464FF400400D46FFF7DB
:10149000B7FF04281BD135B125704FF40040BDE8DB
:1014A0003840FFF7ADBFFF2324F0030504F0030429
:1014B0002968E40003FA04F421EA04042846FFF74B
:1014C000BDFF21462846BDE83840FFF7C3BF38BD01
:1014D0002DE9F0430022012703250E6807FA02F3E5
:1014E00033EA060431D14FEA420C05FA0CF4E44326
:1014F00091F804E0D0F800900EFA0CF804EA09091B
:101500000EF1FF3E48EA0908BEF1010FC0F8008065
:1015100011D8D0F808E004EA0E0E4C7904FA0CF465
:1015200044EA0E048460848824EA03048B7993409F
:101530009BB223438380C36805FA0CF423EA0404B6
:10154000CB7903FA0CF32343C3600132102AC5D1CF
:10155000BDE8F08310B50F2401F00703C90800EBC4
:101560008100016A9B009C4021EA04010162016A3A
:101570009A400A43026210BD204B10B59A6802F0EF
:101580000C020C2A30D8DFE802F02F2F2F2F072F64
:101590002F2F072F2F2F2000194B184A0360936815
:1015A0001849C3F30313CC5C0368E34043609468B9
:1015B000C4F302240C5D23FA04F484609268C2F33D
:1015C000C2228A5CD340C36010BD99680E4CC1F33F
:1015D00083419A68615C9B68094BC2F381524B431B
:1015E0000132B3FBF2F3D8E74FF400425B68C3F378
:1015F0004233013302FA03F3CFE700BF0038024061
:101600000024F4003C0300204C030020044BDA6962
:1016100011B11043D861704722EA0000FAE700BF19
:1016200000380240044B1A6A11B110431862704727
:1016300022EA0000FAE700BF00380240044B5A6972
:1016400011B110435861704722EA0000FAE700BF69
:10165000003802404309012B054B00F01F000CBF6E
:101660001B685B6B23FA00F000F00100704700BFBD
:1016700000380240024A536B43F080735363704753
:1016800000380240002382B00193054B0193019B77
:1016900003EB80000190019B196002B0704700BF0E
:1016A00050280040002382B00193054B0193019B19
:1016B00003EB80000190019B186802B0704700BFE7
:1016C0005028004030B50D460446028AEB8892B29D
:1016D00022F440521A43898902828389288923F49B
:1016E000B052AB8822F00C020343688985B00343F3
:1016F0001343A381A38A68469BB223F440730B4330
:10170000A382FFF739FFDDE90231154A944218BF81
:1017100019461923A2894B43296810044CBF49007C
:101720008900B3FBF1F16425B1FBF5F3A28918013F
:10173000120405FB13130BD5DA003232B2FBF5F2BB
:1017400002F0070242EA00039BB2238105B030BDDC
:101750001B013233B3FBF5F303F00F030343F3E74D
:1017600000380140838919B143F4005383817047E5
:1017700023F400531B041B0CF8E7C1F3080181801C
:1017800070478088C0F30800704701F01F0310B550
:10179000C1F342140121012C01FA03F105D10C30EF
:1017A00003683AB11943016010BD022C0CBF103020
:1017B0001430F5E723EA0101F5E70388194214BF65
:1017C0000120002070470123C1F3421210B5012A05
:1017D00001F01F0403FA04F30DD18289134002883B
:1017E00092B26BB10123090A03FA01F10A4214BF54
:1017F0001846002010BD022A0CBF028A828AEDE73B
:101800001846F7E70B0A01219940C94389B20180C4
:10181000704700002DE9F3411F46002304460D46A2
:10182000019316461AB9012002B0BDE8F08140F6D6
:10183000FF7301934FF40031204600F04CFD002867
:1018400052D10121204600F016FD4FF2FF712046D3
:1018500000F02AFD0121204600F0F7FC40F6FF735E
:10186000DFF8AC8101934146204600F029FD0028B5
:1018700041D039460122204600F008FD40F6FF73B2
:101880005F4F01933946204600F025FD002838D0EF
:10189000012E42D10021204600F0EDFCF0F78AFF36
:1018A00031462046238B00F0DBFCF0F7A3FF40F627
:1018B000FF73544E01933146204600F00CFD30B3C7
:1018C000204600F0EEFC287040F6FF734E4D019369
:1018D0002946204600F0FFFC0028A4D0019B5A1E98
:1018E0000192002BF4D104E0019B5A1E0192002BBF
:1018F000A0D1002098E7019B5A1E0192002BB2D183
:10190000F7E7019B5A1E0192002BBBD1F1E7019B27
:101910005A1E0192002BCED1EBE7022E25D1F0F713
:1019200049FF4FF40061204600F0BEFC0021204634
:1019300000F0A1FC238BF0F75DFF40F6FF73334E00
:1019400001933146204600F0C6FC40B101212046FB
:1019500000F086FC238A2B70238A6B70B4E7019B0E
:101960005A1E0192002BECD1C3E740F6FF77033EED
:10197000238BDFF898802E44B542019728D1234E5F
:101980003146204600F0A7FC70B30021204600F04D
:1019900072FC204600F085FC40F6FF731B4E287059
:1019A00001933146204600F096FC18B301212046F1
:1019B00000F056FC204600F074FC6870204600F0F1
:1019C00070FCA87080E7019B5A1E0192002B90D0FA
:1019D0004146204600F07FFC0028F4D0204600F06D
:1019E00060FC05F8010BC7E7019B5A1E0192002B12
:1019F000C6D17EE7019B5A1E0192002BD1D178E718
:101A00000200001040000010100000100400001040
:101A1000010003002DE9F3411E460023019340F627
:101A2000FF7304460D4617460193002A00F081809B
:101A30004FF40031204600F04EFC002842D1012135
:101A4000204600F002FC40F6FF73DFF87C81019332
:101A50004146204600F034FC00283CD031460022AC
:101A6000204600F013FC40F6FF73534E01933146BD
:101A7000204600F025FC002833D0297820466E1C33
:101A800000F00DFC3D4440F6FF77DFF83081AE42B8
:101A9000019731D1494D2946204600F01CFC002811
:101AA00036D02046012100F0DBFB40F6FF73444DA9
:101AB000444C01932946204600F00DFC00282DD10E
:101AC000012005E0019B5A1E0192002BB0D100209D
:101AD00002B0BDE8F081019B5A1E0192002BB7D1E4
:101AE000F5E7019B5A1E0192002BC0D1EFE7019B45
:101AF0005A1E0192002BEAD04146204600F0EBFB33
:101B00000028F4D016F8011B204600F0C8FBBEE701
:101B1000019B5A1E0192002BBDD1D8E7019B5A1E92
:101B20000192002BC6D1D2E7019B5A1E0192002BD5
:101B3000CDD04FF40031204600F0CDFB0028F3D18A
:101B40000121204600F081FB40F6FF731E4D0193FA
:101B50002946204600F0B4FB10B30022314620464F
:101B600000F094FB40F6FF73134D01932946204685
:101B700000F0A6FBD0B12046012100F071FB40F639
:101B8000FF730F4D0F4C01932946204600F0A3FB35
:101B9000002895D0019B5A1E0192002BF4D196E7A4
:101BA000019B5A1E0192002BD2D190E7019B5A1E35
:101BB0000192002BDAD18AE78200070004000010AE
:101BC0001000001000540040010003002DE9F34113
:101BD0001E46002304460D46019317461AB90120FC
:101BE00002B0BDE8F08140F6FF7301934FF400317D
:101BF000204600F070FB002837D10121204600F07C
